:100000000C9455470C9476470C944AD10C9476473F
:100010000C9476470C9476470C9476470C9476476C
:100020000C9476470C9476470C9476470C9475D3D1
:100030000C9476470C9476470C9406B40C9476474F
:100040000C9476470C9476470C9476470C9476473C
:100050000C9476470C9476470C9476470C9476472C
:100060000C9476470C9464D10C94F3D00C9476479E
:100070000C94C7CA0C9469CA0C94A5CA0C94764710
:100080000C9415D20C9476470C9476470C947647D2
:100090000C9476470C9476470C9476470C947647EC
:1000A0000C9476470C9476470C9476470C94E1BAFE
:1000B0000C9485BB0C9476470C9476470C94F7B55A
:1000C0000C9476470C9476470C9476470C947647BC
:1000D0000C9476470C9476470C9476470C947647AC
:1000E0000C947EA50C9476470C9476470C94764736
:1000F0000C9476470C9476470C9476470C9476478C
:100100000C94B8BA0C945CBB0C948FBA0C9433BBAF
:100110000C9476470C9476470C9476470C9476476B
:100120000C9476470C9476470C9476470C9476475B
:100130000C9476470C945BB50C9476470C947647F8
:100140000C9476470C9476470C9476470C9476473B
:100150000C9476470C9476470C9474A50C947647CF
:100160000C9476470C9476470C9476470C9476471B
:100170000C9476470C9476470C9476470C9476470B
:100180000C9476470C9476470C9476470C947647FB
:100190000C9476470C9476470C9476470C947647EB
:1001A0000C940ABB0C94AEBB0C9476470C94764727
:1001B0000C94A9B50C9476470C9476470C9476472A
:1001C0000C9476470C9476470C9476470C947647BB
:1001D0000C9476470C9476470C9476470C947647AB
:1001E0000C9476470C947647097113711D71277131
:1001F0003271387738773877387738773871387799
:10020000387738773877387738773A7144714E7164
:100210005871627138773877387738773877387728
:100220006C713877C27138773877387738773877A4
:1002300038773877017238771D753877387738779F
:10024000387738773877387738771D753877387753
:1002500038772E7233723D724772497253725E72F2
:100260003877697238773877A67238773877387781
:100270003877387738773877387738773877387706
:100280003877387738773877B07238773877387783
:10029000387738773877387738773877BA72F772AF
:1002A00034737D738773A073A073AA73B473BE7322
:1002B000C873D273D773E173EB73367736773677BB
:1002C00036773677367736773677367736773677C6
:1002D00036773677367736773677367736773677B6
:1002E0003677AA7336773677367736773677367736
:1002F0003677367736773677367736773677367796
:10030000367736773677F573FF730974137436775B
:100310003677367736773677367736773677A0730F
:10032000C376827686768E766A766E7676767A76FC
:100330009A76AF76B776BB76BF761B7792768E7459
:100340009F74B074387738772874FA703877C1742E
:10035000D274E3741D7591730575387739743877E5
:10036000F4744A741D743877387738775B746C741A
:100370007D7428BA30BA38BA40BA48BA50BA58BAB6
:1003800060BA4BBDB0BCB8BCC0BCC8BCD0BCD8BC4B
:10039000E0BCE8BCF0BCF8BC00BD08BD10BD18BD99
:1003A00030BD30BD30BD30BD30BD30BD30BD30BDE5
:1003B00030BD30BD30BD30BD30BD30BD30BD30BDD5
:1003C00030BD30BD30BD30BD30BD30BD30BD30BDC5
:1003D00030BD30BD30BD30BD30BD30BD30BD30BDB5
:1003E00030BD30BD30BD20BD28BD084AD73B3BCE17
:1003F000016E84BCBFFDC12F3D6C74319ABD568324
:100400003DDA3D00C77F11BED9E4BB4C3E916BAADB
:10041000AABE000000803F05A84CCDB2D44EB9382A
:1004200036A9020C50B9918688083CA6AAAA2ABE11
:10043000000000803F07634236B79BD8A71A39688F
:100440005618AEBAAB558C1D3CB7CC5763BD6DED9D
:10045000FD753EF6177231BF000000803F080000B6
:1004600000BE922449123EABAAAA2ABECDCCCC4CE7
:100470003E00000080BEABAAAAAA3E00000000BF5A
:10048000000000803F0000000000084178D3BB431B
:1004900087D1133D190E3CC3BD4282AD2B3E68ECA3
:1004A0008276BED98FE1A93E4C80EFFFBE01C4FF2A
:1004B0007F3F0000000000000C9432AD0C94D55634
:1004C0000C9428BD0C94E7560C94A1630C940AC1BB
:1004D0000C94D3A60C9486760C9413740C9416CAC0
:1004E0000C9460BA0C94955A0C942E720C94DBB94F
:1004F0000C9430BD0C94B7760C948F5B0C94C17443
:100500000C946D5A0C94ED560C9448CF0C94715A7F
:100510000C9444710C94FFB90C9418BD0C9405759F
:100520000C945B5B0C941B680C94EA5D0C9440BAD1
:100530000C948C470C9409710C9438770C94F8BC8B
:100540000C9482470C94FE560C94FFC10C94915964
:100550000C94095F0C94A15A0C9485570C9480BCA0
:100560000C9478470C943E5D0C94DFA60C944E716D
:100570000C9458710C944BBD0C942EAD0C94625D90
:100580000C946D630C94B9590C94855A0C94CC63FB
:100590000C94915A0C947B5B0C94DB560C9420BD0C
:1005A0000C94EB730C941D570C94F2AC0C94AF7636
:1005B0000C94DCCC0C94C8790C94F3B90C94616E57
:1005C0000C94DA910C942ECE0C947D740C943D72A4
:1005D0000C94775B0C94D05A0C9458BA0C943E57F8
:1005E0000C94E94A0C9427710C948D5A0C941E5863
:1005F0000C9449720C94AB590C94C8560C949D5AA7
:100600000C94735B0C949A580C94E8BC0C940EAD4B
:100610000C9409570C941D710C94A95E0C942154F0
:100620000C94E1560C94F76C0C94E3740C94A55A5A
:100630000C9439740C948E740C941A630C94675B4C
:100640000C94FBB90C943C640C94DFB90C941B6BB8
:100650000C94E8780C9457570C94EF5A0C94A5839B
:100660000C9428570C94B15A0C94C3760C94017FC7
:100670000C94CB470C942AAD0C94655A0C9470786A
:100680000C9438BA0C94D2740C94F4570C94CBA6F6
:100690000C94DDAC0C9465CE0C94F7720C943A710A
:1006A0000C9448BA0C94A0730C948AAE0C94FF730B
:1006B0000C94CE670C9400BD0C9499AB0C943271E1
:1006C0000C9436AD0C9495AB0C94A36E0C94126301
:1006D0000C946C710C9487580C949F740C94E4B92E
:1006E0000C94E3A60C9448680C947ABC0C94477262
:1006F0000C9493AB0C94E6590C94236B0C941E63EE
:100700000C9453720C94B0720C94795A0C94C8BC2B
:100710000C945D680C949AB80C94C7A60C94C059BC
:100720000C9482760C94D2730C94DA6D0C9408BD00
:100730000C94AA730C9480B90C94DBA60C947F5B88
:100740000C940ACC0C9472790C9416630C94E8C641
:100750000C94575B0C94C7590C94F0BC0C947D73AB
:100760000C94DC470C942CB90C941A5D0C94C8734F
:100770000C944A740C94BF760C94C05C0C94F07882
:100780000C9487730C946A760C94C0BC0C94C25D74
:100790000C94707F0C94975B0C94805E0C94605961
:1007A0000C948A770C9433790C94D05E0C9462711B
:1007B0000C9470CD0C94935B0C94C45D0C94815A92
:1007C0000C94B0740C9469720C9488670C949660C5
:1007D0000C942DC70C9401720C9422C10C9461AE40
:1007E0000C946E760C94FA700C947A760C944B817F
:1007F0000C9413710C9436770C9428740C94C8786C
:100800000C9409C10C94A5C90C9417C90C94CE681A
:100810000C94055A0C9433720C94895D0C943473C7
:100820000C94BE730C94595E0C94B4730C94F474D1
:100830000C948EB80C945B740C9418B90C940F5EE5
:100840000C94BD570C94615A0C94165D0C945E7216
:100850000C9473620C94A8B90C9409740C94695AA2
:100860000C9459AB0C94A35B0C94755A0C945BAB31
:100870000C94AE5B0C94D0BC0C9453630C94BB767C
:100880000C94895A0C945BC10C9457620C9446B931
:100890000C9428BA0C94D7B90C94C1620C94345EB1
:1008A0000C94B8BC0C94A95A0C941D740C94125757
:1008B0000C9433570C9430BA0C949ABC0C94835B10
:1008C0000C9408590C9422630C9404CA0C94C378B9
:1008D0000C94F4780C94F3560C9405670C949D7961
:1008E0000C94E4CE0C94995A0C9450BA0C94C3A670
:1008F0000C94B0BC0C9492760C94F7B90C94747F61
:100900000C94E0BC0C94D7730C94F56D0C94D7A6A2
:100910000C9491730C9493D00C9410BD0C94F878B3
:100920000C941D750C9404640C94DCCD0C943EC1A5
:100930000C94624E0C948B5B0C94635B0C94125B76
:100940000C947D5A0C948C590C94AD5A0C94D8BCD0
:100950000C946B5B0C94875B0C94A6720C94F35A0A
:100960000C946C740C9476760C9487630C946E578C
:100970000C949A760C94CFA60C949EBC0C94BA72EC
:100980000C94FD670C948E760C9438710C946F5B0C
:100990000C945F5B0C94787F0C94EC780C94E1736E
:1009A0000C945DAB0C9457580C94F5730C947A77B7
:1009B0000C94B2590C94C2710C9484C90C9482B8F2
:1009C0000C94E7A60C941B770C94CAA75B2573259F
:1009D000735D20257320257320706F736974696FB0
:1009E0006E2531382E336625730A005B2573257317
:1009F0005D202573202573206F666673657425322C
:100A0000302E336625730A005B257325735D202520
:100A100073207A65726F206261636B6F6666253141
:100A2000392E336625730A005B257325735D2025F7
:100A300073206C61746368206261636B6F66662506
:100A400031382E336625730A005B257325735D20CC
:100A50002573206C617463682076656C6F636974BC
:100A6000792531332E306625732F6D696E0A005B50
:100A7000257325735D20257320736561726368207B
:100A800076656C6F636974792531322E3066257313
:100A90002F6D696E0A005B257325735D2025732019
:100AA000737769746368206D617825313764205BE2
:100AB000303D6F66662C313D686F6D696E672C3214
:100AC0003D6C696D69742C333D6C696D69742B687C
:100AD0006F6D696E675D0A005B257325735D202568
:100AE0007320737769746368206D696E253137648C
:100AF000205B303D6F66662C313D686F6D696E67B7
:100B00002C323D6C696D69742C333D6C696D697470
:100B10002B686F6D696E675D0A005B257325735DD9
:100B2000202573207261646975732076616C756528
:100B30002532302E346625730A005B257325735DDC
:100B4000202573206A756E6374696F6E2064657604
:100B5000696174696F6E2531342E346625732028DF
:100B60006C61726765722069732066617374657267
:100B7000290A005B257325735D202573206A657241
:100B80006B20686F6D696E672531362E3066257370
:100B90002F6D696E5E33202A2031206D696C6C697F
:100BA0006F6E0A005B257325735D202573206A65CF
:100BB000726B206D6178696D756D2531352E3066EB
:100BC00025732F6D696E5E33202A2031206D696C8C
:100BD0006C696F6E0A005B257325735D2025732099
:100BE00074726176656C206D696E696D756D253105
:100BF000372E336625730A005B257325735D202528
:100C0000732074726176656C206D6178696D756DA5
:100C10002531372E336625730A005B257325735DF6
:100C20002025732076656C6F63697479206D617817
:100C3000696D756D2531312E306625732F6D696EA6
:100C40000A005B257325735D202573206665656446
:100C500072617465206D6178696D756D2531312E15
:100C6000306625732F6D696E0A005B257325735DF1
:100C70002025732061786973206D6F646525313894
:100C8000642025730A005B6D615D20206D696E2014
:100C9000617263207365676D656E742531382E331C
:100CA0006625730A005B736C5D2020736F66742089
:100CB0006C696D697420656E61626C6525313264A2
:100CC0000A005B63745D202063686F7264616C204E
:100CD000746F6C6572616E63652531372E346625DD
:100CE000730A005B6A615D20206A756E6374696FC8
:100CF0006E20616363656C65726174696F6E25381F
:100D00002E306625730A005B6764695D2064656642
:100D100061756C742067636F6465206469737461C6
:100D20006E6365206D6F6465253264205B303D47DE
:100D300039302C313D4739315D0A005B6770615DA8
:100D40002064656661756C742067636F64652070EC
:100D500061746820636F6E74726F6C253364205BFE
:100D6000303D4736312C313D4736312E312C323D26
:100D70004736345D0A005B67636F5D2064656661BA
:100D8000756C742067636F646520636F6F72642095
:100D900073797374656D253364205B312D3620289B
:100DA0004735342D473539295D0A005B67756E5D1F
:100DB0002064656661756C742067636F6465207577
:100DC0006E697473206D6F6465253564205B303DFA
:100DD0004732302C313D4732315D0A005B67706C21
:100DE0005D2064656661756C742067636F6465205F
:100DF000706C616E6525313064205B303D47313762
:100E00002C313D4731382C323D4731395D0A0025C0
:100E10006320776F726B206F66667365743A253155
:100E2000322E336625730A002563206D616368697D
:100E30006E6520706F736E3A2531312E33662573DF
:100E40000A00256320706F736974696F6E3A2531EB
:100E5000352E336625730A00546F6F6C206E756DE6
:100E60006265722020202020202020202025640A76
:100E700000466565642072617465206D6F64653A33
:100E800020202020202025730A0044697374616E9D
:100E90006365206D6F64653A202020202020202586
:100EA000730A0050617468204D6F64653A202020F9
:100EB000202020202020202025730A00506C616E05
:100EC000653A2020202020202020202020202020C3
:100ED0002025730A004D6F74696F6E206D6F646515
:100EE0003A20202020202020202025730A00436F54
:100EF0006F7264696E6174652073797374656D3A9D
:100F000020202025730A00556E6974733A20202032
:100F100020202020202020202020202025730A00AF
:100F2000486F6D696E672073746174653A20202084
:100F3000202020202025730A0046656564686F6CB8
:100F4000642073746174653A20202020202025736A
:100F50000A004D6F74696F6E2073746174653A2076
:100F60002020202020202025730A004379636C650F
:100F70002073746174653A202020202020202020D6
:100F800025730A00526177206D616368696E652080
:100F900073746174653A20202025730A004D6163E3
:100FA00068696E652073746174653A202020202082
:100FB000202025730A004C696E65206E756D626590
:100FC000723A2531302E30660A004665656420721B
:100FD0006174653A2531362E336625732F6D696E3F
:100FE0000A0056656C6F636974793A2531372E3380
:100FF0006625732F6D696E0A0050101F10FF0F4792
:101000003935202D20756E6974732D7065722D72BF
:1010100065766F6C7574696F6E206D6F64650047DF
:101020003934202D20756E6974732D7065722D6DA5
:10103000696E757465206D6F64652028692E652E54
:10104000206665656472617465206D6F6465290052
:10105000473933202D20696E766572736520746977
:101060006D65206D6F6465008C106C104739312000
:101070002D20696E6372656D656E74616C206469A4
:101080007374616E6365206D6F646500473930204D
:101090002D206162736F6C7574652064697374616F
:1010A0006E6365206D6F646500DD10C510AF10477D
:1010B0003634202D20636F6E74696E756F757320E2
:1010C0006D6F6465004736312E31202D20657861C3
:1010D00063742073746F70206D6F646500473631E0
:1010E000202D2065786163742070617468206D6FB5
:1010F00064650017110811F910473139202D205966
:101100005A20706C616E6500473138202D20585A86
:1011100020706C616E6500473137202D20585920B2
:10112000706C616E6500A311911178115711301127
:10113000473830202D2063616E63656C206D6F74BD
:10114000696F6E206D6F646520286E6F6E6520611B
:1011500063746976652900473320202D20636F75FD
:101160006E74657220636C6F636B77697365206161
:101170007263206665656400473220202D20636C11
:101180006F636B7769736520617263206665656460
:1011900000473120202D206C696E656172206665E4
:1011A000656400473020202D206C696E65617220D7
:1011B000747261766572736520287365656B2900AA
:1011C0006A12501236121C120212E811CE11473563
:1011D00039202D20636F6F7264696E6174652073AE
:1011E000797374656D203600473538202D20636F84
:1011F0006F7264696E6174652073797374656D20B4
:101200003500473537202D20636F6F7264696E613A
:1012100074652073797374656D203400473536200A
:101220002D20636F6F7264696E61746520737973CA
:1012300074656D203300473535202D20636F6F7244
:1012400064696E6174652073797374656D20320012
:10125000473534202D20636F6F7264696E61746549
:101260002073797374656D203100473533202D204C
:101270006D616368696E6520636F6F7264696E612A
:1012800074652073797374656D009D1297129012C6
:10129000486F6D696E6700486F6D6564004E6F74CE
:1012A00020486F6D656400D112CC12C712C112BC08
:1012B00012B312456E6420486F6C6400486F6C6412
:1012C00000446563656C00506C616E0053796E6319
:1012D000004F666600E412E012DB12486F6C640097
:1012E00052756E0053746F70000E130413FE12F7E4
:1012F00012F3124A6F6700486F6D696E6700507293
:101300006F6265004D616368696E696E67004F6664
:10131000660044133E13381333132F13291320137D
:1013200053687574646F776E004379636C6500452C
:101330006E640053746F7000416C61726D00526591
:1013400061647900496E697469616C697A696E6774
:1013500000A713A1139B13961392138E1389138363
:10136000137D1376137213691353687574646F7762
:101370006E004A6F6700486F6D696E67004379635E
:101380006C650050726F626500486F6C6400527546
:101390006E00456E640053746F7000416C61726D35
:1013A00000526561647900496E697469616C697A9B
:1013B000696E6700CE13B813473231202D206D6956
:1013C0006C6C696D65746572206D6F646500473281
:1013D00030202D20696E63686573206D6F64650031
:1013E0000814FD13F113E8135B7261646975735D92
:1013F000005B696E686962697465645D005B737443
:10140000616E646172645D005B64697361626C65E6
:10141000645D0022141E1419142064656700206D99
:101420006D0020696E002A2A2A204E4F54494345F8
:10143000202A2A2A20526573657474696E672062B7
:10144000617564207261746520746F202573005B80
:10145000626175645D20555342206261756420723B
:1014600061746525313564205B313D393630302C6F
:10147000323D31393230302C333D33383430302C3A
:10148000343D35373630302C353D31313532303022
:101490002C363D3233303430305D0A005B72786D6B
:1014A0005D2073657269616C205258206D6F6465B0
:1014B00025313564205B303D636861725F6D6F6418
:1014C000652C313D6C696E655F6D6F64655D0A000A
:1014D0005B65785D2020656E61626C6520666C6F6F
:1014E0007720636F6E74726F6C25313064205B30CF
:1014F0003D6F66662C313D584F4E2F584F46462C57
:10150000323D5254532F4354535D0A005B65655D71
:101510002020656E61626C65206563686F253138D7
:1015200064205B303D6F66662C313D6F6E5D0A0056
:101530005B65635D2020657870616E64204C462099
:10154000746F2043524C46206F6E205458253664E9
:10155000205B303D6F66662C313D6F6E5D0A0092F8
:10156000158D15871581157B1574156D1532333062
:1015700034303000313135323030003537363030AC
:1015800000333834303000313932303000393630C1
:1015900030003000737973006662000000000702BB
:1015A000E878895DC25DE0390020DC43737973001F
:1015B0006676000000000703EC78895DC25DE439BF
:1015C000EC51783F737973006870000000000700E9
:1015D000F078895DD05EEC390000803F737973004C
:1015E0006876000000000700F478895DC878F0395B
:1015F000000000417379730069640000000004007A
:10160000F8787078C25DDC3900000000000000004E
:101610006E00000000000100615A5757805E5B3287
:1016200000000000000000006C696E650000010011
:10163000615A6E57805E5B320000000000000000BF
:1016400076656C0000000002C7598557C25DDC3921
:1016500000000000000000006665656400000002F4
:10166000E659BD57C25DDC390000000000000000F3
:101670007374617400000000655AC856C25DDC399D
:1016800000000000000000006D61637300000000B6
:10169000695AD556C25DDC39000000000000000028
:1016A00063796373000000006D5ADB56C25DDC395C
:1016B00000000000000000006D6F74730000000067
:1016C000715AE156C25DDC390000000000000000E4
:1016D000686F6C6400000000755AE756C25DDC3923
:1016E0000000000000000000756E6974000000003A
:1016F0007D5AF356C25DDC39000000000000000096
:10170000636F6F7200000000815AFE56C25DDC39C3
:1017100000000000000000006D6F6D6F0000000011
:10172000855A0957C25DDC39000000000000000046
:10173000706C616E00000000895A1257C25DDC397E
:1017400000000000000000007061746800000000EC
:101750008D5A1D57C25DDC390000000000000000FA
:101760006469737400000000915A2857C25DDC3927
:10177000000000000000000066726D6F00000000B5
:10178000955A3357C25DDC390000000000000000AC
:10179000746F6F6C00000000995A3E57C25DDC39CF
:1017A000000000006D706F006D706F780000000326
:1017B000A35B1E58C25DDC39000000006D706F0035
:1017C0006D706F7900000003A35B1E58C25DDC39A9
:1017D000000000006D706F006D706F7A00000003F4
:1017E000A35B1E58C25DDC39000000006D706F0005
:1017F0006D706F6100000003A35B1E58C25DDC3991
:10180000000000006D706F006D706F6200000003DB
:10181000A35B1E58C25DDC39000000006D706F00D4
:101820006D706F6300000003A35B1E58C25DDC395E
:1018300000000000706F7300706F73780000000389
:10184000975BF457C25DDC3900000000706F7300D5
:10185000706F737900000003975BF457C25DDC3949
:1018600000000000706F7300706F737A0000000357
:10187000975BF457C25DDC3900000000706F7300A5
:10188000706F736100000003975BF457C25DDC3931
:1018900000000000706F7300706F7362000000033F
:1018A000975BF457C25DDC3900000000706F730075
:1018B000706F736300000003975BF457C25DDC39FF
:1018C000000000006F6673006F667378000000030D
:1018D000AE5B5758C25DDC39000000006F667300D4
:1018E0006F66737900000003AE5B5758C25DDC3948
:1018F000000000006F6673006F66737A00000003DB
:10190000AE5B5758C25DDC39000000006F667300A3
:101910006F66736100000003AE5B5758C25DDC392F
:10192000000000006F6673006F66736200000003C2
:10193000AE5B5758C25DDC39000000006F66730073
:101940006F66736300000003AE5B5758C25DDC39FD
:1019500000000000686F6D00686F6D65000000009A
:10196000795AED569159DC3900000000686F6D001E
:10197000686F6D7800000000975B1A5DC25D3032C1
:1019800000000000686F6D00686F6D790000000056
:10199000975B1A5DC25D313200000000686F6D0018
:1019A000686F6D7A00000000975B1A5DC25D32328D
:1019B00000000000686F6D00686F6D61000000003E
:1019C000975B1A5DC25D333200000000686F6D00E6
:1019D000686F6D6200000000975B1A5DC25D343273
:1019E00000000000686F6D00686F6D63000000000C
:1019F000975B1A5DC25D35320000000070726200B4
:101A0000707262650000000009C11A5DC25D363265
:101A100000000000707262007072627800000003C3
:101A200009C1895DC25D373200000000707262003A
:101A3000707262790000000309C1895DC25D3B32AA
:101A400000000000707262007072627A0000000391
:101A500009C1895DC25D3F32000000007072620002
:101A6000707262610000000309C1895DC25D43328A
:101A70000000000070726200707262620000000379
:101A800009C1895DC25D47320000000070726200CA
:101A9000707262630000000309C1895DC25D4B3250
:101AA000000000006A6F67006A6F6778000000003E
:101AB00009C1165DAB595532000000006A6F67001E
:101AC0006A6F67790000000009C1165DB25955328E
:101AD000000000006A6F67006A6F677A000000000C
:101AE00009C1165DB9595532000000006A6F6700E0
:101AF0006A6F67610000000009C1165DC059553268
:101B000000000000707772007077723100000000F2
:101B1000FFB92CB9C25DDC3900000000707772009B
:101B20007077723200000000FFB92CB9C25DDC3959
:101B300000000000707772007077723300000000C0
:101B4000FFB92CB9C25DDC3900000000707772006B
:101B50007077723400000000FFB92CB9C25DDC3927
:101B60000000000031000000316D61000000030042
:101B7000DBB91A5DC45D3058000040403100000000
:101B80003173610000000303DFB9895D82B83B58FF
:101B90006666E63F310000003174720000000B04FD
:101BA000E4B9895D8EB83F580000B44331000000AD
:101BB000316D690000000300F3B91A5D9AB831581D
:101BC000000000413100000031706F000000030090
:101BD000F7B91A5DEA5D35580000803F310000001A
:101BE00031706D0000000300FBB91A5D18B936585A
:101BF0000000004032000000326D61000000030070
:101C0000DBB91A5DC45D4F5800000040320000008F
:101C10003273610000000303DFB9895D82B85A584E
:101C20006666E63F320000003274720000000B046A
:101C3000E4B9895D8EB85E585C8F224132000000A5
:101C4000326D690000000300F3B91A5D9AB850586C
:101C5000000000413200000032706F0000000300FD
:101C6000F7B91A5DEA5D54580000803F3200000069
:101C700032706D0000000300FBB91A5D18B95558A9
:101C80000000004033000000336D610000000300DD
:101C9000DBB91A5DC45D6E580000803F3300000060
:101CA0003373610000000303DFB9895D82B879589E
:101CB0006666E63F330000003374720000000B04D8
:101CC000E4B9895D8EB87D585C8F224133000000F5
:101CD000336D690000000300F3B91A5D9AB86F58BC
:101CE000000000413300000033706F00000003006B
:101CF000F7B91A5DEA5D73580000803F33000000B9
:101D000033706D0000000300FBB91A5D18B97458F8
:101D10000000004034000000346D6100000003004A
:101D2000DBB91A5DC45D8D5800000000340000006E
:101D30003473610000000303DFB9895D82B89858ED
:101D40006666E63F340000003474720000000B0445
:101D5000E4B9895D8EB89C585C8F22413400000044
:101D6000346D690000000300F3B91A5D9AB88E580B
:101D7000000000413400000034706F0000000300D8
:101D8000F7B91A5DEA5D92580000000034000000C7
:101D900034706D0000000300FBB91A5D18B9935848
:101DA000000000407800000078616D000000030032
:101DB000125B87589A58EC300000803F7800000092
:101DC00078766D0000000B005B5B895DC162F130CD
:101DD0000080BB44780000007866720000000B00B1
:101DE000575B895DC162ED300080BB447800000024
:101DF00078746E0000000B03635B895DC162F9308B
:101E0000000000007800000078746D0000000B03F3
:101E10005F5B895DC162F53000000A437800000015
:101E2000786A6D0000000B00675B895D0859FD3022
:101E30000000FA4378000000786A680000000B0098
:101E40006B5B895D6059013100007A4478000000C5
:101E5000786A640000000B046F5B895DC162093120
:101E60000AD7233C7800000078736E00000003005E
:101E7000775B1A5D80BC10300000803F7800000066
:101E800078737800000003007B5B1A5D80BC113022
:101E900000000000780000007873760000000B005E
:101EA0007F5B895DC16211310000FA437800000058
:101EB000786C760000000B00835B895DC162153190
:101EC0000000C84178000000786C620000000B033D
:101ED000875B895DC16219310000A0407800000075
:101EE000787A620000000B038B5B895DC1621D3153
:101EF000000000007900000079616D00000003001F
:101F0000125B87589A5821310000803F7900000009
:101F100079766D0000000B005B5B895DC162263144
:101F20000080BB44790000007966720000000B005D
:101F3000575B895DC16222310080BB44790000009B
:101F400079746E0000000B03635B895DC1622E3102
:101F5000000000007900000079746D0000000B03A0
:101F60005F5B895DC1622A310000E64279000000B2
:101F7000796A6D0000000B00675B895D085932319A
:101F80000000FA4379000000796A680000000B0045
:101F90006B5B895D6059363100007A44790000003E
:101FA000796A640000000B046F5B895DC1623E3199
:101FB0000AD7233C7900000079736E00000003000B
:101FC000775B1A5D80BC12300000803F7900000012
:101FD00079737800000003007B5B1A5D80BC1330CE
:101FE00000000000790000007973760000000B000B
:101FF0007F5B895DC16246310000FA4379000000D1
:10200000796C760000000B00835B895DC1624A3108
:102010000000C84179000000796C620000000B03E9
:10202000875B895DC1624E310000A04079000000ED
:10203000797A620000000B038B5B895DC1625231CB
:10204000000040407A0000007A616D00000003004B
:10205000125B87589A5856310000803F7A00000082
:102060007A766D0000000B005B5B895DC1625B31BD
:102070000080BB447A0000007A66720000000B000A
:10208000575B895DC16257310080BB447A00000014
:102090007A746E0000000B03635B895DC16263317B
:1020A00000008CC27A0000007A746D0000000B03FF
:1020B0005F5B895DC1625F31000000007A00000053
:1020C0007A6A6D0000000B00675B895D0859673113
:1020D0000000FA437A0000007A6A680000000B00F2
:1020E0006B5B895D60596B3100007A447A000000B7
:1020F0007A6A640000000B046F5B895DC162733112
:102100000AD7233C7A0000007A736E0000000300B7
:10211000775B1A5D80BC1430000000007A0000007C
:102120007A737800000003007B5B1A5D80BC153079
:102130000000803F7A0000007A73760000000B00F8
:102140007F5B895DC1627B310000FA437A00000049
:102150007A6C760000000B00835B895DC1627F3181
:102160000000C8417A0000007A6C620000000B0396
:10217000875B895DC16283310000A0407A00000066
:102180007A7A620000000B038B5B895DC162873144
:10219000000000006100000061616D0000000300AC
:1021A000125B87589A588B31000040406100000054
:1021B00061766D00000003005B5B895DD05E90314D
:1021C0000000B4446100000061667200000003007A
:1021D000575B895DD05E8C310000B4446100000023
:1021E00061746E0000000303635B895DC162983116
:1021F000000080BF6100000061746D0000000303F7
:102200005F5B895DD05E9431000080BF610000009B
:10221000616A6D0000000300675B895D08599C31AD
:102220000000FA4361000000616A680000000300DA
:102230006B5B895D6059A0310000FA4361000000CA
:10224000616A6400000003046F5B895DD05EA831A1
:102250000AD7233C610000006172610000000B039B
:10226000735B895DD05EAC31CF2E654261000000AA
:1022700061736E0000000300775B1A5D80BC16304E
:102280000000803F610000006173780000000300DF
:102290007B5B1A5D80BC173000000000610000000D
:1022A00061737600000003007F5B895DD05EB03112
:1022B0000000164461000000616C7600000003001D
:1022C000835B895DD05EB4310000C84261000000CC
:1022D000616C620000000303875B895DD05EB831EA
:1022E0000000A04061000000617A6200000003036A
:1022F0008B5B895DD05EBC31000000406200000055
:1023000062616D0000000300125B87589A58C0316B
:10231000000000006200000062766D000000030013
:102320005B5B895DD05EC5310000B4446200000093
:102330006266720000000300575B895DD05EC131A8
:102340000000B4446200000062746E0000000303E9
:10235000635B895DC162CD31000080BF6200000017
:1023600062746D00000003035F5B895DD05EC9315C
:10237000000080BF62000000626A6D000000030080
:10238000675B895D0859D1310000FA4362000000A3
:10239000626A6400000003006F5B895DD05EDD311E
:1023A0000AD7233C620000006272610000000B0348
:1023B000735B895DD05EE131CF2E65426300000022
:1023C00063616D0000000300125B87589A58F53175
:1023D000000000006300000063766D000000030051
:1023E0005B5B895DD05EFA310000B444630000009D
:1023F0006366720000000300575B895DD05EF631B2
:102400000000B4446300000063746E000000030326
:10241000635B895DC1620232000080BF630000001F
:1024200063746D00000003035F5B895DD05EFE3165
:10243000000080BF63000000636A6D0000000300BD
:10244000675B895D085906320000FA4363000000AB
:10245000636A6400000003006F5B895DD05E123226
:102460000AD7233C630000006372610000000B0385
:10247000735B895DD05E1632CF2E654270310000ED
:102480007031667271000300C3A6895DD05E0C577F
:102490000000C84270310000703163736C000300AB
:1024A000C7A6895DD05E105700E0F6457031000088
:1024B0007031637368000300CBA6895DD05E14574A
:1024C0000000484670310000703163706C000303F7
:1024D000CFA6895DD05E1857B81E053E703100004A
:1024E0007031637068000303D3A6895DD05E1C570A
:1024F0007B142E3E70310000703177736C00030046
:10250000D7A6895DD05E2057000000007031000022
:102510007031777368000300DBA6895DD05E2457B5
:102520000000000070310000703177706C00030310
:10253000DFA6895DD05E2857CDCCCC3D7031000040
:102540007031777068000303E3A6895DD05E2C5775
:10255000CDCCCC3D703100007031706F660003034C
:10256000E7A6895DD05E3057CDCCCC3D67353400D1
:102570006735347800000B038F5B895DC1625C3086
:1025800000000000673534006735347900000B0324
:102590008F5B895DC16260300000000067353400E8
:1025A0006735347A00000B038F5B895DC16264304C
:1025B00000000000673534006735346100000B030C
:1025C0008F5B895DC16268300000000067353400B0
:1025D0006735346200000B038F5B895DC1626C302C
:1025E00000000000673534006735346300000B03DA
:1025F0008F5B895DC1627030000000006735350077
:102600006735357800000B038F5B895DC1627430DC
:1026100000000000673535006735357900000B0391
:102620008F5B895DC162783000000000673535003E
:102630006735357A00000B038F5B895DC1627C30A2
:1026400000000000673535006735356100000B0379
:102650008F5B895DC1628030000000006735350006
:102660006735356200000B038F5B895DC162843082
:1026700000000000673535006735356300000B0347
:102680008F5B895DC16288300000A0C1673536006C
:102690006735367800000B038F5B895DC1628C3033
:1026A00000000000673536006735367900000B03FF
:1026B0008F5B895DC1629030000000006735360095
:1026C0006735367A00000B038F5B895DC1629430F9
:1026D00000000000673536006735366100000B03E7
:1026E0008F5B895DC162983000000000673536005D
:1026F0006735366200000B038F5B895DC1629C30D9
:1027000000000000673536006735366300000B03B4
:102710008F5B895DC162A030000000006735370023
:102720006735377800000B038F5B895DC162A43089
:1027300000000000673537006735377900000B036C
:102740008F5B895DC162A8300000000067353700EB
:102750006735377A00000B038F5B895DC162AC304F
:1027600000000000673537006735376100000B0354
:102770008F5B895DC162B0300000000067353700B3
:102780006735376200000B038F5B895DC162B4302F
:1027900000000000673537006735376300000B0322
:1027A0008F5B895DC162B83000000000673538007A
:1027B0006735387800000B038F5B895DC162BC30E0
:1027C00000000000673538006735387900000B03DA
:1027D0008F5B895DC162C030000000006735380042
:1027E0006735387A00000B038F5B895DC162C430A6
:1027F00000000000673538006735386100000B03C2
:102800008F5B895DC162C830000000006735380009
:102810006735386200000B038F5B895DC162CC3085
:1028200000000000673538006735386300000B038F
:102830008F5B895DC162D0300000000067353900D0
:102840006735397800000B038F5B895DC162D43036
:1028500000000000673539006735397900000B0347
:102860008F5B895DC162D830000000006735390098
:102870006735397A00000B038F5B895DC162DC30FC
:1028800000000000673539006735396100000B032F
:102890008F5B895DC162E030000000006735390060
:1028A0006735396200000B038F5B895DC162E430DC
:1028B00000000000673539006735396300000B03FD
:1028C0008F5B895DC162E83000000000673932002B
:1028D00067393278000001038F5B895DC25DCD32BC
:1028E00000000000673932006739327900000103C7
:1028F0008F5B895DC25DD132000000006739320014
:102900006739327A000001038F5B895DC25DD53281
:1029100000000000673932006739326100000103AE
:102920008F5B895DC25DD9320000000067393200DB
:1029300067393262000001038F5B895DC25DDD3261
:10294000000000006739320067393263000001037C
:102950008F5B895DC25DE1320000000067323800A4
:102960006732387800000103935B895DC25DE53210
:102970000000000067323800673238790000010338
:10298000935B895DC25DE932000000006732380068
:102990006732387A00000103935B895DC25DED32D6
:1029A0000000000067323800673238610000010320
:1029B000935B895DC25DF132000000006732380030
:1029C0006732386200000103935B895DC25DF532B6
:1029D00000000000673238006732386300000103EE
:1029E000935B895DC25DF9320000000067333000FF
:1029F0006733307800000103935B895DC25DFD326F
:102A000000000000673330006733307900000103B5
:102A1000935B895DC25D01330000000067333000C5
:102A20006733307A00000103935B895DC25D053333
:102A3000000000006733300067333061000001039D
:102A4000935B895DC25D093300000000673330008D
:102A50006733306200000103935B895DC25D0D3313
:102A6000000000006733300067333063000001036B
:102A7000935B895DC25D1133000000006A696400E8
:102A80006A6964610000000009C1625DA95E063ADE
:102A9000000000006A6964006A6964620000000066
:102AA00009C1625DA95E0A3A000000006A6964001B
:102AB0006A6964630000000009C1625DA95E0E3AA4
:102AC000000000006A6964006A6964640000000034
:102AD00009C1625DA95E123A0000000073797300BB
:102AE0006A61000000000F00B15A895DC1622A309E
:102AF0000050C347737973006374000000000F0433
:102B0000D05A895DC1622E300AD7233C7379730095
:102B1000736C000000000700EF5A1A5DC45D32308C
:102B20000000000073797300737400000000070058
:102B30009ABC1A5D7ABC05300000803F737973003F
:102B40006D74000000000702D7B9895D46B92C58A2
:102B500000000040000000006D6500000000000063
:102B60000AC1A8B9A8B9DC390000000000000000C3
:102B70006D640000000000000AC180B980B9DC3932
:102B80000000000073797300656A00000000070010
:102B9000707F1A5DEA5DF8390000803F7379730039
:102BA0006A76000000000700747F1A5D017F9E3C7A
:102BB00000004040737973006A7300000000070052
:102BC000787F1A5DEA5DA03C0000803F7379730056
:102BD0007476000000000700FFC11A5DEA5D9F598E
:102BE0000000803F737973007176000000000700D9
:102BF00036AD1A5D345E65570000000073797300CE
:102C0000737600000000070099AB1A5D0F5E7257E3
:102C10000000803F737973007369000000000700B3
:102C200095AB3E5D5DAB735700007A4373797300DB
:102C3000656300000000070012631A5DCC63E22F99
:102C40000000000073797300656500000000070054
:102C500016631A5D3C64E32F000000007379730073
:102C600065780000000007001A631A5D0464E42F11
:102C70000000803F7379730072786D0000000700D8
:102C80001E631A5DEA5DE52F0000803F73797300D3
:102C9000626175640000040022631A5D7362E02FB4
:102CA0000000A0400000000073720000000000005F
:102CB00093AB59AB5BABDC390000000000000000B7
:102CC00071720000000000002AADDDACC25DDC398D
:102CD000000000000000000071690000000000001A
:102CE0002EADF2ACC25DDC39000000000000000037
:102CF000716F00000000000032AD0EADC25DDC3926
:102D000000000000000000006572000000000000EC
:102D100009C1CAA7C25DDC39000000000000000044
:102D2000716600000000000009C1165D8C59DC3995
:102D300000000000000000007278000000000000A9
:102D40003EC15762C25DDC39000000000000000097
:102D50006D736700000000000AC1165DC25DDC39BA
:102D60000000000000000000636C6561720000005C
:102D700009C1624E624EDC39000000000000000014
:102D8000746573740000000009C172799EBCDC395F
:102D900000000000000000006465666100000000A3
:102DA00009C19D79C05CDC39000000000000000012
:102DB000626F6F740000000009C1C879C378DC3904
:102DC000000000000000000068656C70000000005A
:102DD00009C13379C25DDC39000000000000000049
:102DE000680000000000000009C13379C25DDC39D1
:102DF000000000007379730067706C00000007002A
:102E00009D5A1A5D0F5E4030000000007379730018
:102E100067756E0000000700A15A1A5DEA5D413037
:102E20000000803F7379730067636F000000070044
:102E3000A55A1A5DC45D3F300000004073797300ED
:102E40006770610000000700A95A1A5D0F5E4230EA
:102E50000000004073797300676469000000070098
:102E6000AD5A1A5DEA5D433000000000000000002A
:102E7000676300000000000009C17A778A77DC39B7
:102E800000000000000000006D61000000000B0465
:102E9000F35A895DC1623730CDCCCC3D00000000D3
:102EA000666400000000030022C11A5DEA5D9F3CD9
:102EB000000000007564610075646130000003006B
:102EC0003EC1625DA95E9839000000007564610032
:102ED00075646131000003003EC1625DA95E9C39EA
:102EE0000000000075646100756461320000030039
:102EF0003EC1625DA95EA0390000000075646100FA
:102F000075646133000003003EC1625DA95EA439AF
:102F10000000000075646200756462300000030008
:102F20003EC1625DA95EA8390000000075646200C0
:102F300075646231000003003EC1625DA95EAC3978
:102F400000000000756462007564623200000300D6
:102F50003EC1625DA95EB039000000007564620088
:102F600075646233000003003EC1625DA95EB4393E
:102F700000000000756463007564633000000300A6
:102F80003EC1625DA95EB83900000000756463004F
:102F900075646331000003003EC1625DA95EBC3907
:102FA0000000000075646300756463320000030074
:102FB0003EC1625DA95EC039000000007564630017
:102FC00075646333000003003EC1625DA95EC439CD
:102FD0000000000075646400756464300000030044
:102FE0003EC1625DA95EC8390000000075646400DE
:102FF00075646431000003003EC1625DA95ECC3996
:103000000000000075646400756464320000030011
:103010003EC1625DA95ED0390000000075646400A5
:1030200075646433000003003EC1625DA95ED4395B
:10303000000000005F7465005F74657800000002A6
:103040005BC1895DC25DD554000000005F746500FE
:103050005F746579000000025BC1895DC25DD9546F
:10306000000000005F7465005F74657A0000000274
:103070005BC1895DC25DDD54000000005F746500C6
:103080005F746561000000025BC1895DC25DE1544F
:10309000000000005F7465005F746562000000025C
:1030A0005BC1895DC25DE554000000005F7465008E
:1030B0005F746563000000025BC1895DC25DE95415
:1030C000000000005F7472005F74727800000002FC
:1030D0005BC1895DC25DFA55000000005F7472003B
:1030E0005F747279000000025BC1895DC25DFE55AC
:1030F000000000005F7472005F74727A00000002CA
:103100005BC1895DC25D0256000000005F74720001
:103110005F747261000000025BC1895DC25D06568A
:10312000000000005F7472005F74726200000002B1
:103130005BC1895DC25D0A56000000005F747200C9
:103140005F747263000000025BC1895DC25D0E5650
:10315000000000005F7473005F74733100000002B0
:103160005BC1895DC25D6555000000005F70730042
:103170005F707331000000025BC1895DC25D7555EF
:10318000000000005F6373005F63733100000002A2
:103190005BC1895DC25D8555000000005F657300FD
:1031A0005F657331000000025BC1895DC25D9555AA
:1031B000000000005F7873005F7873310000000248
:1031C0005BC1895DC25DC758000000005F66650095
:1031D0005F666531000000025BC1895DC25DA55577
:1031E000000000005F7473005F747332000000021F
:1031F0005BC1895DC25D6955000000005F707300AE
:103200005F707332000000025BC1895DC25D795559
:10321000000000005F6373005F6373320000000210
:103220005BC1895DC25D8955000000005F65730068
:103230005F657332000000025BC1895DC25D995514
:10324000000000005F7873005F78733200000002B6
:103250005BC1895DC25DDF58000000005F666500EC
:103260005F666532000000025BC1895DC25DA955E1
:10327000000000005F7473005F747333000000028D
:103280005BC1895DC25D6D55000000005F70730019
:103290005F707333000000025BC1895DC25D7D55C4
:1032A000000000005F6373005F637333000000027F
:1032B0005BC1895DC25D8D55000000005F657300D4
:1032C0005F657333000000025BC1895DC25D9D557F
:1032D000000000005F7873005F7873330000000225
:1032E0005BC1895DC25DF758000000005F66650044
:1032F0005F666533000000025BC1895DC25DAD554C
:10330000000000005F7473005F74733400000002FB
:103310005BC1895DC25D7155000000005F70730084
:103320005F707334000000025BC1895DC25D81552E
:10333000000000005F6373005F63733400000002ED
:103340005BC1895DC25D9155000000005F6573003F
:103350005F657334000000025BC1895DC25DA155E9
:10336000000000005F7873005F7873340000000293
:103370005BC1895DC25D0F59000000005F6665009A
:103380005F666534000000025BC1895DC25DB155B6
:1033900000000000000000005F64616D000000009C
:1033A00009C1055A055ADC39000000000000000080
:1033B000736530300000020009C13E5D595E7E57E2
:1033C00000000000000000007365303100000200C2
:1033D00009C13E5D595E80570000000000000000FA
:1033E000736530320000020009C13E5D595E8257AC
:1033F0000000000000000000736530330000020090
:1034000009C13E5D595E84570000000000000000C5
:10341000736530340000020009C13E5D595E865775
:10342000000000000000000073653035000002005D
:1034300009C13E5D595E8857000000000000000091
:10344000736530360000020009C13E5D595E8A573F
:10345000000000000000000073653037000002002B
:1034600009C13E5D595E8C5700000000000000005D
:10347000736530380000020009C13E5D595E8E5709
:1034800000000000000000007365303900000200F9
:1034900009C13E5D595E9057000000000000000029
:1034A000736531300000020009C13E5D595E9257DC
:1034B00000000000000000007365313100000200D0
:1034C00009C13E5D595E94570000000000000000F5
:1034D000736531320000020009C13E5D595E9657A6
:1034E000000000000000000073653133000002009E
:1034F00009C13E5D595E98570000000000000000C1
:10350000736531340000020009C13E5D595E9A576F
:10351000000000000000000073653135000002006B
:1035200009C13E5D595E9C5700000000000000008C
:10353000736531360000020009C13E5D595E9E5739
:103540000000000000000000736531370000020039
:1035500009C13E5D595EA057000000000000000058
:10356000736531380000020009C13E5D595EA25703
:103570000000000000000000736531390000020007
:1035800009C13E5D595EA457000000000000000024
:10359000736532300000020009C13E5D595EA657D6
:1035A00000000000000000007365323100000200DE
:1035B00009C13E5D595EA8570000000000000000F0
:1035C000736532320000020009C13E5D595EAA57A0
:1035D00000000000000000007365323300000200AC
:1035E00009C13E5D595EAC570000000000000000BC
:1035F000736532340000020009C13E5D595EAE576A
:103600000000000000000000736532350000020079
:1036100009C13E5D595EB057000000000000000087
:10362000736532360000020009C13E5D595EB25733
:103630000000000000000000736532370000020047
:1036400009C13E5D595EB457000000000000000053
:10365000736532380000020009C13E5D595EB657FD
:103660000000000000000000736532390000020015
:1036700009C13E5D595EB85700000000000000001F
:10368000737973000000000009C19660095FDC399E
:103690000000000000000000703100000000000089
:1036A00009C19660095FDC390000000000000000DD
:1036B000310000000000000009C19660095FDC399C
:1036C00000000000000000003200000000000000C8
:1036D00009C19660095FDC390000000000000000AD
:1036E000330000000000000009C19660095FDC396A
:1036F0000000000000000000340000000000000096
:1037000009C19660095FDC3900000000000000007C
:10371000780000000000000009C19660095FDC39F4
:103720000000000000000000790000000000000020
:1037300009C19660095FDC3900000000000000004C
:103740007A0000000000000009C19660095FDC39C2
:103750000000000000000000610000000000000008
:1037600009C19660095FDC3900000000000000001C
:10377000620000000000000009C19660095FDC39AA
:1037800000000000000000006300000000000000D6
:1037900009C19660095FDC390000000000000000EC
:1037A000673534000000000009C19660095FDC390C
:1037B0000000000000000000673535000000000038
:1037C00009C19660095FDC390000000000000000BC
:1037D000673536000000000009C19660095FDC39DA
:1037E0000000000000000000673537000000000006
:1037F00009C19660095FDC3900000000000000008C
:10380000673538000000000009C19660095FDC39A7
:1038100000000000000000006735390000000000D3
:1038200009C19660095FDC3900000000000000005B
:10383000673932000000000009C19660095FDC3979
:1038400000000000000000006732380000000000A7
:1038500009C19660095FDC3900000000000000002B
:10386000673330000000000009C19660095FDC3951
:1038700000000000000000006D706F0000000000FC
:1038800009C19660095FDC390000000000000000FB
:10389000706F73000000000009C19660095FDC3999
:1038A00000000000000000006F66730000000000D0
:1038B00009C19660095FDC390000000000000000CB
:1038C000686F6D000000000009C19660095FDC3977
:1038D00000000000000000007072620000000000A4
:1038E00009C19660095FDC3900000000000000009B
:1038F000707772000000000009C19660095FDC3932
:1039000000000000000000006A6F67000000000077
:1039100009C19660095FDC3900000000000000006A
:103920006A6964000000000009C19660095FDC3923
:10393000000000000000000075646100000000004D
:1039400009C19660095FDC3900000000000000003A
:10395000756462000000000009C19660095FDC39EF
:10396000000000000000000075646300000000001B
:1039700009C19660095FDC3900000000000000000A
:10398000756464000000000009C19660095FDC39BD
:1039900000000000000000005F74650000000000EF
:1039A00009C19660095FDC390000000000000000DA
:1039B0005F7472000000000009C19660095FDC3985
:1039C00000000000000000005F74730000000000B1
:1039D00009C19660095FDC390000000000000000AA
:1039E0005F7073000000000009C19660095FDC3958
:1039F00000000000000000005F6373000000000092
:103A000009C19660095FDC39000000000000000079
:103A10005F6573000000000009C19660095FDC3932
:103A200000000000000000005F787300000000004C
:103A300009C19660095FDC39000000000000000049
:103A40005F6665000000000009C19660095FDC390F
:103A500000000000000000006D00000000000000F9
:103A600009C18763C25DDC3900000000000000006E
:103A7000710000000000000009C16D63C25DDC3907
:103A800000000000000000006F00000000000000C7
:103A900009C15363C25DDC39000000000000000072
:103AA000240000000000000009C1A163C25DDC39F0
:103AB00000000000486F6D696E67206572726F725A
:103AC000202D2025632061786973207365747469E3
:103AD0006E6773206D6973636F6E66696775726573
:103AE000640050726F62696E67206572726F722037
:103AF0002D20256320617869732063616E6E6F7479
:103B0000206D6F766520647572696E672070726FC4
:103B100062696E67005B69645D202054696E794755
:103B2000204944253330730A005B68765D202068A5
:103B3000617264776172652076657273696F6E2554
:103B400031362E32660A005B68705D202068617233
:103B5000647761726520706C6174666F726D253177
:103B6000352E32660A005B66765D20206669726DCE
:103B7000776172652076657273696F6E2531362EB6
:103B800032660A005B66625D20206669726D77614D
:103B90007265206275696C642531382E32660A00C0
:103BA000456E7465722024626F6F743D3120746FAE
:103BB00020656E7465722074686520626F6F742072
:103BC0006C6F616465722E0A000A0A0A232323209F
:103BD00054696E794720424F4F54204C4F41444521
:103BE000522048656C70202323230A00456E7465BB
:103BF000722024646566613D3120746F20726573A4
:103C00006574207468652073797374656D20746FB2
:103C10002074686520666163746F727920646566DC
:103C200061756C742076616C7565732E0A546869D1
:103C3000732077696C6C206F766572777269746532
:103C400020616E79206368616E67657320796F7596
:103C50002068617665206D6164652E0A000A0A0A93
:103C60002323232054696E794720524553544F52E1
:103C7000452044454641554C54532048656C7020BE
:103C80002323230A00496E766F6B652073656C668B
:103C9000207465737420627920656E746572696E34
:103CA000672024746573743D4E20776865726520C3
:103CB0004E206973206F6E65206F663A0A202024BB
:103CC000746573743D312020736D6F6B652074656E
:103CD00073740A202024746573743D322020686F49
:103CE0006D696E67207465737420202028796F7564
:103CF000206D757374207472697020686F6D696EC1
:103D000067207377697463686573290A20202474B7
:103D10006573743D3320207371756172652074651D
:103D20007374202020286120736572696573206F89
:103D3000662073717561726573290A202024746589
:103D400073743D3420206172632074657374202085
:103D50002020202028736F6D65206C6172676520BC
:103D6000636972636C6573290A2020247465737417
:103D70003D3520206477656C6C2074657374202059
:103D80002020286D6F7665732073706163656420F1
:103D900062792031207365636F6E64206477656C8F
:103DA0006C73290A202024746573743D36202066C4
:103DB000656564686F6C6420746573742028656E33
:103DC000746572202120616E64207E20746F2068EB
:103DD0006F6C6420616E6420726573746172742C00
:103DE00020726573706563746976656C79290A2041
:103DF0002024746573743D3720204D20636F646503
:103E00007320746573742020284D20636F6465737C
:103E100020696E7465726D696E676C656420776980
:103E20007468206D6F766573290A20202474657389
:103E3000743D3820204A534F4E20746573742020FF
:103E4000202020286D6F74696F6E20746573742054
:103E500072756E207573696E67204A534F4E2063EA
:103E60006F6D6D616E6473290A202024746573740C
:103E70003D392020696E76657273652074696D65C1
:103E800020746573740A202024746573743D313086
:103E900020726F74617279206D6F74696F6E207417
:103EA0006573740A202024746573743D3131207366
:103EB0006D616C6C206D6F76657320746573740A28
:103EC000202024746573743D313220736C6F772029
:103ED0006D6F76657320746573740A202024746591
:103EE00073743D313320636F6F7264696E61746502
:103EF0002073797374656D206F66667365742074C2
:103F000065737420284739322C204735342D4735C6
:103F100039290A0A546573747320617373756D656A
:103F200020612063656E7465726564205859206F46
:103F3000726967696E20616E64206174206C6561CE
:103F400073742038306D6D20636C656172616E63CF
:103F50006520696E20616C6C2064697265637469A8
:103F60006F6E730A546573747320617373756D6536
:103F7000205A20686173206174206C65617374201D
:103F800034306D6D20706F73696974697665206374
:103F90006C656172616E63650A5465737473207336
:103FA00074617274207769746820612047302058EA
:103FB00030205930205A30206D6F76650A486F6D79
:103FC000696E672069732074686520657863657021
:103FD00074696F6E2E204E6F20696E697469616C12
:103FE00020706F736974696F6E206F7220636C65E7
:103FF0006172616E636520697320617373756D65AD
:10400000640A000A0A0A2323232054696E79472090
:1040100053454C4620544553542048656C7020232A
:1040200023230A0045616368202420636F6D6D615E
:104030006E642061626F766520616C736F206469C5
:1040400073706C6179732074686520746F6B656E32
:1040500020666F7220656163682073657474696E91
:104060006720696E205B205D20627261636B6574FE
:10407000730A546F20766965772073657474696E6E
:10408000677320656E746572206120746F6B656E56
:104090003A0A0A2020243C746F6B656E3E0A0A4679
:1040A0006F72206578616D706C652024796672206E
:1040B000746F20646973706C61792074686520592D
:1040C000206D6178206665656420726174650A0AF6
:1040D000546F207570646174652073657474696EC3
:1040E000677320656E74657220746F6B656E2065F2
:1040F0007175616C732076616C75653A0A0A2020CF
:10410000243C746F6B656E3E3D3C76616C75653E1C
:104110000A0A466F72206578616D706C652024799B
:1041200066723D38303020746F2073657420746877
:10413000652059206D617820666565642072617420
:104140006520746F20383030206D6D2F6D696E756D
:1041500074650A466F7220636F6E66696775726177
:1041600074696F6E2064657461696C732073656532
:104170003A2068747470733A2F2F67697468756297
:104180002E636F6D2F73796E746865746F732F541F
:10419000696E79472F77696B692F54696E79472D5E
:1041A000436F6E66696775726174696F6E0A005459
:1041B0006865736520636F6D6D616E6473206172F5
:1041C000652061637469766520666F7220636F6E27
:1041D00066696775726174696F6E3A0A202024738C
:1041E00079732053686F772073797374656D202815
:1041F00067656E6572616C292073657474696E679A
:10420000730A2020243120202053686F77206D6F9F
:10421000746F7220312073657474696E677320281F
:104220006F72207768617465766572206D6F746F48
:104230007220796F752077616E7420312C322C33A7
:104240002C34290A2020247820202053686F7720DE
:104250005820617869732073657474696E67732080
:10426000286F72207768617465766572206178695D
:104270007320796F752077616E7420782C792C7A91
:104280002C612C622C63290A2020246D20202053CD
:10429000686F7720616C6C206D6F746F722073652E
:1042A0007474696E67730A2020247120202053687B
:1042B0006F7720616C6C206178697320736574740A
:1042C000696E67730A2020246F20202053686F775F
:1042D00020616C6C206F66667365742073657474FE
:1042E000696E67730A2020242420202053686F778A
:1042F00020616C6C2073657474696E67730A20208A
:10430000246820202053686F7720746869732068C0
:10431000656C702073637265656E0A0A000A0A0A8A
:104320002323232054696E794720434F4E46494743
:1043300055524154494F4E2048656C702023232329
:104340000A000A466F722064657461696C656420B6
:1043500054696E794720696E666F207365653A20EF
:1043600068747470733A2F2F6769746875622E636E
:104370006F6D2F73796E746865746F732F54696EE7
:1043800079472F77696B692F0A466F7220746865C9
:10439000206C6174657374206669726D77617265F3
:1043A000207365653A2068747470733A2F2F6769BB
:1043B000746875622E636F6D2F73796E746865749F
:1043C0006F732F54696E79470A506C65617365206D
:1043D0006C6F6720616E79206973737565732061F6
:1043E0007420687474703A2F2F7777772E73796EF4
:1043F000746865746F732E636F6D2F666F72756D61
:10440000730A486176652066756E0A000A4E6F74FD
:10441000653A2054696E79472067656E65726174EC
:104420006573206175746F6D617469632073746165
:10443000747573207265706F727473206279206472
:10444000656661756C740A546869732063616E20D7
:1044500062652064697361626C65642062792065BD
:104460006E746572696E67202473763D300A5365F9
:1044700065207468652077696B692062656C6F7769
:1044800020666F72206D6F72652064657461696C5F
:10449000732E0A00546865736520636F6D6D616EDD
:1044A0006473206172652061637469766520667249
:1044B0006F6D2074686520636F6D6D616E64206C34
:1044C000696E653A0A205E78202020202020202076
:1044D000202020202052657365742028636F6E743D
:1044E000726F6C207829202D20736F66747761724B
:1044F000652072657365740A20203F2020202020EB
:1045000020202020202020204D616368696E6520D6
:10451000706F736974696F6E20616E642067636F7A
:104520006465206D6F64656C2073746174650A2026
:104530002024202020202020202020202020205344
:10454000686F7720616E642073657420636F6E6698
:10455000696775726174696F6E2073657474696ED2
:1045600067730A20202120202020202020202020C6
:1045700020202046656564686F6C64202D2073746C
:104580006F70206D6F74696F6E20776974686F75D6
:1045900074206C6F73696E6720706F736974696FD4
:1045A0006E0A20207E202020202020202020202075
:1045B00020204379636C65205374617274202D2030
:1045C000726573746172742066726F6D20666565C2
:1045D00064686F6C640A202068202020202020203E
:1045E00020202020202053686F7720746869732072
:1045F00068656C702073637265656E0A202024689C
:1046000020202020202020202020202053686F7789
:1046100020636F6E66696775726174696F6E20687A
:10462000656C702073637265656E0A202024746562
:1046300073742020202020202020204C69737420B7
:1046400073656C662D74657374730A202024746519
:1046500073743D4E2020202020202052756E207340
:10466000656C662D74657374204E0A202024686F73
:104670006D653D312020202020202052756E206164
:1046800020686F6D696E67206379636C650A20200E
:1046900024646566613D3120202020202020526561
:1046A00073746F726520616C6C2073657474696ECD
:1046B000677320746F2022666163746F72792220A1
:1046C00064656661756C74730A000A0A0A23232301
:1046D0002054696E79472048656C70202323230A93
:1046E000005B6A735D20206A736F6E207365726968
:1046F000616C697A65207374796C65253964205B17
:10470000303D72656C617865642C313D73747269FB
:1047100063745D0A005B6A765D20206A736F6E20A9
:10472000766572626F7369747925313564205B3008
:104730003D73696C656E742C313D666F6F74657284
:104740002C323D6D657373616765732C333D636F08
:104750006E666967732C343D6C696E656E756D2C81
:10476000353D766572626F73655D0A005B656A5DF3
:104770002020656E61626C65206A736F6E206D6FBC
:10478000646525313364205B303D746578742C3169
:104790003D4A534F4E5D0A00C958C358BC58B758DC
:1047A000AE58A35898588C58805872585B584C583B
:1047B0003F5833581F581258FD57E957E657E357EB
:1047C000D457BF57AA579B578B57795762574557AE
:1047D00028570F57F956E856D656C956B7569D561C
:1047E0009A569756945691568E568B56885685569D
:1047F00082567F567C5679567656735670566D564D
:104800006A566756645661565E565B5658565556FC
:1048100052564F564C5649564656435640563D56AC
:104820003A563756345631562E562B56285625565C
:1048300022561F561C5619561656135610560D560C
:104840000A56075604560156FE55D755B35593558B
:1048500079555F55455521550455EC54D654BC54F3
:1048600098547B546954495432541954F753DE53C5
:10487000C053A4538C537A535C53475343533F5311
:104880003B53375333532F532B53275323531F5328
:104890001B53175313530F530B530753ED52D3525C
:1048A000C052A45292527B525A5249522952095232
:1048B000EF51D551BE518B515E513E511C51F650B6
:1048C000CF50B35094507A5060503B501250FA4F32
:1048D000CF4FA34F6D4F384F264F144F054FF24E19
:1048E000D94EB74EA54E934E814E6F4E5D4E4B4EF8
:1048F000394E274E154E034EF14DDF4DCD4DBB4D7C
:10490000B74DB34DAF4DAB4DA74DA34D9F4D9B4DF7
:10491000974D934D8F4D8B4D874D834D7F4D7B4DE7
:10492000774D734D6F4D6B4D574D394D1D4DF24CBD
:10493000CD4CA84CA44CA04C9C4C984C944C904C06
:104940008C4C884C844C804C7C4C784C744C704C17
:104950005C4C404C244C084CEC4BD04BB44B984B2B
:104960007C4B604B444B284B0C4B084B044B004B8F
:10497000FC4AF84AF44AF04ADC4AB44A8D4A674A8B
:104980003A4A144AE749E349DF49DB49C849A7499C
:1049900092494A6F6767696E67206379636C652027
:1049A0006661696C65640050726F626520656E6453
:1049B000706F696E74206973207374617274696EAC
:1049C0006720706F696E740050726F626520637942
:1049D000636C65206661696C65640032343900324D
:1049E00034380032343700486F6D696E6720457285
:1049F000726F72202D20486F6D696E672073776922
:104A00007463686573206D6973636F6E666967753B
:104A100072656400486F6D696E67204572726F72CF
:104A2000202D204E65676174697665206C61746322
:104A300068206261636B6F666600486F6D696E67C0
:104A4000204572726F72202D2054726176656C2041
:104A50006D696E2026206D61782061726520746812
:104A6000652073616D6500486F6D696E67204572E2
:104A7000726F72202D204C617463682076656C6FB4
:104A800063697479206973207A65726F00486F6D6D
:104A9000696E67204572726F72202D2053656172B6
:104AA00063682076656C6F63697479206973207A16
:104AB00065726F00486F6D696E67204572726F7224
:104AC000202D20426164206F72206E6F2061786912
:104AD000732073706563696669656400486F6D690A
:104AE0006E67206379636C65206661696C6564003C
:104AF0003233390032333800323337003233360044
:104B0000323335003233340032333300536F66743E
:104B1000206C696D697420657863656564656420DF
:104B20002D2043206D617800536F6674206C696D91
:104B30006974206578636565646564202D20432071
:104B40006D696E00536F6674206C696D69742065C1
:104B500078636565646564202D2042206D6178006E
:104B6000536F6674206C696D697420657863656540
:104B7000646564202D2042206D696E00536F667459
:104B8000206C696D6974206578636565646564206F
:104B90002D2041206D617800536F6674206C696D23
:104BA0006974206578636565646564202D20412003
:104BB0006D696E00536F6674206C696D6974206551
:104BC00078636565646564202D205A206D617800E6
:104BD000536F6674206C696D6974206578636565D0
:104BE000646564202D205A206D696E00536F6674D1
:104BF000206C696D697420657863656564656420FF
:104C00002D2059206D617800536F6674206C696D9A
:104C10006974206578636565646564202D2059207A
:104C20006D696E00536F6674206C696D69742065E0
:104C300078636565646564202D2058206D61780077
:104C4000536F6674206C696D69742065786365655F
:104C5000646564202D2058206D696E00536F667462
:104C6000206C696D697420657863656564656400AE
:104C700032313900323138003231370032313600CA
:104C800032313500323134003231330032313200CA
:104C900032313100323130003230390032303800B8
:104CA000323037003230360054726170657A6F6985
:104CB0006420706C616E6E6572206661696C6564FB
:104CC00020746F20636F6E7665726765004C696D46
:104CD00069742073776974636820686974202D2073
:104CE00053687574646F776E206F63637572726555
:104CF00064004D616368696E6520697320616C6151
:104D0000726D6564202D20436F6D6D616E64206E41
:104D10006F742070726F636573736564004D6F7696
:104D200065206C657373207468616E206D696E69AF
:104D30006D756D2074696D65004D6F7665206C65CD
:104D40007373207468616E206D696E696D756D2076
:104D50006C656E6774680047656E657269632054A0
:104D6000696E7947206572726F720031393900318E
:104D700039380031393700313936003139350031B1
:104D800039340031393300313932003139310031B1
:104D90003930003138390031383800313837003196
:104DA000383600313835003138340031383300318D
:104DB00038320031383100313830005420776F728A
:104DC0006420697320696E76616C69640054207791
:104DD0006F7264206973206D697373696E67005226
:104DE00020776F726420697320696E76616C6964E4
:104DF000005220776F7264206973206D6973736944
:104E00006E67005120776F726420697320696E7637
:104E1000616C6964005120776F7264206973206D42
:104E2000697373696E67004C20776F7264206973D1
:104E300020696E76616C6964004C20776F72642023
:104E40006973206D697373696E67004820776F72AC
:104E50006420697320696E76616C6964004820770C
:104E60006F7264206973206D697373696E670045A2
:104E700020776F726420697320696E76616C696453
:104E8000004520776F7264206973206D69737369C0
:104E90006E67004420776F726420697320696E76B4
:104EA000616C6964004420776F7264206973206DBF
:104EB000697373696E67005020776F72642069733D
:104EC000206E6F7420612076616C696420746F6F4E
:104ED0006C206E756D626572005020776F72642071
:104EE0006973206E6F7420616E20696E74656765EA
:104EF00072005020776F7264206973206E6567615D
:104F000074697665005020776F7264206973207A27
:104F100065726F005020776F726420697320696E2C
:104F200076616C6964005020776F72642069732029
:104F30006D697373696E6700417263207370656396
:104F4000696669636174696F6E206572726F722041
:104F50002D20656E64706F696E74206973207374A0
:104F6000617274696E6720706F696E74004172635C
:104F70002073706563696669636174696F6E20652B
:104F800072726F72202D2072616469757320617274
:104F900063206F7574206F6620746F6C6572616E2C
:104FA000636500417263207370656369666963615C
:104FB00074696F6E206572726F72202D206D697337
:104FC00073696E67206F6666736574287329004184
:104FD00072632073706563696669636174696F6E7B
:104FE000206572726F72202D206D697373696E6710
:104FF000206178697328657329004172632073709A
:105000006563696669636174696F6E206572726F4A
:1050100072005370696E646C65206D7573742062E4
:1050200065207475726E696E6720666F7220746891
:10503000697320636F6D6D616E64005370696E6497
:105040006C65206D757374206265206F66662066DE
:105050006F72207468697320636F6D6D616E640098
:105060005370696E646C65205320776F7264206999
:105070007320696E76616C6964005370696E646C4C
:1050800065205320776F7264206973206D69737394
:10509000696E67005370696E646C65207370656536
:1050A00064206578636565646564206D6178696D09
:1050B000756D005370696E646C652073706565640E
:1050C0002062656C6F77206D696E696D756D00503B
:1050D000726F6772616D6D656420706F696E7420A8
:1050E00073616D652061732063757272656E7420E3
:1050F000706F696E740043757474657220636F6DB0
:1051000070656E736174696F6E2063616E6E6F742B
:1051100020626520656E61626C6564005265717520
:1051200065737465642076656C6F63697479206556
:10513000786365656473206C696D697473004730CA
:10514000206F72204731206D757374206265206175
:10515000637469766520666F722047353300526F3D
:105160007461727920617865732063616E6E6F740B
:10517000206265207573656420776974682074689F
:10518000697320636F6D6D616E6400496E76657240
:1051900073652074696D65206D6F64652063616E51
:1051A0006E6F74206265207573656420776974681A
:1051B000207468697320636F6D6D616E640046656D
:1051C000656472617465206E6F74207370656369C5
:1051D000666965640053656C656374656420706C12
:1051E000616E6520697320696E76616C6964005335
:1051F000656C656374656420706C616E65206973AD
:10520000206D697373696E670041786973207461FA
:105210007267657420706F736974696F6E2069734B
:1052200020696E76616C69640041786973207461ED
:105230007267657420706F736974696F6E2069732B
:10524000206D697373696E670041786973206973B3
:105250002064697361626C656400417869732069D8
:105260007320696E76616C696420666F7220746861
:10527000697320636F6D6D616E640041786973209E
:1052800063616E6E6F742062652070726573656E07
:1052900074004178697320776F7264206D6973734D
:1052A000696E670047636F6465206D6F64616C2091
:1052B00067726F75702076696F6C6174696F6E00CC
:1052C0004D20636F646520756E737570706F7274B6
:1052D00065640047636F646520636F6D6D616E6424
:1052E00020756E737570706F727465640047656EBB
:1052F000657269632047636F646520696E707574B9
:10530000206572726F7200313239003132380031EB
:10531000323700313236003132350031323400312B
:10532000323300313232003132310031323000312B
:105330003139003131380031313700313136003107
:10534000313500313134004A534F4E207374726945
:105350006E6720746F6F206C6F6E67004A534F4EFC
:1053600020696E7075742068617320746F6F206D92
:10537000616E79207061697273004A534F4E2073D9
:10538000796E746178206572726F7200496E707503
:10539000742076616C75652072616E676520657238
:1053A000726F7200496E707574206578636565640C
:1053B00073206D6178696D756D2076616C7565001F
:1053C000496E707574206C657373207468616E200B
:1053D0006D696E696D756D2076616C756500496EDD
:1053E0007075742065786365656473206D617820DD
:1053F0006C656E67746800436F6D6D616E64206EDE
:105400006F742061636365707465642061742074D7
:105410006869732074696D6500506172616D6574AF
:1054200065722063616E6E6F7420626520726561C3
:105430006400506172616D657465722069732072D9
:105440006561642D6F6E6C7900556E737570706F49
:1054500072746564206E756D626572206F72204A89
:10546000534F4E207479706500426164206E756DF3
:1054700062657220666F726D617400496E76616C50
:105480006964206F72206D616C666F726D65642057
:10549000636F6D6D616E6400556E7265636F676EEC
:1054A000697A656420636F6D6D616E64206F722030
:1054B000636F6E666967206E616D650047656E6536
:1054C00072696320617373657274696F6E206661BF
:1054D000696C757265004D656D6F727920666175D6
:1054E0006C742064657465637465640053746163EF
:1054F0006B206F766572666C6F7720646574656388
:1055000074656400436F6E74726F6C6C65722061B9
:105510007373657274696F6E206661696C7572650C
:105520000043616E6F6E6963616C206D61636869D1
:105530006E6520617373657274696F6E2066616950
:105540006C75726500506C616E6E6572206173736C
:10555000657274696F6E206661696C75726500535F
:1055600074657070657220617373657274696F6EB3
:10557000206661696C75726500456E636F64657263
:1055800020617373657274696F6E206661696C75F2
:10559000726500494F207375622D73797374656D60
:1055A00020617373657274696F6E206661696C75D2
:1055B000726500436F6E666967207375622D73793B
:1055C0007374656D20617373657274696F6E2066A4
:1055D00061696C75726500494F206D656D6F7279F8
:1055E00020616C6C6F636174696F6E2061737365A9
:1055F0007274696F6E206661696C75726500383807
:105600000038370038360038350038340038330079
:105610003832003831003830003739003738003739
:10562000370037360037350037340037330037322C
:105630000037310037300036390036380036370051
:105640003636003635003634003633003632003612
:105650003100363000353900353800353700353601
:105660000035350035340035330035320035310032
:1056700035300034390034380034370034360034E3
:1056800035003434003433003432003431003430E7
:105690000033390033380033370033360042616459
:1056A00020737461747573207265706F72742073E7
:1056B000657474696E670050657273697374656EA2
:1056C0006365206572726F7200466C6F6174206949
:1056D00073204E414E00466C6F61742069732069DF
:1056E0006E66696E697465004D6F76652074696DCC
:1056F00065206973204E414E004D6F7665207469B8
:105700006D6520697320696E66696E69746500470E
:10571000656E6572696320657863657074696F6E24
:10572000207265706F7274004661696C65642074E4
:105730006F2067657420706C616E6E657220627593
:10574000666665720053797374656D20616C617271
:105750006D202D207368757474696E6720646F778F
:105760006E00496E697469616C697A6174696F6E03
:10577000206661696C75726500526561642D6F6E9B
:105780006C79206164647265737300496E76616C34
:105790006964204164647265737300446976696466
:1057A00065206279207A65726F00466C6F6174695A
:1057B0006E6720706F696E74206572726F72004937
:1057C0006E7465726E616C2072616E6765206572C1
:1057D000726F7200496E7465726E616C20657272D0
:1057E0006F720031390031380046756E6374696F2D
:1057F0006E206973207374756262656400456E740F
:105800006572696E6720626F6F74206C6F6164658A
:105810007200496E697469616C697A696E670042E9
:1058200075666665722066756C6C202D20666174E5
:10583000616C004275666665722066756C6C00422C
:10584000756666657220656D707479004E6F2073A1
:1058500075636820646576696365004D61782066CC
:10586000696C652073697A65206578636565646530
:10587000640046696C65206E6F74206F70656E0001
:10588000456E64206F662066696C6500456E642015
:105890006F66206C696E6500486172642072657382
:1058A0006574005465726D696E6174656400436F60
:1058B0006D706C657465004E6F6F70004561676157
:1058C000696E004572726F72004F4B005B703170F1
:1058D0006F665D2070776D207068617365206F66FC
:1058E000662020202531352E3366205B302E2E3168
:1058F0005D0A005B70317770685D2070776D2063A2
:1059000063772070686173652068692531352E33AF
:1059100066205B302E2E315D0A005B703177706C33
:105920005D2070776D2063637720706861736520F8
:105930006C6F2531352E3366205B302E2E315D0A9B
:10594000005B70317773685D2070776D20636377DB
:105950002073706565642068692531352E306620B6
:1059600052504D0A005B703177736C5D2070776D1B
:1059700020636377207370656564206C6F25313513
:105980002E30662052504D0A005B70316370685DA6
:105990002070776D20637720706861736520686977
:1059A000202531352E3366205B302E2E315D0A00E6
:1059B0005B703163706C5D2070776D206377207051
:1059C00068617365206C6F202531352E3366205B4E
:1059D000302E2E315D0A005B70316373685D20707C
:1059E000776D206377207370656564206869202572
:1059F00031352E30662052504D0A005B7031637392
:105A00006C5D2070776D206377207370656564200E
:105A10006C6F202531352E30662052504D0A005BC8
:105A200070316672715D2070776D20667265717578
:105A3000656E63792020202531352E306620487A26
:105A40000A0053595354454D205245414459004C86
:105A50006F6164696E6720636F6E66696773206645
:105A6000726F6D20454550524F4D00496E69746903
:105A7000616C697A696E6720636F6E66696773200F
:105A8000746F204F4D43204F746865724D696C6C84
:105A90002073657474696E6773007B226572223AA5
:105AA0007B226662223A25302E32662C22737422C3
:105AB0003A25642C226D7367223A222573227D7D5C
:105AC0000A007B65723A7B66623A25302E32662C7C
:105AD00073743A25642C6D73673A222573227D7D99
:105AE0000A005B71765D20207175657565207265B1
:105AF000706F727420766572626F7369747925377E
:105B000064205B303D6F66662C313D73696E676C57
:105B1000652C323D747269706C655D0A00716F3A74
:105B200025640A0071693A25640A0071723A256495
:105B30000A005B73765D2020737461747573207244
:105B400065706F727420766572626F7369747925FF
:105B50003664205B303D6F66662C313D66696C743F
:105B6000657265642C323D766572626F73655D0A9D
:105B7000005B73695D202073746174757320696EB6
:105B800074657276616C2531342E3066206D730A2F
:105B9000004D6F746F7220256320706F77657220DF
:105BA000656E61626C65642073746174653A253258
:105BB0002E30660A005B257325735D206D257320EA
:105BC000706F776572206D616E6167656D656E746B
:105BD00025313064205B303D64697361626C6564BB
:105BE0002C313D616C77617973206F6E2C323D6989
:105BF0006E206379636C652C333D7768656E206D2C
:105C00006F76696E675D0A005B257325735D206D95
:105C1000257320706F6C6172697479253138642046
:105C20005B303D6E6F726D616C2C313D72657665D7
:105C30007273655D0A005B257325735D206D2573A6
:105C4000206D6963726F73746570732531366420DB
:105C50005B312C322C342C385D0A005B25732573A4
:105C60005D206D25732074726176656C207065729D
:105C7000207265766F6C7574696F6E2531302E34C5
:105C80006625730A005B257325735D206D257320DF
:105C90007374657020616E676C652532302E3366D3
:105CA00025730A005B257325735D206D2573206DB8
:105CB000617020746F206178697325313564205BD1
:105CC000303D582C313D592C323D5A2E2E2E5D0A36
:105CD000005B6D745D20206D6F746F722069646C61
:105CE000652074696D656F75742531342E326620B8
:105CF0005365630A00045D005DFB5C20646567001A
:105D0000206D6D0020696E005B73745D20207377D9
:105D100069746368207479706525313864205B305C
:105D20003D4E4F2C313D4E435D0A00546573742047
:105D3000232564206E6F7420666F756E640A004EB2
:105D4000312054314D360A4E32204731370A4E3316
:105D5000204732310A4E382046313830300A4E3929
:105D60002047310A4E3130302047393220582D3209
:105D7000352E313737592D33342E303732205A2DC6
:105D8000312E303030202854454D502C2052454D76
:105D90004F5645204C41544552290A4E3334332046
:105DA000582D32352E353935592D33342E3334397B
:105DB0000A4E33343420582D32352E373031592D98
:105DC00033342E3433360A4E33343520582D3235A1
:105DD0002E373931592D33342E3532300A4E333483
:105DE0003620582D32352E383634592D33342E3650
:105DF00030310A4E33343720582D32352E39323077
:105E0000592D33342E3637390A4E33343820582D35
:105E100032352E393630592D33342E3735340A4E3B
:105E200033343920582D32352E393832592D333408
:105E30002E3832360A4E33353020582D32352E3931
:105E40003837592D33342E3839350A4E3335312011
:105E5000582D32352E393736592D33342E393631C7
:105E60000A4E33353220582D32352E393438592DDB
:105E700033352E3032330A4E33353320582D3235F8
:105E80002E393033592D33352E3038320A4E3335D2
:105E90003420582D32352E383431592D33352E31AA
:105EA00033380A4E33353520582D32352E373633B8
:105EB000592D33352E3139300A4E33353620582D91
:105EC00032352E363639592D33352E3233390A4E86
:105ED00033353720582D32352E353539592D333558
:105EE0002E3238340A4E33353820582D32352E3480
:105EF0003333592D33352E3332350A4E333539206D
:105F0000582D32352E323931592D33352E33363323
:105F10000A4E33363020582D32352E313334592D38
:105F200033352E3339370A4E33363120582D32343B
:105F30002E393633592D33352E3432380A4E333616
:105F40003220582D32342E373737592D33352E34F1
:105F500035350A4E33363320582D32342E35373707
:105F6000592D33352E3437370A4E33363420582DD9
:105F700032342E333637592D33352E3439360A4ED6
:105F800033363520582D32342E313434592D3335B3
:105F90002E3531310A4E33363620582D32332E39D4
:105FA0003039592D33352E3532320A4E33363720BB
:105FB000582D32332E363631592D33352E35323970
:105FC0000A4E33363820582D32332E343033592D83
:105FD00033352E3533320A4E33363920582D32338D
:105FE0002E313333592D33352E3533320A4E333774
:105FF0003020582D32322E383533592D33352E3549
:1060000032370A2F4E3235313820473058302E3350
:106010003237592D33332E3532315A2D312E30301F
:10602000300A4E32353139204D3330004E31204761
:1060300032300A4E3520473430204731370A4E314E
:1060400030205431204D30360A284E313520473922
:1060500030204730205830205930205A30290A4EFD
:106060003230205335303030204D3033200A4E321C
:10607000352058302E3036342059302E33323620E9
:106080005A300A4E343020473031204631362E30D7
:106090000A4E35302058302E3036342059302E33C9
:1060A00032360A4E35352058302E303630205930B1
:1060B0002E3239330A4E36302058302E30373720C2
:1060C00059302E3236370A4E36352058302E31317F
:1060D000312059302E3235370A4E37302058302E85
:1060E0003134392059302E3235320A4E3735205866
:1060F000302E3138382059302E3235350A4E38306E
:106100002058302E3232372059302E3236380A4E4F
:1061100038352058302E3235372059302E3237312D
:106120000A4E39302058302E3333352059302E3234
:1061300036350A4E39352058302E34313220593018
:106140002E3237310A4E3130302058302E34373429
:106150002059302E3238370A4E3130352058302E03
:106160003439312059302E3238390A4E313130200D
:1061700058302E3531372059302E3237330A4E31D0
:1061800031352058302E3534342059302E323633C4
:106190000A4E3132302058302E3538302059302ECA
:1061A0003236310A4E3132352058302E35393520CD
:1061B00059302E3236330A4E3133302058302E3695
:1061C00032312059302E3237340A4E31333520588F
:1061D000302E3635392059302E3330360A4E313490
:1061E000302058302E3637332059302E3333350A8D
:1061F0004E3134352058302E3637392059302E3331
:1062000036310A4E3135302058302E363738205945
:10621000302E3338390A4E3135352058302E363746
:10622000302059302E3432300A4E3136302058303A
:106230002E3637302059302E3434360A4E3136352A
:106240002058302E3638302059302E3437340A4E0C
:106250003137302058302E3730342059302E3439F1
:10626000370A4E3137352058302E373332205930E7
:106270002E3531350A4E3138302058302E373934EA
:106280002059302E3533350A4E3138352058302ECE
:106290003837322059302E3536370A4E31393020D2
:1062A00058302E3935302059302E3630340A4E31A0
:1062B00039352058312E3033312059302E3634378D
:1062C0000A4E3230302058312E3134392059302E98
:1062D0003732320A4E3230352058312E33303820A2
:1062E00059302E3835340A4E3231302058312E3460
:1062F00033302059302E3938340A4E323135205857
:10630000312E3434372059302E3938360A4E323255
:10631000302058312E3632382059302E3832320A59
:106320004E3232352058312E3733322059302E3705
:1063300031340A4E3233302058322E303039205921
:10634000302E3338310A4E3233352058322E313127
:10635000362059302E3236360A4E323430205832FA
:106360002E3232382059302E3135370A4E323435FC
:106370002058322E3238302059302E3132330A4EE6
:106380003235302058322E3333322059302E3039C6
:10639000340A4E3235352058322E343233205930BB
:1063A0002E3037300A4E3236302058322E343839BB
:1063B0002059302E3036350A4E3236352058322E9E
:1063C0003535372059302E3036360A4E32373020A8
:1063D00058322E3632372059302E3038340A4E3269
:1063E00037352058322E3639332059302E31303956
:1063F0000A4E3238302058322E3733302059302E62
:106400003133330A4E3238352058322E3830352069
:1064100059302E3139300A4E3239302058322E3828
:1064200032392059302E3231360A4E323935205821
:10643000322E3838302059302E3239310A4E33302E
:10644000302058322E3838342059302E3330300A2C
:106450004E3330352058322E3839382059302E33CB
:1064600033320A4E3331302058322E3930352059EC
:10647000302E3336370A4E3331352058322E3931EB
:10648000302059302E3430370A4E333230205832D3
:106490002E3930382059302E3434360A4E333235C6
:1064A0002058322E3930312059302E3439350A4EA9
:1064B0003333302058322E3839372059302E343982
:1064C000350A4E3333352058322E38393020593082
:1064D0002E3532340A4E3334302058322E3834328E
:1064E0002059302E3630340A4E3334352058322E6F
:1064F0003831342059302E3636350A4E3335302077
:1065000058322E3739342059302E3735300A4E3331
:1065100035352058322E3739312059302E3833381E
:106520000A4E3336302058322E3831392059302E29
:106530003937360A4E3336352058322E3833372025
:1065400059312E3034340A4E3337302058322E38F9
:1065500036322059312E3131320A4E3337352058F8
:10656000322E3837372059312E3134350A4E3338F0
:10657000302058322E3931322059312E3231370AFB
:106580004E3338352058322E3931372059312E329A
:1065900032360A4E3339302058322E3935312059AF
:1065A000312E3238310A4E3339352058322E3937B0
:1065B000302059312E3239350A4E3430302058329D
:1065C0002E3939362059312E3239350A4E3430358C
:1065D0002058332E3031332059312E3237350A4E80
:1065E0003431302058332E3032342059312E323568
:1065F000340A4E3431352058332E3037302059315B
:106600002E3135310A4E3432302058332E30373760
:106610002059312E3133340A4E3432352058332E3E
:106620003132352059312E3033390A4E343330204F
:1066300058332E3133382059312E3031390A4E3407
:1066400033352058332E3230352059302E393038FA
:106650000A4E3434302058332E3238322059302EFE
:106660003739370A4E3434352058332E33363120FB
:1066700059302E3639310A4E3435302058332E34C5
:1066800032362059302E3539320A4E3435352058BD
:10669000332E3435362059302E3534330A4E3436C5
:1066A000302058332E3437392059302E3439330ABC
:1066B0004E3436352058332E3439342059302E3468
:1066C00037320A4E3437302058332E353035205982
:1066D000302E3434360A4E3437352058332E353187
:1066E000382059302E3431370A4E34383020583360
:1066F0002E3533302059302E3339310A4E34383567
:106700002058332E3536342059302E3330300A4E4F
:106710003439302058332E3537372059302E323522
:10672000330A4E3439352058332E35363820593017
:106730002E3231320A4E3530302058332E35343433
:106740002059302E3137360A4E3530352058332E09
:106750003534312059302E3134360A4E353130201F
:1067600058332E3535332059302E3131390A4E35D4
:1067700031352058332E3537362059302E313036CA
:106780000A4E3532302058332E3539372059302EC5
:106790003130320A4E3532352058332E36313820DA
:1067A00059302E3130390A4E3533302058332E3699
:1067B00033392059302E3132390A4E35333520588D
:1067C000332E3635302059302E3135390A4E353496
:1067D000302058332E3636332059302E3137380A90
:1067E0004E3534352058332E3637382059302E3137
:1067F00039320A4E3535302058332E363939205942
:10680000302E3139370A4E3535352058332E373250
:10681000332059302E3139360A4E35363020583330
:106820002E3736342059302E3137390A4E35363529
:106830002058332E3830352059302E3136350A4E17
:106840003537302058332E3838342059302E3135F2
:10685000390A4E3537352058332E393439205930DE
:106860002E3136350A4E3538302058332E393636EB
:106870002059302E3137350A4E3538352058332ED1
:106880003937382059302E3139340A4E35393020D5
:1068900058332E3937382059302E3232330A4E359C
:1068A00039352058332E3936302059302E32343590
:1068B0000A4E3630302058332E3833342059302E9B
:1068C0003331310A4E3630352058332E37363220A8
:1068D00059302E3334350A4E3631302058332E3766
:1068E00032362059302E3338390A4E363135205859
:1068F000332E3730332059302E3435380A4E363265
:10690000302058332E3638322059302E3533300A65
:106910004E3632352058332E3637392059302E3501
:1069200033340A4E3633302058332E36323620591F
:10693000302E3638310A4E3633352058332E353620
:10694000382059302E3832380A4E363430205833F9
:106950002E3434342059312E3038300A4E36343506
:106960002058332E3430352059312E3136370A4EE7
:106970003635302058332E3430342059312E3136CC
:10698000370A4E3635352058332E333837205931B3
:106990002E3230380A4E3636302058332E333834C3
:1069A0002059312E3230380A4E3636352058332EA3
:1069B0003336352059312E3236350A4E36373020AF
:1069C00058332E3335352059312E3238350A4E366C
:1069D00037352058332E3334382059312E33303860
:1069E0000A4E3638302058332E3333332059312E67
:1069F0003335300A4E3638352058332E3332312075
:106A000059312E3339310A4E3639302058332E332E
:106A100031312059312E3432380A4E36393520582A
:106A2000332E3333392059312E3432330A4E373036
:106A3000302058332E3434302059312E3430360A39
:106A40004E3730352058332E3531302059312E34E1
:106A500030380A4E3731302058332E3538352059EA
:106A6000312E3432310A4E3731352058332E3631FB
:106A7000312059312E3433390A4E373230205833D1
:106A80002E3631312059312E3434310A4E373235D9
:106A90002058332E3631352059312E3434310A4EB8
:106AA0003733302058332E3633362059312E343890
:106AB000380A4E3733352058332E36333420593187
:106AC0002E3531370A4E3734302058332E36323295
:106AD0002059312E3534330A4E3734352058332E71
:106AE0003630352059312E3536330A4E3735302081
:106AF00058332E3537362059312E3537350A4E3733
:106B000035352058332E3534342059312E3538312F
:106B10000A4E3736302058332E3437392059312E2B
:106B20003539320A4E3736352058332E3435312038
:106B300059312E3539380A4E3737302058332E33F5
:106B400038372059312E3632360A4E3737352058ED
:106B5000332E3339302059312E3633360A4E3738FA
:106B6000302058332E3533322059312E3630320A08
:106B70004E3738352058332E3630312059312E35A6
:106B800039370A4E3739302058332E3636382059A7
:106B9000312E3539380A4E3739352058332E3738AB
:106BA000322059312E3631320A4E383030205833A7
:106BB0002E3739342059312E3631380A4E38303597
:106BC0002058332E3836382059312E3633360A4E77
:106BD0003831302058332E3931382059312E36355E
:106BE000350A4E3831352058332E39343520593155
:106BF0002E3636370A4E3832302058332E39363456
:106C00002059312E3638350A4E3832352058332E39
:106C10003936372059312E3638350A4E3833302040
:106C200058332E3937342059312E3639390A4E38F7
:106C300033352058332E3938342059312E373235F8
:106C40000A4E3834302058332E3938342059312EFA
:106C50003735380A4E3834352058332E39373020FE
:106C600059312E3739300A4E3835302058332E39C5
:106C700034352059312E3831370A4E3835352058C1
:106C8000332E3931382059312E3832360A4E3836C3
:106C9000302058332E3839312059312E3832370AC6
:106CA0004E3836352058332E3834322059312E386C
:106CB00030390A4E3837302058332E37393820597A
:106CC000312E3738340A4E3837352058332E373482
:106CD000362059312E3737320A4E38383020583363
:106CE0002E3639382059312E3736340A4E38383559
:106CF0002058332E3633352059312E3736360A4E4A
:106D00003839302058332E3535332059312E373825
:106D1000350A4E3839352058332E3437382059311A
:106D20002E3832300A4E3930302058332E34303934
:106D30002059312E3836340A4E3930352058332E0A
:106D40003334352059312E3931380A4E393130201B
:106D500058332E3236342059322E3032330A4E39DF
:106D600031352058332E3234382059322E303531D7
:106D70000A4E3932302058332E3234302059322ED8
:106D80003038310A4E3932352058332E33313620DF
:106D900059322E3038360A4E3933302058332E339C
:106DA00039302059322E3130340A4E39333520589B
:106DB000332E3431342059322E3132310A4E3934A7
:106DC000302058332E3433312059322E3135330AA6
:106DD0004E3934352058332E3433332059322E3146
:106DE00038300A4E3935302058332E343237205956
:106DF000322E3230350A4E3935352058332E343163
:106E0000332059322E3232340A4E3936302058333C
:106E10002E3339322059322E3234320A4E39363539
:106E20002058332E3333352059322E3234340A4E23
:106E30003937302058332E3237382059322E3233FA
:106E4000360A4E3937352058332E323536205932EE
:106E50002E3234320A4E3938302058332E323339FC
:106E60002059322E3235310A4E3938352058332EDA
:106E70003231312059322E3238300A4E39393020F1
:106E800058332E3137342059322E3335360A4E39A5
:106E900039352058332E3135392059322E33393790
:106EA0000A4E313030302058332E313530205932AF
:106EB0002E3433380A4E313030352058332E3134A9
:106EC000302059322E3438310A4E3130313020588A
:106ED000332E3133322059322E3531300A4E313093
:106EE00031352058332E3131382059322E35343354
:106EF0000A4E313032302058332E30393920593251
:106F00002E3537360A4E313032352058332E303553
:106F1000312059322E3633310A4E31303330205839
:106F2000332E3030332059322E3636360A4E313039
:106F300033352058322E3935372059322E363835F0
:106F40000A4E313034302058322E39303720593201
:106F50002E3639390A4E313034352058322E3836F3
:106F6000302059322E3731310A4E313035302058E9
:106F7000322E3831392059322E3732370A4E3130DD
:106F800035352058322E3736382059322E373435A1
:106F90000A4E313036302058322E373136205932B1
:106FA0002E3735370A4E313036352058322E3637A7
:106FB000352059322E3735370A4E31303730205888
:106FC000322E3537392059322E3733310A4E31308F
:106FD00037352058322E3537302059322E3732335C
:106FE0000A4E313038302058322E3535392059325A
:106FF0002E3732300A4E313038352058322E353364
:10700000302059322E3730310A4E31303930205845
:10701000322E3530312059322E3639330A4E313046
:1070200039352058322E3437312059322E36383304
:107030000A4E313130302058322E34343320593218
:107040002E3636380A4E313130352058322E33390B
:10705000362059322E3633340A4E313131302058F1
:10706000322E3335342059322E3539310A4E3131F2
:1070700031352058322E3335322059322E353931C0
:107080000A4E313132302058322E333235205932C7
:107090002E3534330A4E313132352058322E3331C9
:1070A000352059322E3532310A4E313133302058A5
:1070B000322E3330372059322E3439380A4E31319E
:1070C00033352058322E3239362059322E34363468
:1070D0000A4E313134302058322E32393320593271
:1070E0002E3432370A4E313134352058322E32396F
:1070F000352059322E3336360A4E3131353020584C
:10710000322E3332312059322E3330330A4E313160
:1071100035352058322E3335382059322E32343717
:107120000A4E313136302058322E3431392059321E
:107130002E3230330A4E313136352058322E34312A
:10714000392059322E3137390A4E313137302058F3
:10715000322E3430352059322E3135380A4E313105
:1071600037352058322E3336322059322E313233D1
:107170000A4E313138302058322E333534205932CE
:107180002E3130340A4E313138352058322E3335D5
:10719000342059322E3039310A4E313139302058AD
:1071A000322E3338302059322E3036350A4E3131B6
:1071B00039352058322E3431302059322E30353185
:1071C0000A4E313230302058322E3431302059328C
:1071D0002E3034370A4E313230352058322E34308A
:1071E000352059322E3032380A4E31323130205863
:1071F000322E3430382059322E3031300A4E31326E
:1072000031352058322E3431362059312E39393526
:107210000A4E313232302058322E34333320593135
:107220002E3938320A4E313232352058322E34332C
:10723000382059312E3936330A4E31323330205806
:10724000322E3434372059312E3934380A4E313207
:1072500033352058322E3436312059312E393338D7
:107260000A4E313234302058322E343830205931E1
:107270002E3933310A4E313234352058322E3437DC
:10728000382059312E3839390A4E313235302058AC
:10729000322E3438372059312E3837350A4E3132B4
:1072A00035352058322E3530342059312E3835348A
:1072B0000A4E313236302058322E3532372059318D
:1072C0002E3834380A4E313236352058322E353485
:1072D000392059312E3834390A4E3132373020585E
:1072E000322E3537372059312E3836310A4E313269
:1072F00037352058322E3630342059312E38363634
:107300000A4E313238302058322E3633312059313E
:107310002E3835340A4E313238352058322E363434
:10732000302059312E3832370A4E31323930205818
:10733000322E3634302059312E3739320A4E31321E
:1073400039352058322E3632392059312E373539D9
:107350000A4E313330302058322E363132205931F6
:107360002E3732370A4E313330352058322E3537EA
:10737000362059312E3639340A4E313331302058C7
:10738000322E3533362059312E3636320A4E3133CD
:1073900031352058322E3437302059312E3631369F
:1073A0000A4E313332302058322E333435205931A1
:1073B0002E3535310A4E313332352058322E3330A6
:1073C000372059312E3532310A4E3133333020587F
:1073D000322E3236302059312E3438320A4E313383
:1073E00033352058322E3234332059312E3437374A
:1073F0000A4E313334302058322E3232382059314F
:107400002E3436390A4E313334352058322E32324A
:10741000322059312E3434380A4E31333530205829
:10742000322E3232382059312E3432350A4E313331
:1074300035352058322E3235342059312E343035FE
:107440000A4E313336302058322E323638205931F8
:107450002E3337330A4E313336352058322E3237F9
:10746000392059312E3334320A4E313337302058D7
:10747000322E3330382059312E3238370A4E3133DC
:1074800037352058322E3334302059312E323534AE
:107490000A4E313338302058322E343037205931AB
:1074A0002E3230310A4E313338352058322E3434B2
:1074B000312059312E3135360A4E3133393020588A
:1074C000322E3435342059312E3133310A4E313396
:1074D00039352058322E3436302059312E3130365D
:1074E0000A4E313430302058322E3436342059315F
:1074F0002E3130320A4E313430352058322E343766
:10750000312059312E3033360A4E31343130205843
:10751000322E3436362059302E3937310A4E313436
:1075200031352058322E3435312059302E38393704
:107530000A4E313432302058322E34313520593011
:107540002E3739310A4E313432352058322E34300C
:10755000332059302E3736370A4E313433302058E5
:10756000322E3338382059302E3736350A4E3134E2
:1075700033352058322E3330362059302E383431BE
:107580000A4E313434302058322E323232205930C3
:107590002E3931310A4E313434352058322E3131C2
:1075A000342059302E3939350A4E3134353020588F
:1075B000322E3030322059312E3037360A4E3134A7
:1075C00035352058312E3930352059312E31333967
:1075D0000A4E313436302058312E37353420593167
:1075E0002E3232330A4E313436352058312E36336E
:1075F000372059312E3237380A4E3134373020583F
:10760000312E3538322059312E3330310A4E313453
:1076100037352058312E3535382059312E33313514
:107620000A4E313438302058312E3436302059311A
:107630002E3335320A4E313438352058312E333915
:10764000392059312E3336300A4E313439302058F2
:10765000312E3333382059312E3335340A4E3134FC
:1076600039352058312E3238372059312E333239BE
:107670000A4E313530302058312E323438205931CD
:107680002E3239340A4E313530352058312E3231D0
:10769000372059312E3235340A4E313531302058A9
:1076A000312E3231342059312E3235320A4E3135B5
:1076B00031352058312E3137322059312E3139357C
:1076C0000A4E313532302058312E3132382059317E
:1076D0002E3133390A4E313532352058312E313181
:1076E000302059312E3131370A4E31353330205860
:1076F000302E3935382059302E3934310A4E313553
:1077000033352058302E3839312059302E38373320
:107710000A4E313534302058302E38323520593029
:107720002E3830380A4E313534352058302E373522
:10773000352059302E3734370A4E31353530205800
:10774000302E3631392059302E3633330A4E31350A
:1077500035352058302E3437372059302E353236D3
:107760000A4E313536302058302E343737205930D4
:107770002E3532340A4E313536352058302E3431DC
:10778000312059302E3437360A4E313537302058B3
:10779000302E3333312059302E3435340A4E3135C2
:1077A00037352058302E3237382059302E34323782
:1077B0000A4E313538302058302E3233312059308E
:1077C0002E3339370A4E313538352058302E31387E
:1077D000332059302E3337390A4E3135393020585D
:1077E000302E3133352059302E3336350A4E31356F
:1077F00039352058302E3037362059302E33343139
:107800000A4E3136303520473030204633302E3066
:107810000A4E31363130204D3035200A4E31363166
:107820003520473930205830205930205A300A4E00
:1078300031363135204D33300A28456E64206F666D
:1078400020434E432050726F6772616D2900284DAE
:1078500053472A2A2A2A204D6963726F7374657010
:107860002054657374205B76315D202A2A2A2A29E8
:107870000A473030204731372047323120473430F3
:107880002047343920473830204739300A6730786C
:107890003079307A300A7B22316D69223A317D0AA3
:1078A0007B22326D69223A317D0A7B22336D692257
:1078B0003A317D0A7B22346D69223A317D0A673084
:1078C000207831300A7B22316D69223A327D0A7884
:1078D000300A7B22316D69223A347D0A7831300AD0
:1078E0007B22316D69223A387D0A78300A67302070
:1078F0007931300A7B22326D69223A327D0A793041
:107900000A7B22326D69223A347D0A7931300A7B52
:1079100022326D69223A387D0A79300A6730207A3E
:1079200031300A7B22336D69223A327D0A7A300A7D
:107930007B22336D69223A347D0A7A31300A7B2208
:10794000336D69223A387D0A7A300A673020613116
:10795000300A7B22346D69223A327D0A61300A7B1B
:1079600022346D69223A347D0A6131300A7B223437
:107970006D69223A387D0A61300A6D3200284D5314
:10798000472A2A2A2A20436F6F7264696E617465E0
:10799000206F6666736574732074657374205B76FC
:1079A000315D202A2A2A2A290A6730306731376751
:1079B00032316734306734396738306739300A67B5
:1079C00035340A673932783079307A300A663630A1
:1079D000300A284D53472A2A2A2A207465737420B6
:1079E000473932206F6666736574732A2A2A2A29FA
:1079F0000A286D73675374657020313A204D6F7695
:107A0000652066726F6D20302C3020746F2033300B
:107A10002C30206D6D20696E20706F7369746976EB
:107A200065205820646972656374696F6E290A283D
:107A30006D73675374657020323A205265736574B4
:107A4000206F726967696E20746F20302E30207548
:107A500073696E6720473932290A286D736753743A
:107A6000657020333A204D6F766520746F20323078
:107A70002C302E2053686F756C64206D6F766520F6
:107A80003230206D6D20696E20706F736974697675
:107A900065205820646972656374696F6E20616E39
:107AA0006420737461747573207265706F727420D2
:107AB00073686F756C642073746172742066726F82
:107AC0006D20302C30290A286D736753746570203F
:107AD000343A204D6F766520746F20302E30202090
:107AE0002053686F756C64206D6F7665203230208E
:107AF0006D6D20696E206E656761746976652058CA
:107B000020646972656374696F6E20616E642073AE
:107B10007461747573207265706F72742073686F0E
:107B2000756C642073746172742066726F6D20329C
:107B3000302C30290A67317833300A67393278308F
:107B40000A67317832300A6731783079300A247325
:107B5000720A67393278300A673470302E350A2855
:107B60004D53472A2A2A2A207465737420473535D5
:107B7000206F6666736574732A2A2A2A290A286D7B
:107B800073675374657020313A2053657420436FD6
:107B90006F7264696E6174652073797374656D20AA
:107BA00032205B6735355D20746F206F66667365C4
:107BB00074206F662035302C3530290A286D7367A4
:107BC0005374657020323A2053656C6563742047A6
:107BD000353520636F6F7264696E617465207379E7
:107BE0007374656D290A286D73675374657020334B
:107BF0003A204D6F766520746F20302C302E20484F
:107C00006561642073686F756C64206D6F766520A4
:107C1000646961676F6E616C6C7920696E202B58A6
:107C200020616E64202B5920616E6420737461742E
:107C30007573207265706F72742073686F756C64F1
:107C40002073746172742066726F6D20302C30293D
:107C50000A6731304C3270327835307935300A6706
:107C600035350A6730783079300A673470302E3510
:107C70000A284D53472A2A2A2A20746573742047FC
:107C80003533206162736F6C757465206F76657231
:107C90007269646573202A2A2A2A290A286D736763
:107CA0005374657020313A2052756E2061207371D3
:107CB0007561726520696E2047353520737973745C
:107CC000656D290A286D73675374657020323A20F8
:107CD00052756E20612073717561726520772F4730
:107CE0003533206F76657272696465290A6730786A
:107CF0003079300A673078323079300A673078323C
:107D0000307932300A673078307932300A6730782B
:107D10003079300A673470302E350A673533673072
:107D2000783079300A673533673078323079300A05
:107D300067353367307832307932300A67353367E8
:107D40003078307932300A673533673078307930BF
:107D50000A6730783079300A673470302E350A2857
:107D60004D53472A2A2A2A20746573742052657459
:107D700075726E20746F20686F6D65202A2A2A2A1A
:107D8000290A286D73675374657020313A20526553
:107D90007475726E20746F20686F6D6520757369DD
:107DA0006E6720473238290A286D736753746570EF
:107DB00020323A20526573657420746F2047353441
:107DC00020636F6F72642073797374656D290A671D
:107DD00032380A6735340A6D333000284D53472A4C
:107DE0002A2A2A2054657374206163637572616363
:107DF00079206F6620736C6F77206D6F76657320C6
:107E00005B76315D202A2A2A2A290A6735350A67D6
:107E100030783079300A673470302E350A67347024
:107E2000302E350A67317831306632320A673534A0
:107E30000A6730783079300A6D333000284D534767
:107E40002A2A2A2A20546573742076657279207351
:107E5000686F7274206D6F766573205B76315D207C
:107E60002A2A2A2A290A6730783079300A6734703A
:107E7000302E350A673178302E3166313030300A95
:107E800078300A78302E310A78300A78302E310A6C
:107E900078300A78302E310A78300A78302E310A5C
:107EA00078300A78302E310A78300A78302E310A4C
:107EB00078300A78302E310A78300A78302E310A3C
:107EC00078300A78302E310A78300A78302E310A2C
:107ED00078300A78302E310A78300A78302E310A1C
:107EE00078300A78302E310A78300A78302E310A0C
:107EF000673470302E350A78300A78302E30310AE7
:107F000078300A78302E30310A78300A78302E30C6
:107F1000310A78300A78302E30310A78300A7830D9
:107F20002E30310A78300A78302E30310A78300A13
:107F300078302E30310A78300A78302E30310A7895
:107F4000300A78302E30310A78300A78302E3031CD
:107F50000A78300A78302E30310A78300A78302E9C
:107F600030310A78300A78302E30310A78300A7889
:107F7000302E30310A6730783079300A6D3200287F
:107F80004D53472A2A2A2A20526F74617279204160
:107F9000786973204D6F74696F6E20546573742017
:107FA0005B76315D202A2A2A2A290A673030673118
:107FB0003767323167343067343967383067393082
:107FC0000A6730783079307A306130623063300A55
:107FD0006735350A6730783079300A6633363030A5
:107FE000300A6730613336300A623336300A633321
:107FF00036300A61300A62300A63300A6731613113
:108000003434300A62313434300A63313434300A63
:1080100061300A62300A63300A67316131343430CA
:1080200062373230633336300A783079307A3061F3
:1080300030623063300A6731783630613134343041
:1080400062373230633336300A783079307A3061D3
:1080500030623063300A67317836307935306131DB
:1080600034343062373230633336300A7830793026
:108070007A306130623063300A6731783630793572
:1080800030783235613134343062373230633336F0
:10809000300A783079307A306130623063300A6784
:1080A00035340A6730783079300A6D333000284D26
:1080B00053472A2A2A2A20496E766572736520540E
:1080C000696D65204D6F74696F6E205465737420FF
:1080D0005B76315D202A2A2A2A290A6730306731E7
:1080E0003767323167343067343967383067393051
:1080F0000A6735350A6730783079300A6739330ACC
:1081000066302E30310A67317831300A7931300AE1
:108110007A31300A6131300A78300A79300A7A309F
:108120000A61300A67317831307931307A2D313057
:108130006131300A6730783079307A3061300A66E0
:10814000302E310A6732783130792D31307A2D3244
:10815000306931300A6730783079307A300A6733E5
:10816000783130792D31307A2D32306931300A67EB
:1081700030783079307A300A673278323079307A34
:108180002D32306931300A6730783079307A300AF0
:10819000673378323079306931300A673078307936
:1081A000307A300A6732783079307A2D333069315D
:1081B000300A6733783079307A306931300A673085
:1081C000783079307A300A673278307930693230F5
:1081D0002028435720333630206465677265657305
:1081E000290A673378307930693230202843435781
:1081F000203336302064656772656573290A6739F4
:10820000340A6735340A6730783079300A6D333094
:10821000007B226763223A2267303067313767324A
:1082200031673430673439673830673930227D0A36
:108230007B226763223A22673535227D0A7B2267DB
:1082400063223A22673078307930227D0A7B2267B8
:1082500063223A2266353030227D0A7B2267632210
:108260003A22284D53477371756172657329227DD7
:108270000A7B226763223A226730783230227D0AF5
:108280007B226763223A22793230227D0A7B226781
:1082900063223A227830227D0A7B226763223A22C7
:1082A0007930227D0A7B226763223A226731783156
:1082B00030227D0A7B226763223A22793130227D87
:1082C0000A7B226763223A227830227D0A7B22676A
:1082D00063223A227930227D0A7B226763223A2286
:1082E000284D5347636972636C657329227D0A7B4D
:1082F000226763223A226732783130792D31306932
:108300003130227D0A7B226763223A22673078303F
:108310007930227D0A7B226763223A2267337831E3
:1083200030792D3130693130227D0A7B226763221A
:108330003A22673078307930227D0A7B22676322C7
:108340003A2267327832307930693130227D0A7BC7
:10835000226763223A22673078307930227D0A7BA7
:10836000226763223A2267337832307930693130BC
:10837000227D0A7B226763223A2267307830793087
:10838000227D0A7B226763223A2267327830793075
:10839000693130227D0A7B226763223A2267337873
:1083A000307930693130227D0A7B226763223A229C
:1083B000673534227D0A7B226763223A2267307850
:1083C000307930227D0A7B226763223A226D333076
:1083D000227D00284D53472A2A2A2A204D636F64A4
:1083E00065732074657374205B76315D202A2A2AB8
:1083F0002A290A6735350A6730783079300A6D33B3
:108400000A673470310A6D350A673470310A6D3489
:108410000A673470310A6D350A673470310A6D3776
:108420000A673470310A6D390A673470310A6D3861
:108430000A673470310A6D390A663530300A6730A0
:108440007832300A7932300A6D330A78300A6D3466
:108450000A79300A6D350A67317831300A6D370A8A
:108460007931300A6D380A78300A6D390A79300A64
:108470006732783130792D31306931300A6D330A05
:108480006730783079300A6D340A67337831307963
:108490002D31306931300A6D350A673078307930E6
:1084A0000A6D370A673278323079306931300A6DB7
:1084B000380A6730783079300A6D390A6733783294
:1084C0003079306931300A6730783079300A673274
:1084D000783079306931300A6733783079306931F2
:1084E000300A6735340A6730783079300A6D3330B6
:1084F00000284D53472A2A2A2A2046656564686F5A
:108500006C642054657374205B76315D202A2A2ABE
:108510002A290A284D53472A2A2A2A204D616E7596
:10852000616C6C7920656E746572202120616E64C7
:10853000207E20647572696E67206D6F76656D654B
:108540006E7420746F2074657374202A2A2A2A2975
:108550000A6735350A6730783079300A6734703306
:108560000A67303067313767323167343067343902
:108570006738306739300A663630300A673078310C
:1085800030307637362E3736350A783079300A670C
:1085900035340A6730783079300A6D333000284D31
:1085A00053472A2A2A2A204477656C6C2054657325
:1085B00074205B76315D202A2A2A2A290A67303006
:1085C0006731376732316739300A6735350A6730C6
:1085D000783079300A663530300A67307831300AC1
:1085E000673470310A67307832300A673470310A84
:1085F00067307831300A673470310A67307830304C
:108600000A673470310A79350A6735340A67307879
:108610003079300A6D330A673470310A6730783147
:10862000307931300A6D350A673470310A67307835
:1086300032307932300A6D340A673470310A67306B
:108640007833307933300A6D380A673470310A670D
:10865000307834307934300A6D390A673470310A31
:1086600067307835307935300A6730783079300ABC
:108670006D3330004E31206730306731376732312B
:108680006734306734396738306739300A4E3130F3
:10869000206730783079300A4E32302066353030FD
:1086A0000A4E3330206732783130792D31306931DC
:1086B0003020284357203237302064656772656563
:1086C00073290A4E3430206730783079300A4E35BD
:1086D00030206733783130792D31306931302028BE
:1086E0004343572039302064656772656573290AF2
:1086F0004E3630206730783079300A4E3830206777
:10870000327832307930693130202843572031387F
:10871000302064656772656573290A4E37302067BB
:1087200030783079300A4E383020673378323079FB
:108730003069313020284343572031383020646578
:108740006772656573290A4E393020673078307951
:10875000300A4E39392046313230300A4E3130300D
:1087600020673278307930693230202843572033FF
:1087700036302064656772656573290A4E31313081
:1087800020673278307930693230202843572033DF
:10879000363020616761696E290A4E3132302066B9
:1087A00037303020284368616E67652066656564F0
:1087B0002072617465207768696C6520696E204756
:1087C00032206D6F74696F6E206D6F6465290A4E7B
:1087D00031333020673278307930693230202843A5
:1087E0005720333630203372642074696D65290A4E
:1087F0004E31343020673278307930693230202879
:10880000435720333630203474682074696D6529ED
:108810000A4E31353020663530300A4E3136302040
:108820006733783079307A343069323020284343E6
:108830005720333630206465677265657320776929
:108840007468206C696E6561722074726176656C03
:10885000290A4E313730206733783079307A3069E1
:108860003230202843435720333630206167616916
:108870006E290A4E313830206637303020286D732B
:10888000672A2A2A2A4368616E67652066656564DF
:108890002072617465207768696C6520696E204775
:1088A00033206D6F74696F6E206D6F64652A2A2A9C
:1088B0002A290A4E313930206733783079306932CD
:1088C00030202843435720333630203372642074DD
:1088D000696D65290A4E323030206733783079303F
:1088E00069323020284343572033363020347468AF
:1088F0002074696D65290A4E32313020286D736706
:108900002A2A2A2A473138204576616C20746573FB
:10891000742A2A2A2A290A4E323230204731205816
:1089200033302E373037205A35302E373237204605
:108930003530300A4E32333020473138204730321C
:10894000205836372E373338205A32332E363137C7
:108950002052323520463235300A4E3234302067CC
:1089600038300A4E323530206730783079307A30FE
:108970000A4E323630206D333000284D53472A2AB4
:108980002A2A2053717561726573204D6F74696F67
:108990006E2054657374205B76315D202A2A2A2A62
:1089A000290A6730306731376732316734306734CE
:1089B000396738306739300A6730783079300A677C
:1089C0003078323020287472617665727365206168
:1089D0002032306D6D2073717561726520696E2073
:1089E0005820616E642059290A7932300A78300A99
:1089F00079300A673178313066353030202864723A
:108A0000617720612031306D6D2073717561726501
:108A100020696E205820616E6420592061742046C0
:108A2000353030290A7931300A78300A79300A67CE
:108A3000307A3230202874726176657273652061F5
:108A40002032306D6D2073717561726520696E2002
:108A50005820616E64205A290A7832300A7A300A26
:108A600078300A67317832307932307A3230663590
:108A7000303020286665656420612032306D6D20BD
:108A8000646961676F6E616C20696E20582C205993
:108A900020616E64205A290A783079307A300A7859
:108AA00034307934307A34302028747261766572CB
:108AB000736520612034306D6D20637562652069B7
:108AC0006E20582C205920616E64205A290A78346F
:108AD0003079307A300A78307934307A34300A7824
:108AE00034307934307A300A783079307A34300A58
:108AF00078307934307A300A78343079307A3430DA
:108B00000A783079307A300A6738300A673078303E
:108B100079300A673078310A673078300A6D33303F
:108B200000284D53472A2A2A2A20486F6D696E670C
:108B30002054657374205B76315D202A2A2A2A2905
:108B40000A6732382E32783079307A300A6D333015
:108B500000284D53472A2A2A2A20536D6F6B65201F
:108B600054657374205B76315D202A2A2A2A290AEB
:108B700047303020473137204732312047343020CA
:108B800047343920473830204739300A6D3367344D
:108B900070310A6D35673470310A6D346734703165
:108BA0000A6D33673470310A6D35673470310A6D80
:108BB00037673470310A6D39673470310A6D386740
:108BC0003470310A6D390A6730783079307A300A7A
:108BD000673030207832300A78300A7932300A79BA
:108BE000300A7A32300A7A300A6132300A61300A49
:108BF0004730302078323020793230207A323020BD
:108C00006132300A473030207830207930207A3095
:108C10002061300A473031206633302078322079A5
:108C200032207A322061320A7830207930207A304E
:108C30002061300A673078310A673078300A6D3247
:108C4000002C000A00257300256C750025312E309C
:108C500066002573002C000A0025733A2573002551
:108C6000733A256C750025733A25312E3066002540
:108C7000733A2573005B74765D20207465787420E8
:108C8000766572626F7369747925313564205B3063
:108C90003D73696C656E742C313D766572626F73DD
:108CA000655D0A0025660A00256C750A0025640AC0
:108CB0000025730A0074696E7967205B25735D2057
:108CC0006572723A2025733A202573200074696E0C
:108CD0007967205B25735D206F6B3E2000456E64D5
:108CE000206F6620636F6D6D616E642066696C65D0
:108CF0000A0017C9E8C684C9A5C904CA2DC7DCCCB7
:108D0000E8C670CDDCCD0ACC2DC700004006400679
:108D10001040B800B8DCCCE8C670CDDCCD0ACC2D54
:108D2000C70000400620060840B800B848CFE8C693
:108D300065CEE4CE93D02ECEA008400605060901EC
:108D40000848CFE8C665CEE4CE16CA2DC7B00840A5
:108D5000060540B030800000000000F0E0D0C010F8
:108D60000100CF673322211F1B1301016E616E00CA
:108D7000696E66004E414E494E495459494E46CDA2
:108D8000CCCC3D0AD7233C17B7D13877CC2B3295C2
:108D900095E6241FB14F0A000020410000C84200A0
:108DA000401C4620BCBE4CCA1B0E5AAEC59D74006A
:108DB000407A10F35A00A0724E18090010A5D4E8AA
:108DC0000000E87648170000E40B54020000CA9A3D
:108DD0003B000000E1F5050000809698000000408F
:108DE000420F000000A086010000001027000000D4
:108DF00000E803000000006400000000000A00001A
:108E00000000000100000000002C76D888DC674FCD
:108E10000823DFC1DFAE59E1B1B796E5E3E453C6FD
:108E20003AE651997696E8E6C28426EB898C9B62F5
:108E3000ED407C6FFCEFBC9C9F40F2BAA56FA5F49F
:108E400090055A2AF75C936B6CF9676DC11BFCE0C7
:108E5000E40D47FEF520E6B500D0ED902E0300941A
:108E60003577050080841E080000204E0A000000AF
:108E7000C80C333333330F986E12831141EF8D21B9
:108E800014893BE65516CFFEE6DB18D1844B381B20
:108E9000F77C1D901DA4BBE424203284725E2281E5
:108EA00000C9F124ECA1E53D270011241FBECFEF3E
:108EB000CDBFDFE5DEBF00E00CBF13E2A0E0B0E213
:108EC000E4E2F8EC01E00BBF02C007900D92A63877
:108ED000B107D9F729E5A6E8B3E201C01D92A23B8C
:108EE000B207E1F70E941A800C9410E40C94000081
:108EF000FC0160817181828193810E94E1D5609340
:108F0000AD320895FC0160817181828193810E945C
:108F1000E1D56093AC320895AF92BF92CF92DF92C9
:108F2000EF92FF920F931F93CF93DF937B018C01FE
:108F300080E3C82E82E3D82EE601AA24A394BC2E97
:108F4000BC18F70161917191819191917F012CEA97
:108F500035EC47E257E30E9470D718164CF4F8013D
:108F600040815181628173818B2D0E948881A8820A
:108F70000C5F1F4F2196F2E3C633DF0701F7DF9145
:108F8000CF911F910F91FF90EF90DF90CF90BF9006
:108F9000AF900C949381FC016081718182819381F7
:108FA0000E94E1D56093AE32613019F481E00E94F5
:108FB0008F7781E00C94B077CF93DF93CDB7DEB796
:108FC0006897CDBFDEBFFC01608171818281938192
:108FD0000E94E1D56093AF3281E0613019F40E94C4
:108FE0008F770CC00E94B077CE01019628E1FC017A
:108FF00011922A95E9F7BC010E94CB476896CDBF34
:10900000DEBFDF91CF9108950F931F93CF93DF932E
:10901000CDB7DEB72D97CDBFDEBF27E0E8EDF0E29C
:109020008E010F5F1F4FD80101900D922A95E1F735
:10903000BC01660F771F680F791F660F771F660FD9
:10904000771F660F771F68567A4E45E050E0CE01D5
:1090500008960E9480E1688570E0C8010E94AEE138
:10906000009739F46B8570E0C8010E94AEE100976B
:1090700011F0801B01C08FEF2D96CDBFDEBFDF91B9
:10908000CF911F910F910895EF92FF920F931F932D
:10909000CF93DF938C01F62EE72EEC012D96FC0189
:1090A00061857285838594850E94E1D51F926F93B7
:1090B000DF93CF930F5E1F4F1F930F93DF93CF93D9
:1090C000EF92FF92EEEAF9E581818F9380818F9391
:1090D0000E9447E2EDB7FEB73C96EDBFFEBFDF91C1
:1090E000CF911F910F91FF90EF9008950F931F93D1
:1090F000CF93DF93EC01162F072F8C819D810E9467
:10910000044883305CF58F3FA1F528C09E01235FA2
:109110003F4F9F938F938C858F938B858F938A85F9
:109120008F9389858F933F932F936196DF93CF938E
:109130003F932F930F931F938091AF598F938091FB
:10914000AE598F930E9447E28DB79EB740968DBF70
:109150009EBFDF91CF911F910F910895E7E1F4E158
:10916000659174914FE450E086EA9CE30E9480E1AF
:10917000CDCFE091A632F0E0EE0FFF1FED5EFB4E8B
:10918000659174914FE450E086EA9CE30E9480E18F
:10919000BDCF0F931F93CF93DF93EC01162F072FB3
:1091A0008C819D810E94044883307CF58F3FC1F5FE
:1091B0002CC0AE014F5E5F4F9E01235F3F4F9F93D8
:1091C0008F938C858F938B858F938A858F938985D9
:1091D0008F935F934F933F932F935F934F933F935F
:1091E0002F930F931F938091AF598F938091AE5916
:1091F0008F930E9447E28DB79EB742968DBF9EBF68
:10920000DF91CF911F910F910895E7E1F4E165910E
:1092100074914FE450E086EA9CE30E9480E1C9CF5C
:10922000E091A632F0E0EE0FFF1FED5EFB4E659180
:1092300074914FE450E086EA9CE30E9480E1B9CF4C
:10924000DF92EF92FF920F931F93CF93DF93CDB7EF
:10925000DEB72897CDBFDEBF8B01E42ED52E37E0D9
:10926000EFEDF0E2DE01119601900D923A95E1F7F3
:1092700028870E940448F82E288582E08F1518F070
:10928000E22FF0E002C0E2E0F0E0EE0FFF1FED5E43
:10929000FB4E659174914FE450E086EA9CE30E9496
:1092A00080E19F938F93F80183818F9382818F93C5
:1092B00081818F9380818F93E1E0F0E0EC0FFD1FBF
:1092C000EF0DF11D80811F928F93DF92EF928091BD
:1092D000AF598F938091AE598F930E9447E2CDBFD3
:1092E000DEBF2896CDBFDEBFDF91CF911F910F91DA
:1092F000FF90EF90DF9008954F925F926F927F9270
:10930000AF92BF92CF92DF92EF92FF920F931F9393
:10931000CF93DF93C0E3D2E305EF10E35C018991C3
:10932000813009F042C0F801C480D580E680F78022
:109330004080518062807380A3019201C701B60111
:109340000E94C4D39F772CEA35EC47E257E30E9492
:109350006DD587FD2AC020E034E244E759ECC7010F
:10936000B6010E9470D718165CF4F5012081318196
:1093700042815381C701B6010E9470D7181604F1CB
:1093800020E034E244E759ECC301B2010E9470D7F7
:1093900018165CF4F5012081318142815381C301AB
:1093A000B2010E946DD587FD0BC00B5C1F4FF4E02E
:1093B000AF0EB11C82E3C633D80709F0B0CF02C0AC
:1093C0008CED01C080E0DF91CF911F910F91FF9054
:1093D000EF90DF90CF90BF90AF907F906F905F90B5
:1093E0004F90089580912C32811105C080912B32CD
:1093F00080932A3229C0823031F487E080932A3268
:1094000080912B3221C0833031F489E080932A325D
:1094100080912B3219C0843031F48AE080932A3253
:1094200080912B3211C080912D32813031F485E052
:1094300080932A3280912B3207C0823019F486E063
:1094400080932A3280912B32863019F080912A3213
:1094500008958BE080932A32089580912B320895ED
:1094600080932D32813059F018F0823041F0089508
:109470008BE592E38093593290935A32089585EFA9
:1094800095E58093593290935A320895FC01848176
:109490000895845B9F4FFC0180810895855B9F4FF9
:1094A000FC0180810895825B9F4FFC0180810895BB
:1094B000815B9F4FFC0180810895875B9F4FFC017A
:1094C000808108950C948996CD96FC01608171810C
:1094D000828193810895FC01648308958B5A9F4F84
:1094E000FC01608308958F5B9F4FFC014083518393
:1094F00062837383089560935B3270935C328093D0
:109500005D3290935E3280EE91E20C94E261BF9204
:10951000CF92DF92EF92FF920F931F93CF93DF933F
:10952000D090A8327C010DEC12E38091A73290E03C
:10953000EC01CC0FDD1FC80FD91FCC0FDD1FCC0FE6
:10954000DD1FCC0FDD1FCC5BDF4C81E0D816A9F00E
:10955000B881A981CA80BB8040912033413091F409
:10956000F80120813181428153816B2F7A2F8C2D1C
:109570009B2D0E94C5D39B0109C020E030E080E014
:1095800090E004C02B2F3A2F8C2D9B2DA901BC01FC
:10959000F701458F568F678F70A3F4E0EF0EF11C33
:1095A0000C5F1F4F249682E3053E180771F6DF918A
:1095B000CF911F910F91FF90EF90DF90CF90BF90D0
:1095C0000895835B9F4FFC0160838BE592E30C94CD
:1095D000874A4F925F926F927F928F929F92AF9243
:1095E000BF92CF92DF92EF92FF920F931F93CF9390
:1095F000DF93CDB7DEB76897CDBFDEBF8C0160913A
:10960000203370E080E090E00E940FD62B013C01F7
:10961000F80160817181828193810E94E1D570E0BF
:109620005B01AA0CBB1CA60EB71EAA0CBB1CAA0C85
:10963000BB1CAA0CBB1CC5018C5B9F4C5C010DECD8
:1096400012E3FE0131964F01F501C190D190E190F6
:10965000F1905F01F80161917191819191918F0178
:10966000A30192010E9412D89B01AC01C701B6016F
:109670000E94C5D3F40161937193819391934F013B
:10968000F2E3053E1F0701F7CE0101960E946C969A
:109690008BE592E30E94874A6896CDBFDEBFDF91DB
:1096A000CF911F910F91FF90EF90DF90CF90BF90DF
:1096B000AF909F908F907F906F905F904F900895A4
:1096C0008B55924369F4E62FF0E0EE0FFF1FEE0F8B
:1096D000FF1FEB54FD4C608171818281938108955D
:1096E000862F0C946196CF92DF92EF92FF920F93A8
:1096F0001F93CF93DF93EC0182E3CB35D80709F0BA
:109700004AC070E0FB01EE0FFF1FEE0FFF1FEB548E
:10971000FD4CC080D180E280F3808091A8328130FE
:1097200059F18091A73290E0FC01EE0FFF1FE80F86
:10973000F91FEE0FFF1FE60FF71FEE0FFF1FEE0FD3
:10974000FF1FEC5BFF4C00811181B281A38120914E
:1097500020332130B1F4FB01EE0FFF1FEE0FFF1F8E
:10976000E353FD4C2081318142815381B8018B2F1D
:109770009A2F0E94C5D308C060E070E080E090E0BE
:1097800003C0B8018B2F9A2F9B01AC01C701B60112
:109790000E94C4D303C0862F0E947596C55BDF4F1D
:1097A0002881211106C023E333E34BEC51E40E94EE
:1097B00074D5DF91CF911F910F91FF90EF90DF90C3
:1097C000CF90089588E1E0E6F2E3A5EBB2E30190E3
:1097D0000D928A95E1F78091A43281110CC080919D
:1097E0005F32813041F41092983210929932109287
:1097F0009A3210929B3208954F925F926F927F92AD
:109800008F929F92AF92BF92CF92DF92EF92FF9290
:109810000F931F93CF93DF93CDB7DEB76997CDBF7B
:10982000DEBF80912C32811155C080915132813040
:1098300009F050C00E9487C681114CC0109251326D
:109840009CE5692E90E3792E26E3822E912C8E01E1
:109850000E5E1F4F36EEA32E30E2B32E33C0F7015B
:1098600081917F011F928F935F924F92BF92AF922F
:109870001F930F930E9412E3B80184E493E20E94C5
:10988000475F8D839E83F60181919191A191B19162
:109890006F018A879B87AC87BD87CE0101960E94A6
:1098A000365CCDBFDEBF9EEDE91690E2F906B9F653
:1098B000E8E16E0E711CFFEF8F1A9F0A8CE3881689
:1098C000910441F0240189EDE82E80E2F82E630135
:1098D00088E7C8CF80E06996CDBFDEBFDF91CF912A
:1098E0001F910F91FF90EF90DF90CF90BF90AF90BE
:1098F0009F908F907F906F905F904F9008952F92E0
:109900003F924F925F926F927F928F929F92AF920F
:10991000BF92CF92DF92EF92FF920F931F93CF935C
:10992000DF93CDB7DEB72997CDBFDEBF4C015B011A
:109930004090AA325090A8322090A73260902033F5
:109940007090A6326B0180E692E3888799875CEE7F
:10995000E52E50E3F52E98E1299E10011124840193
:10996000D6016D917D918D919D916D012CEA35EC23
:1099700047E257E30E946DD587FD80C0F7018081E3
:109980008150823008F07AC041104CC0F1E05F167F
:1099900009F1E885F985E20DF31DEC51F240808173
:1099A000898391819D83B281A381E1E06E1217C00A
:1099B000E885F985E359FF4F208131814281538148
:1099C000BC018B2F9A2F0E94C5D369837D838E8320
:1099D0009F8307C019821D821E821F8202C0BE8320
:1099E000AF8371100CC023E333E34BEC51E4D80197
:1099F0006D917D918D919C910E9412D805C0F801C6
:109A0000608171818281938129813D814E815F8155
:109A10000E94C5D3A885B9856D937D938D939C9342
:109A200013972CC0A885B9858D919D910D90BC91FF
:109A3000A02D89839A83AB83BC8371100EC023E36E
:109A400033E34BEC51E4F8016081718182819381B1
:109A50000E9412D89B01AC0105C0D8012D913D9107
:109A60004D915C9169817A818B819C810E94C5D3E3
:109A7000E885F985608371838283938388859985DE
:109A800004968887998795E3E90EF11C0C5F1F4FB8
:109A9000A885B985AC56B24309F062CF6090A63272
:109AA0007090AA32F091A832F983C090A732209129
:109AB00020332D838CE0A80EB11CABE8B1E3A8875E
:109AC000B9874CE6E42E42E3F42EB8E1CB9E600168
:109AD00011248401F50161917191819191915F014E
:109AE0002CEA35EC47E257E30E946DD587FD8CC028
:109AF000A885B9858C91882309F486C0815082306D
:109B000030F4F80124843584468457843BC06110C6
:109B100016C023E333E34BEC51E4D8011C966D915E
:109B20007D918D919C911F970E9412D820E030E08A
:109B300044EB53E40E9412D81B012C010DC020E01D
:109B400030E044EB53E4F80164857585868597859C
:109B50000E9412D81B012C012BED3FE049EC50E490
:109B6000A885B98591966D917D918D919C919497E1
:109B70000E9412D89B01AC01C201B1010E9474D5B0
:109B80001B012C01711031C0B981B130E1F0F70136
:109B9000EC0DFD1DEC51F240A081B18192808380DB
:109BA000ED81E130A1F4F701E359FF4F20813181CC
:109BB00042815381BD01892D982D0E94C5D3DB01BF
:109BC000982E892E04C0A0E0B0E0912C812CA20137
:109BD0009101BD01892D982D0E94C5D3D7016D93A8
:109BE0007D938D939C9313970FC0A2019101F70170
:109BF00060817181828193810E94C5D3D7016D9369
:109C00007D938D939C931397E885F985F596E88766
:109C1000F987F4E0EF0EF11C0C5F1F4F88859985E2
:109C20008A52924309F056CF2996CDBFDEBFDF910D
:109C3000CF911F910F91FF90EF90DF90CF90BF9049
:109C4000AF909F908F907F906F905F904F903F90DC
:109C50002F90089580912830909129308F3E924125
:109C600011F08FE508958091DF339091E0338F3EBE
:109C70009241B9F78091B1329091B2328F3E9241C8
:109C800081F780912733909128338F3E924149F795
:109C900080914D5690914E568F3E924111F7809192
:109CA0000A5790910B578F3E9241D9F680E0089564
:109CB000CF93C82F0E948CA782E080932B328C2FE9
:109CC000CF91089580912C32811104C083E080935C
:109CD0002B3203C085E080932B3280E00895CF9330
:109CE000C82F0E94FBB280E00E949CAE8C2F0E9485
:109CF0008CA786E080932B328C2FCF910895809390
:109D0000A53280E008958093A63280E00895809384
:109D1000AA3280E008954F925F926F927F929F9255
:109D2000AF92BF92CF92DF92EF92FF920F931F9369
:109D3000CF93DF93C82FB62E8A01F22ED32F8FEF49
:109D40008C0F863008F082C06091B33370E080E001
:109D500090E00E940FD62CEA35EC47E257E30E94D0
:109D60006DD587FD75C082E0B81619F0E4E1BE122A
:109D700071C09090A632CF2CDD2E8C2F90E0EC019C
:109D8000CC0FDD1FC80FD91FCC0FDD1FCC0FDD1F7F
:109D9000CC0FDD1FCC5BDF4C780105EB12E3AA246E
:109DA000A394F60161917191819191916F012CEAD7
:109DB00035EC47E257E30E9470D71816DCF5F2E065
:109DC000BF1214C091100CC023E333E34BEC51E4F9
:109DD000F70160817181828193810E9412D824C031
:109DE000F70160817181828193811EC0F8014080FA
:109DF00051806280738091100EC023E333E34BECFB
:109E000051E4F70160817181828193810E9412D8AF
:109E10009B01AC0105C0F701208131814281538152
:109E2000C301B2010E94C4D3688379838A839B8370
:109E3000A09251322496F4E0EF0EF11C0C5F1F4FFC
:109E400082E30D3C180709F0ACCF06C081EA05C0DB
:109E50008CEA03C08DEA01C080E0DF91CF911F91B1
:109E60000F91FF90EF90DF90CF90BF90AF909F90B9
:109E70007F906F905F904F900895CF93DF93CDB711
:109E8000DEB76897CDBFDEBF8093A732682F70E042
:109E900080E090E00E940DD669837A838B839C8357
:109EA0001D821E821F82188619861A861B861C86B2
:109EB0001D861E861F86188A198A1A8A1B8A1C8A82
:109EC0001D8A1E8A1F8A188EAE014F5F5F4FBA012E
:109ED00089EE9AE40E94CA8280E06896CDBFDEBF18
:109EE000DF91CF910895CF93DF93EBE5F2E386E521
:109EF000DF011D928A95E9F78BE5A9E2B3E3ED0155
:109F0000982F19929A95E9F7A4E8B3E3ED01199215
:109F10008A95E9F78FEE92E180932830909329306B
:109F20008093DF339093E0338093B1329093B232D9
:109F3000809327339093283380934D5690934E56B9
:109F400080930A5790930B57E0935932F0935A320B
:109F5000809141308093A63280913F300E943D4FE6
:109F6000809140308093A532809142308093A93215
:109F7000809143308093AA3281E08093A432809311
:109F8000213394E090935F32109252321092533208
:109F90001092543280932B3280932A320E943AAD31
:109FA000DF91CF910C940C84CF92DF92EF92FF92CD
:109FB000CF93C82F6A017B01E82FF0E0DF01AA0FE1
:109FC000BB1FAA0FBB1FAB54BD4C4D935D936D934C
:109FD0007C931397EE0FFF1FEE0FFF1FE05AFD4C0F
:109FE00040835183628373838C2F0E947D81B701EC
:109FF000A6018C2F0E948881CF91FF90EF90DF9077
:10A00000CF900C9493819F92AF92BF92CF92DF92A8
:10A01000EF92FF920F931F93CF93DF93CDB7DEB7ED
:10A020006897CDBFDEBF962EA72EC62ED72E7C01F9
:10A0300000E010E0B12CF601619171918191919154
:10A040006F012CEA35EC47E257E30E9470D71816EF
:10A05000A4F58091A63281110EC023E333E34BECCB
:10A0600051E4F70160817181828193810E9412D84D
:10A07000AB01BC0105C0F701408151816281738150
:10A08000E1E0F0E0EC0FFD1FE00FF11F4083518392
:10A0900062837383C801885D9F4CFC01E357FD4FC9
:10A0A0004083518362837383E555F1094083518373
:10A0B000628373838B2D0E947D81B3940C5F1F4F4D
:10A0C000F4E0EF0EF11C0831110509F0B4CF492D71
:10A0D0005A2DBE016F5F7F4F8CE897E40E94CA82C1
:10A0E00080E06896CDBFDEBFDF91CF911F910F91C9
:10A0F000FF90EF90DF90CF90BF90AF909F9008952A
:10A100004F925F926F927F928F929F92AF92BF9287
:10A11000CF92DF92EF92FF920F931F93CF93DF9333
:10A12000CDB7DEB76897CDBFDEBF21E020932033E7
:10A130008090A7329090A6325B016C0105EB12E390
:10A14000882D90E07C01EE0CFF1CE80EF91EEE0C51
:10A15000FF1CEE0CFF1CEE0CFF1CC7018C5B9F4C20
:10A160007C01F50161917191819191915F012CEADE
:10A1700035EC47E257E30E9470D7181664F5F701F3
:10A180002081318142815381F80160817181828116
:10A1900093810E94C4D32B013C0191100EC023E394
:10A1A00033E34BEC51E4F60160817181828193814C
:10A1B0000E9412D89B01AC0105C0F60120813181BB
:10A1C00042815381C301B2010E94C4D3F801608F60
:10A1D000718F828F938FF4E0CF0ED11C0C5F1F4FD5
:10A1E00084E0E80EF11C92E30D3C190709F0B9CFA9
:10A1F000682D70E080E090E00E940DD669837A833C
:10A200008B839C831D821E821F82188619861A8664
:10A210001B861C861D861E861F86188A198A1A8A26
:10A220001B8A1C8A1D8A1E8A1F8A188EAE014F5FE8
:10A230005F4FBA0189EE9AE40E94CA8280E0689674
:10A24000CDBFDEBFDF91CF911F910F91FF90EF90B7
:10A25000DF90CF90BF90AF909F908F907F906F9046
:10A260005F904F900895CF93DF93CDB7DEB7689797
:10A27000CDBFDEBF109220331092CD321092CE327D
:10A280001092CF321092D0321092D1321092D2323C
:10A290001092D3321092D4321092D5321092D6321C
:10A2A0001092D7321092D8321092D9321092DA32FC
:10A2B0001092DB321092DC321092DD321092DE32DC
:10A2C0001092DF321092E0321092E1321092E232BC
:10A2D0001092E3321092E4326091A73270E080E095
:10A2E00090E00E940DD669837A838B839C831D82C4
:10A2F0001E821F82188619861A861B861C861D865A
:10A300001E861F86188A198A1A8A1B8A1C8A1D8A29
:10A310001E8A1F8A188EAE014F5F5F4FBA0189EE09
:10A320009AE40E94CA8280E06896CDBFDEBFDF91CA
:10A33000CF910895CF93DF93CDB7DEB76897CDBFA8
:10A34000DEBF109220336091A73270E080E090E091
:10A350000E940DD669837A838B839C831D821E8223
:10A360001F82188619861A861B861C861D861E86E5
:10A370001F86188A198A1A8A1B8A1C8A1D8A1E8AB5
:10A380001F8A188EAE014F5F5F4FBA0189EE9AE4C3
:10A390000E94CA8280E06896CDBFDEBFDF91CF9178
:10A3A0000895CF93DF93CDB7DEB76897CDBFDEBFFB
:10A3B00081E0809320336091A73270E080E090E0EC
:10A3C0000E940DD669837A838B839C831D821E82B3
:10A3D0001F82188619861A861B861C861D861E8675
:10A3E0001F86188A198A1A8A1B8A1C8A1D8A1E8A45
:10A3F0001F8A188EAE014F5F5F4FBA0189EE9AE453
:10A400000E94CA8280E06896CDBFDEBFDF91CF9107
:10A410000895CF9310925F320E947F4C809132302A
:10A42000813069F480E692E30E947C49C82F88233A
:10A4300031F00E948CA782E080932B3217C08BE50D
:10A4400092E30E94874A85E080932B3280912C32E0
:10A45000811105C081E080932C320E949DAB8BE579
:10A4600092E30E9496960E94E24BC0E08C2FCF911F
:10A47000089588E1E5EBF2E3A5EEB2E301900D92D9
:10A480008A95E1F780E008950F931F93CF93DF93B0
:10A49000CDB7DEB76A97CDBFDEBF8C0181E0809378
:10A4A000A8328BE592E3698F7A8F0E94874A698D83
:10A4B0007A8DC8010E9409520E9404828823E1F328
:10A4C00088E1E0E0F0E2DE01119601900D928A95BC
:10A4D000E1F7BE016F5F7F4F85EE92E30E94095264
:10A4E0006A96CDBFDEBFDF91CF911F910F91089586
:10A4F00088E1E5EBF2E3ADEFB2E301900D928A95CE
:10A50000E1F780E008950F931F93CF93DF93CDB7CA
:10A51000DEB76A97CDBFDEBF8C0181E08093A832A1
:10A520008BE592E3698F7A8F0E94874A698D7A8DD5
:10A53000C8010E9409520E9404828823E1F388E145
:10A54000E0E0F0E2DE01119601900D928A95E1F7CC
:10A55000BE016F5F7F4F8DEF92E30E9409526A96B2
:10A56000CDBFDEBFDF91CF911F910F910895FB0109
:10A57000DC018091A432811111C09B01AD0160E02A
:10A5800070E080E89FE30E9474D5609398327093E6
:10A59000993280939A3290939B3218C08091A63260
:10A5A000811109C023E333E34BEC51E4CD010E9458
:10A5B00012D8FB0101C0CD01AF01BC01409398321C
:10A5C0005093993260939A3270939B3280E0089551
:10A5D0008093A43280E008958093A93280E00895AA
:10A5E0006093A0327093A1328093A2329093A332F1
:10A5F0000E94228380E008950F931F93CF93DF93EF
:10A60000EC018B018091A432882399F080919832DB
:10A6100090919932A0919A32B0919B32BC01CD01B8
:10A620009F772CEA35EC47E257E30E946DD587FD12
:10A6300030C081E080935F32B801CE010E947F4C30
:10A6400080913230813069F480E692E30E947C4947
:10A65000C82F882331F00E948CA782E080932B3290
:10A6600019C08BE592E30E94874A85E080932B32E4
:10A6700080912C32811105C081E080932C320E94A0
:10A680009DAB8BE592E30E949696C82F0E94E24B09
:10A6900001C0CEE88C2FDF91CF911F910F910895CB
:10A6A000CF93DF93CDB7DEB76897CDBFDEBF682FFE
:10A6B00070E080E090E00E940DD669837A838B83FE
:10A6C0009C831D821E821F82188619861A861B860D
:10A6D0001C861D861E861F86188A198A1A8A1B8A5E
:10A6E0001C8A1D8A1E8A1F8A188EAE014F5F5F4F1B
:10A6F000BA0188E797E40E94CA8280E06896CDBFDD
:10A70000DEBFDF91CF910895CF93DF93CDB7DEB752
:10A710006897CDBFDEBF6091AD3270E080E090E021
:10A720000E940DD669837A838B839C831D821E824F
:10A730001F82188619861A861B861C861D861E8611
:10A740001F86188A198A1A8A1B8A1C8A1D8A1E8AE1
:10A750001F8A188EAE014F5F5F4FBA0182E897E4FF
:10A760000E94CA8280E06896CDBFDEBFDF91CF91A4
:10A770000895CF93DF93CDB7DEB76897CDBFDEBF27
:10A78000682F70E080E090E00E940DD669837A83A4
:10A790008B839C831D821E821F82188619861A86CF
:10A7A0001B861C861D861E861F86188A198A1A8A91
:10A7B0001B8A1C8A1D8A1E8A1F8A188EAE014F5F53
:10A7C0005F4FBA018BEC97E40E94CA8280E06896E2
:10A7D000CDBFDEBFDF91CF910895CF93DF93CDB78B
:10A7E000DEB76897CDBFDEBF682F70E080E090E0F5
:10A7F0000E940DD669837A838B839C831D821E827F
:10A800001F82188619861A861B861C861D861E8640
:10A810001F86188A198A1A8A1B8A1C8A1D8A1E8A10
:10A820001F8A188EAE014F5F5F4FBA018CED97E41F
:10A830000E94CA8280E06896CDBFDEBFDF91CF91D3
:10A840000895CF93FC0160817181828193810E9480
:10A85000E1D560932B3210922D328BE592E38093F9
:10A86000593290935A3280912C32813011F41092E7
:10A870002C3210922E32109254320E944F96C09178
:10A880002B32C430C9F40E94335180913F300E9472
:10A890003D4F809140308093A5328091433080932A
:10A8A000AA3280E00E949CAE80E00E94ED5381E0DD
:10A8B0008093A432C0935F3281E0CF910C9461AA5F
:10A8C00080931D3380931E338093263380E0089558
:10A8D0002CEA35EC47E257E36091CB337091CC33EF
:10A8E0008091CD339091CE330E9470D71816B4F476
:10A8F0008091703390917133A0917233B091733322
:10A90000BC01CD019F772CEA35EC47E257E30E946A
:10A910006DD587FF03C010921D3303C081E0809383
:10A920001D3380E0089580931D33809170339091A2
:10A930007133A0917233B091733380931533909338
:10A940001633A0931733B093183380E008952CEAA0
:10A9500035EC47E257E36091CB337091CC33809173
:10A96000CD339091CE330E9470D71816B4F48091F5
:10A97000703390917133A0917233B0917333BC01F5
:10A98000CD019F772CEA35EC47E257E30E946DD565
:10A9900087FF03C010921E3303C081E080931E33F3
:10A9A00080E0089580931E338091703390917133CD
:10A9B000A0917233B09173338093193390931A330B
:10A9C000A0931B33B0931C3380E008952CEA35EC40
:10A9D00047E257E36091CB337091CC338091CD3314
:10A9E0009091CE330E9470D71816B4F480917033D2
:10A9F00090917133A0917233B0917333BC01CD014A
:10AA00009F772CEA35EC47E257E30E946DD587FF2C
:10AA100003C01092263303C081E08093263380E088
:10AA20000895809326338091703390917133A09173
:10AA30007233B09173338093223390932333A09376
:10AA40002433B093253380E00895BC018DEE90E26D
:10AA50000C94056281E080935232089581E08093E6
:10AA60005332089581E08093543208951F93CF9319
:10AA7000DF93CDB7DEB76897CDBFDEBF0E94899662
:10AA80008130B9F10E940BD20E94878280E00E943F
:10AA9000B2AB10E0812F0E946196AB01BC01812F07
:10AAA0000E94D44F1F5F1630A9F780E090E0A0E429
:10AAB000B0E489839A83AB83BC831D821E821F828C
:10AAC000188619861A861B861C861D861E861F867A
:10AAD000188A198A1A8A1B8A1C8A1D8A1E8A1F8A4A
:10AAE000188EBE016F5F7F4FCB010E94215480E022
:10AAF00001C08AE66896CDBFDEBFDF91CF911F917E
:10AB00000895809152328130A9F420912D32213064
:10AB100079F480912E3281110BC082E080932D3226
:10AB200085EF95E58093593290935A3220932E32D7
:10AB30001092523280915332813091F480912D32B3
:10AB4000882331F0823061F490912E32943051F4A8
:10AB50000E948996811104C0109253320E9436558A
:10AB600090912E32809154328130C1F42091533231
:10AB7000211114C09150933088F01092543295E016
:10AB800090932E3290932B3290912C32911104C0DD
:10AB900080932C320E949DAB0E94FB9E80E0089522
:10ABA00085E080932B3280912C32811105C081E0A9
:10ABB00080932C320C949DAB0895CF93DF93CDB747
:10ABC000DEB76897CDBFDEBF80912C32882311F1AC
:10ABD00080E090E0A0E4B0E489839A83AB83BC83F7
:10ABE0001D821E821F82188619861A861B861C8665
:10ABF0001D861E861F86188A198A1A8A1B8A1C8A35
:10AC00001D8A1E8A1F8A188EBE016F5F7F4FCB017F
:10AC10000E9421546896CDBFDEBFDF91CF91089589
:10AC2000CF93DF93CDB7DEB76897CDBFDEBF80E0AF
:10AC300090E0A0E4B0E489839A83AB83BC831D8257
:10AC40001E821F82188619861A861B861C861D8600
:10AC50001E861F86188A198A1A8A1B8A1C8A1D8AD0
:10AC60001E8A1F8A188EAE014F5F5F4FBA0181E2C4
:10AC700094E50E94CA826896CDBFDEBFDF91CF9176
:10AC80000895CF93DF93CDB7DEB76897CDBFDEBF12
:10AC900080E090E0A0E8B0E489839A83AB83BC8332
:10ACA0001D821E821F82188619861A861B861C86A4
:10ACB0001D861E861F86188A198A1A8A1B8A1C8A74
:10ACC0001D8A1E8A1F8A188EAE014F5F5F4FBA0120
:10ACD00081E294E50E94CA826896CDBFDEBFDF9113
:10ACE000CF910895CF93DF93CDB7DEB72797CDBF30
:10ACF000DEBF97E0EFEDF0E2DE01119601900D92DC
:10AD00009A95E1F7873050F4E1E0F0E0EC0FFD1F99
:10AD1000E80FF11D87FDFA95808101C080E227963A
:10AD2000CDBFDEBFDF91CF910895EF92FF920F93D9
:10AD30001F93CF93DF931F92CDB7DEB77C018B01BA
:10AD4000642F70E080E090E049830E940DD6F70107
:10AD5000618772878387948782E087834981E42FA4
:10AD6000F0E0EE0FFF1FE00FF11F659174914FE4CB
:10AD700050E086EA9CE30E9480E1BC01C7010F908D
:10AD8000DF91CF911F910F91FF90EF900C94A761ED
:10AD9000CF93DF93EC010E94F249482F61E573E104
:10ADA000CE01DF91CF910C94955640912B3262E108
:10ADB00073E10C94955640912C3269EE72E10C943B
:10ADC000955640912D3265ED72E10C949556409167
:10ADD0002E3267EA72E10C94955640912F326AE860
:10ADE00072E10C949556E0915932F0915A32E55B3C
:10ADF000FF4F408164EB73E10C949556E09159321A
:10AE0000F0915A32E45BFF4F408160EC71E10C94A9
:10AE10009556E0915932F0915A32448166E271E1DF
:10AE20000C949556E0915932F0915A32E65BFF4FFF
:10AE3000408163EF70E10C949556E0915932F091A6
:10AE40005A32E25BFF4F408169EA70E10C949556FB
:10AE5000E0915932F0915A32E15BFF4F408168E650
:10AE600070E10C949556E0915932F0915A32E75BBB
:10AE7000FF4F408169EF7FE00C949556CF93DF93AD
:10AE8000EC01E0915932F0915A32EF5AFF4F608154
:10AE900070E080E090E00E940DD669877A878B870A
:10AEA0009C8782E08F8380E0DF91CF910895CF93DC
:10AEB000DF93EC0160915B3270915C3280915D3286
:10AEC00090915E320E940DD669877A878B879C8726
:10AED00082E08F8380E0DF91CF910895CF93DF935D
:10AEE000EC01E0915932F0915A3260817181828196
:10AEF00093810E940DD669877A878B879C8782E031
:10AF00008F8380E0DF91CF910895CF93DF93EC01A1
:10AF100080912D32811105C019861A861B861C86E8
:10AF200014C00E94589669877A878B879C872091E6
:10AF3000405621110AC025E832E441E25DE30E9457
:10AF400012D869877A878B879C878C819D81FC01C9
:10AF5000EE0FFF1FE80FF91FEE0FFF1FEE0FFF1F91
:10AF6000EE0FFF1FE156FA4E85919491888784E099
:10AF70008F8380E0DF91CF910895CF93DF93EC0131
:10AF80002091593230915A32F901FD9660817181D8
:10AF90008281938169877A878B879C873E962081FF
:10AFA00021110AC025E832E441E25DE30E9412D893
:10AFB00069877A878B879C878C819D81FC01EE0F46
:10AFC000FF1FE80FF91FEE0FFF1FEE0FFF1FEE0F21
:10AFD000FF1FE156FA4E85919491888784E08F8314
:10AFE00080E0DF91CF910895CF93DF93EC018C81C6
:10AFF0009D810E940448682F8091593290915A3265
:10B000000E94734B69877A878B879C878C819D818F
:10B01000FC01EE0FFF1FE80FF91FEE0FFF1FEE0FF1
:10B02000FF1FEE0FFF1FE156FA4E8591949188871E
:10B0300084E08F8380E0DF91CF910895CF93DF93F9
:10B04000EC018C819D810E940448209159323091FD
:10B050005A322B55324369F4E82FF0E0EE0FFF1F10
:10B06000EE0FFF1FEB54FD4C608171818281938153
:10B0700002C00E94619669877A878B879C878C8142
:10B080009D81FC01EE0FFF1FE80FF91FEE0FFF1F60
:10B09000EE0FFF1FEE0FFF1FE156FA4E85919491C0
:10B0A000888784E08F8380E0DF91CF910895CF93EC
:10B0B000DF93EC018C819D810E940448E09159321C
:10B0C000F0915A3294E0899FE00DF11D1124458DD5
:10B0D000568D678D70A149875A876B877C878C81D5
:10B0E0009D81FC01EE0FFF1FE80FF91FEE0FFF1F00
:10B0F000EE0FFF1FEE0FFF1FE156FA4E8591949160
:10B10000888784E08F8380E0DF91CF910895CF938B
:10B11000DF93EC010E941A5D69857A858B859C8599
:10B120000E94E1D5462F60EE73E1CE01DF91CF9111
:10B130000C949556CF93DF93EC018C819D810E94F6
:10B140000448833054F48F3FA9F407C0CE010E9415
:10B15000C45D80E01CC08DE61AC020E030E040E411
:10B1600050E469857A858B859C850E9470D7181676
:10B1700094F3ECCF20E030E040E050E469857A853C
:10B180008B859C850E9470D718162CF3DFCFDF913A
:10B19000CF91089595E3899FF0011124E350FF4C6E
:10B1A00060817181828193810895CF92DF92EF92C5
:10B1B000FF92CF93DF936A017B0125E3829FC00159
:10B1C0001124885D9F4CFC01EB52FF4F408351835B
:10B1D00062837383EC01C352DF4F20E034E244E723
:10B1E00059E4C701B6010E9412D89B01AC0160E08E
:10B1F00070E080E89FE30E9474D5688379838A8336
:10B200009B83DF91CF91FF90EF90DF90CF900895D7
:10B21000CF92DF92EF92FF92CF93DF93EC01C9843C
:10B22000DA84EB84FC8420E034E244E759E4C7018B
:10B23000B6010E9470D7181664F420E034E244E7A7
:10B2400059E4C701B6010E9474D569877A878B8754
:10B250009C87CE010E94C162C984DA84EB84FC849D
:10B260008C819D810E94044825E3829FC0011124A6
:10B27000885D9F4CFC01EB52FF4FC082D182E2827D
:10B28000F382EC01C352DF4F20E034E244E759E49B
:10B29000C701B6010E9412D89B01AC0160E070E0CA
:10B2A00080E89FE30E9474D5688379838A839B83B7
:10B2B00080E0DF91CF91FF90EF90DF90CF900895E5
:10B2C000CF92DF92EF92FF92CF93DF93EC01C9848C
:10B2D000DA84EB84FC8420E034E244E759E4C701DB
:10B2E000B6010E9470D7181664F420E034E244E7F7
:10B2F00059E4C701B6010E9474D569877A878B87A4
:10B300009C87CE010E94C16280E0DF91CF91FF90C7
:10B31000EF90DF90CF90089581E08093533280E0EA
:10B3200008952CEA35EC47E257E3FC01618572850C
:10B33000838594850E9470D7181614F40E94B96A08
:10B3400080E0089560915532709156328091573265
:10B350009091583208950E94D05E80E00E943C6D2A
:10B3600080E008950E94D05E81E00E943C6D80E004
:10B3700008950E94D05E82E00E943C6D80E00895B6
:10B380000E94D05E83E00E943C6D80E00895CF93E0
:10B39000DF93EC01E0915932F0915A32E55BFF4FB7
:10B3A000E081F0E0EE0FFF1FED5EFB4E65917491C2
:10B3B0004FE450E086EA9CE30E9480E1AC0162EE3B
:10B3C0007FE0CE01DF91CF910C94E4C1CF93DF9366
:10B3D000EC01E0915932F0915A32E55BFF4FE08188
:10B3E000F0E0EE0FFF1FED5EFB4E659174914FE4B0
:10B3F00050E086EA9CE30E9480E1AC016AEC7FE0C9
:10B40000CE01DF91CF910C94E4C1CF93DF93EC0197
:10B4100081EF90E20E94E5E2CE010E94C759CE0181
:10B420000E94E65966EB7FE0CE010E94ABC16DE958
:10B430007FE0CE010E9476C164E87FE0CE010E94E9
:10B4400076C16BE67FE0CE010E9476C162E57FE0C7
:10B45000CE010E9476C169E37FE0CE010E9476C1F1
:10B4600060E27FE0CE010E9476C167E07FE0CE011E
:10B470000E9476C16EEE7EE0CE010E9476C165ED3F
:10B480007EE0CE010E9476C16CEB7EE0CE010E9490
:10B4900076C163EA7EE0CE010E9476C16AE87EE072
:10B4A000CE010E9476C161E77EE0CE010E9476C1A6
:10B4B00068E57EE0CE010E94ABC180E0DF91CF91D4
:10B4C000089566EB7FE00C94ABC16DE97FE00C94CE
:10B4D00076C164E87FE00C9476C16BE67FE00C9463
:10B4E00076C162E57FE00C9476C169E37FE00C945D
:10B4F00076C160E27FE00C9476C167E07FE00C9457
:10B5000076C16EEE7EE00C9476C165ED7EE00C9423
:10B5100076C16CEB7EE00C9476C163EA7EE00C941D
:10B5200076C16AE87EE00C9476C161E77EE00C9417
:10B5300076C168E57EE00C94ABC16CED7DE00C94C7
:10B54000ABC16BEA7DE00C94ABC166E77DE00C9487
:10B55000ABC16BE37DE00C94ABC167E07DE00C9484
:10B56000ABC1CF93DF93EC01E0915932F0915A32A5
:10B57000E55BFF4FE081F0E0EE0FFF1FED5EFB4E5D
:10B58000659174914FE450E086EA9CE30E9480E16B
:10B59000AC0163EE7CE0CE01DF91CF910C94E4C16D
:10B5A000CF93DF93EC01E0915932F0915A32E55B91
:10B5B000FF4FE081F0E0EE0FFF1FED5EFB4E659167
:10B5C00074914FE450E086EA9CE30E9480E1AC0174
:10B5D00062EC7CE0CE01DF91CF910C94E4C165EA8E
:10B5E0007CE00C948CC1CF93DF93EC01E091593255
:10B5F000F0915A32E55BFF4FE081F0E0EE0FFF1F64
:10B60000ED5EFB4E659174914FE450E086EA9CE359
:10B610000E9480E1AC0166E87CE0CE01DF91CF9131
:10B620000C94E4C10F931F93CF93DF938C01FC0123
:10B6300061857285838594850E94E1D5E62FF0E0CF
:10B64000EE0FFF1FE052FC4E659174914FE450E005
:10B6500086EA9CE30E9480E1E8012D969F938F93F8
:10B66000F80161857285838594850E94E1D51F92DA
:10B670006F93DF93CF930F5E1F4F1F930F93DF9353
:10B68000CF938AE69CE09F938F93EEEAF9E5818160
:10B690008F9380818F930E9447E2EDB7FEB73E966D
:10B6A000EDBFFEBFDF91CF911F910F91089562E42E
:10B6B0007CE00C9476486AE17CE00C94764868EF74
:10B6C0007BE00C94764866ED7BE00C94764864EA67
:10B6D0007BE00C94764863E77BE00C9476486AE361
:10B6E0007BE00C9476486AE17BE00C94764868ED48
:10B6F0007AE00C94444866E97AE00C9444486FE69A
:10B700007AE00C94764869E47AE00C94764868E232
:10B710007AE00C94764868E07AE00C9476486BEE18
:10B7200079E00C94C9486CEC79E00C94C948BC01F0
:10B73000675F7F4F2091A63242E45EE0FC01848186
:10B7400095810C942049BC01675F7F4F21E048E25E
:10B750005EE0FC01848195810C942049BC01675F07
:10B760007F4F21E04FE05EE0FC01848195810C94E5
:10B7700020490F931F93CF93DF93EC010C811D8120
:10B780000E94746408171907C4F48C819D81FC0120
:10B79000EE0FFF1FE80FF91FEE0FFF1FEE0FFF1F49
:10B7A000EE0FFF1FEC55FA4E25913491CE01F901B1
:10B7B000DF91CF911F910F91199485E1DF91CF9186
:10B7C0001F910F9108950F931F93CF93DF93EC0177
:10B7D0000C811D810E94746408171907C4F48C81C0
:10B7E0009D81FC01EE0FFF1FE80FF91FEE0FFF1FF9
:10B7F000EE0FFF1FEE0FFF1FEE55FA4E259134910D
:10B80000CE01F901DF91CF911F910F91199485E13C
:10B81000DF91CF911F910F9108950F931F93CF93B5
:10B82000DF93EC010C811D810E94746408171907D5
:10B83000C4F48C819D81FC01EE0FFF1FE80FF91FFE
:10B84000EE0FFF1FEE0FFF1FEE0FFF1FE056FA4E29
:10B8500025913491CE01F901DF91CF911F910F9184
:10B860001994DF91CF911F910F910895CF93DF939A
:10B87000EC018C819D810E9487648823C9F08C81B2
:10B880009D81FC01EE0FFF1FE80FF91FEE0FFF1F58
:10B89000EE0FFF1FEE0FFF1FE256FA4EE491E1FF9D
:10B8A00005C0CE01DF91CF910C94A38080E001C050
:10B8B00085E1DF91CF9108950F931F93CF93DF938D
:10B8C000EC0181E00E94834E1C821D8280E090E0AA
:10B8D0008E010F5E1F4F47C08C819D819C01220FFE
:10B8E000331FF901E80FF91FEE0FFF1FEE0FFF1FC7
:10B8F000EE0FFF1FE256FA4EE491E0FF2EC0280F34
:10B90000391F220F331F220F331F220F331F2855D9
:10B910003A4EF901459155916591749149875A873D
:10B920006B877C87BC01660F771F680F791F660FD6
:10B93000771F660F771F660F771F68567A4E45E0B0
:10B9400050E0C8010E9480E1CE010E94B95BCE01A7
:10B950000E94365C2C813D8101C09C012F5F3F4FCE
:10B960002C833D83C9010E9477648111B5CF81E0AA
:10B970000E9410A8DF91CF911F910F910C94F8A70E
:10B98000CF93DF93EC012CEA35EC47E257E369856E
:10B990007A858B859C850E946DD587FF05C0CE0179
:10B9A000DF91CF910C949D79CE010E945C5C82E086
:10B9B0008F8340E050E060E87FE349875A876B87D8
:10B9C0007C8780E0DF91CF910895809196399091A6
:10B9D00097398F3E924111F08AE508958091D839C8
:10B9E0009091D9398F3E9241B9F780916C34909102
:10B9F0006D348F3E924181F780918E3790918F37D1
:10BA00008F3E924149F780919037909191378F3EC8
:10BA1000924111F780919439909195398F3E9241DE
:10BA2000D9F68091F53C8111D7CF0895FC0117829A
:10BA300089E60895CF93DF93EC018C819D81FC0111
:10BA4000EE0FFF1FE80FF91FEE0FFF1FEE0FFF1F96
:10BA5000EE0FFF1FEA55FA4EA591B4916C9170E07C
:10BA600080E090E00E940DD669877A878B879C875B
:10BA700082E08F8380E0DF91CF910895CF93DF93B1
:10BA8000EC018C819D81FC01EE0FFF1FE80FF91F77
:10BA9000EE0FFF1FEE0FFF1FEE0FFF1FEA55FA4ECE
:10BAA000A591B4916D917D918D919C910E940DD63F
:10BAB00069877A878B879C8782E08F8380E0DF911C
:10BAC000CF910895CF93DF93DC0114968D919C91D3
:10BAD0001597FC01EE0FFF1FE80FF91FEE0FFF1F78
:10BAE000EE0FFF1FEE0FFF1FEA55FA4EC591D491DE
:10BAF000488159816A817B8119964D935D936D933D
:10BB00007C931C9783E017968C9380E0DF91CF9114
:10BB10000895CF93DF93DC0114968D919C91159736
:10BB2000FC01EE0FFF1FE80FF91FEE0FFF1FEE0FD6
:10BB3000FF1FEE0FFF1FEA55FA4EC591D4914881C1
:10BB400059816A817B8119964D935D936D937C93A6
:10BB50001C97FC01EE0FFF1FE80FF91FEE0FFF1FF0
:10BB6000EE0FFF1FEE0FFF1FE156FA4E85919491E5
:10BB700018968C93189784E017968C9380E0DF9149
:10BB8000CF91089588E608950F931F93CF93DF9385
:10BB9000EC018C819D81FC01EE0FFF1FE80FF91F66
:10BBA000EE0FFF1FEE0FFF1FEE0FFF1FEA55FA4EBD
:10BBB0000591149169857A858B859C850E94E1D5D4
:10BBC000F801608382E08F8380E0DF91CF911F9145
:10BBD0000F910895CF93DF93EC0169857A858B856A
:10BBE0009C850E94E1D56230B0F48C819D81FC017E
:10BBF000EE0FFF1FE80FF91FEE0FFF1FEE0FFF1FE5
:10BC0000EE0FFF1FEA55FA4EA591B4916C9382E0B6
:10BC10008F8380E001C08EE6DF91CF910895CF93AE
:10BC2000DF93EC0169857A858B859C850E94E1D53F
:10BC30006330B0F48C819D81FC01EE0FFF1FE80F93
:10BC4000F91FEE0FFF1FEE0FFF1FEE0FFF1FEA554C
:10BC5000FA4EA591B4916C9382E08F8380E001C08D
:10BC60008EE6DF91CF910895CF93DF93EC01698544
:10BC70007A858B859C850E94E1D56430B0F48C81F7
:10BC80009D81FC01EE0FFF1FE80FF91FEE0FFF1F54
:10BC9000EE0FFF1FEE0FFF1FEA55FA4EA591B4916C
:10BCA0006C9382E08F8380E001C08EE6DF91CF91BC
:10BCB00008950F931F93CF93DF93EC018C819D81A7
:10BCC000FC01EE0FFF1FE80FF91FEE0FFF1FEE0F35
:10BCD000FF1FEE0FFF1FEA55FA4E0591149169857B
:10BCE0007A858B859C850E94E1D5F80160837183FC
:10BCF00082E08F8380E0DF91CF911F910F910895B3
:10BD00000F931F93CF93DF93EC018C819D81FC01F6
:10BD1000EE0FFF1FE80FF91FEE0FFF1FEE0FFF1FC3
:10BD2000EE0FFF1FEA55FA4E0591149169857A8549
:10BD30008B859C850E94E1D5F801608371838283A5
:10BD4000938382E08F8380E0DF91CF911F910F91E9
:10BD50000895CF93DF93DC0114968D919C911597F4
:10BD6000FC01EE0FFF1FE80FF91FEE0FFF1FEE0F94
:10BD7000FF1FEE0FFF1FEA55FA4EC591D491199699
:10BD80004D915D916D917C911C97488359836A8395
:10BD90007B8383E017968C9380E0DF91CF910895A9
:10BDA000CF93DF93DC0114968D919C911597FC0144
:10BDB000EE0FFF1FE80FF91FEE0FFF1FEE0FFF1F23
:10BDC000EE0FFF1FEA55FA4EC591D49119964D9189
:10BDD0005D916D917C911C97488359836A837B8325
:10BDE000FC01EE0FFF1FE80FF91FEE0FFF1FEE0F14
:10BDF000FF1FEE0FFF1FE156FA4E859194911896A2
:10BE00008C93189784E017968C9380E0DF91CF9104
:10BE100008951F93CF93DF93EC018091F839882325
:10BE2000D1F01DE10A80DB81C02D209711F480E064
:10BE300013C08F818F3FD9F3811104C0CE010E94BE
:10BE4000E35B06C0CE010E94B95BCE010E94365C66
:10BE5000115041F7ECCF85E6DF91CF911F91089506
:10BE6000CF93DF93EC01BC018FEF90E20E94B9E128
:10BE7000892B41F0BE0182E091E20E94B9E121E00C
:10BE8000892B09F420E0822FDF91CF9108950F9341
:10BE90001F93CF93DF93CDB7DEB72997CDBFDEBF1A
:10BEA0008B0144E050E0BC01CE0101960E94D9E133
:10BEB00046E050E0B801CE0101960E94C9E10E941F
:10BEC0007464181619060CF03FC07981AA81BB81F1
:10BED0001C810D8128E935E140E050E0F9016491D1
:10BEE000671327C03196E491E11103C0A11121C06D
:10BEF00029C0EA131EC0F9013296E491E11103C092
:10BF0000B11117C01FC0EB1314C0F9013396E491AF
:10BF1000E11103C011110DC015C0E1130AC0F901F0
:10BF20003496E491E11103C0011103C00BC0E01786
:10BF300049F04F5F5F4F285E3F4F4817590709F0A0
:10BF4000CDCF02C0CA0102C08FEF9FEF2996CDBFAF
:10BF5000DEBFDF91CF911F910F910895CF93DF93B3
:10BF6000FC012189222371F1EC016196BE0186E07A
:10BF700091E20E94B9E1892B39F1BE018FEF90E285
:10BF80000E94B9E1892B11F1BE0189E091E20E9482
:10BF9000B9E1892BD9F0BE018DEE90E20E94B9E1A2
:10BFA000892BB1F0BE018CE091E20E94B9E1892BAE
:10BFB00079F0BE0180EE91E20E94B9E1892B51F443
:10BFC00085E009C080E007C082E005C083E003C0CF
:10BFD00084E001C081E0DF91CF910895FC018FEFF3
:10BFE0008783148215821186128613861486108622
:10BFF000118A1586178A108EA081B181109711F4CD
:10C0000016820DC017968C911797873029F41696D3
:10C010008C918F5F868303C016968C918683CF01A7
:10C020000895EF92FF920F931F93CF93DF93EC014C
:10C030000C811D810E947464081719070CF06FC0F1
:10C040000C811D81CE010E94EE5F0C831D837E0159
:10C0500081E1E80EF11CB801660F771F600F711FB8
:10C06000660F771F660F771F660F771F68567A4E29
:10C07000C7010E9461E18E01035F1F4F2C813D814A
:10C08000B901660F771F620F731F660F771F660F68
:10C09000771F660F771F6C567A4EC8010E9461E1C8
:10C0A0008D85882311F18C819D81FC01EE0FFF1F8E
:10C0B000E80FF91FEE0FFF1FEE0FFF1FEE0FFF1F20
:10C0C000E256FA4EE491E2FF02C01D8610C0F8016C
:10C0D00001900020E9F7BF01601B710B605F7F4F8B
:10C0E0006C0F7D1FC7010E94C2E18C819D81FC0104
:10C0F000EE0FFF1FE80FF91FEE0FFF1FEE0FFF1FE0
:10C10000EE0FFF1FEE55FA4E25913491CE01F90145
:10C11000DF91CF911F910F91FF90EF901994DF91D4
:10C12000CF911F910F91FF90EF9008958F929F9262
:10C13000AF92BF92CF92DF92EF92FF920F931F9335
:10C14000CF93DF9300D01F92CDB7DEB76C015C01B7
:10C1500081E1A80EB11C87E0F6018783A4E9EA2EED
:10C16000A5E1FA2E00E010E01DC0B701CE01019656
:10C170000E9461E1BE016F5F7F4FC5010E94B9E17E
:10C18000892B59F44601F9E18F0E911CF601058FB8
:10C19000168FC4010E94116064010F5F1F4FF8E108
:10C1A000EF0EF11CC8010E9477648111DECF249646
:10C1B000CDBFDEBFDF91CF911F910F91FF90EF9028
:10C1C000DF90CF90BF90AF909F908F900895CF93C6
:10C1D000DF931092923710929337A5E5B4E3EEE621
:10C1E000F4E391E08FEFA083B18379965B96ED93B2
:10C1F000FC935C975D961D921C925E97EF0163978E
:10C20000988322961882219788832A9618825996B5
:10C2100027E3EE38F20739F7109277371092783724
:10C2200010926E3410926F341092743487E08093C1
:10C23000753482E790E080937F349093803487E870
:10C2400094E3DF91CF9108950F931F93CF93DF93E2
:10C250000E94E760EC018FEE92E180939639909313
:10C2600097398093D8399093D93980936C349093CF
:10C270006D3480938E3790938F378093903790935F
:10C280009137809394399093953981E00E94834E41
:10C290001C821D82CE010E947A802091E03930916B
:10C2A000E1394091E2395091E33969857A858B858E
:10C2B0009C850E946DD5882339F0CE01DF91CF9106
:10C2C0001F910F910C945C5C0E94FDA71C821D8243
:10C2D00080E090E08E010F5E1F4F2FC06C817D814A
:10C2E0009B01220F331FF901E60FF71FEE0FFF1F0F
:10C2F000EE0FFF1FEE0FFF1FE256FA4EE491E0FF34
:10C3000017C0620F731F660F771F660F771F660FC8
:10C31000771F68567A4E45E050E0C8010E9480E1E0
:10C32000CE010E947A80CE010E94B95B6C817D8132
:10C330006F5F7F4F6C837D83CB010E947764811197
:10C34000CDCFDF91CF911F910F910C9410A8EF9258
:10C35000FF920F931F93CF93DF938C01209192371D
:10C3600030919337EB0109900020E9F72197C61B24
:10C37000D70BAE01420F531F41305240D8F4F901A0
:10C38000EC56F84C7F01AE014F5F5F4FCF010E942A
:10C390009AE140919237509193374F5F5F4F4C0F26
:10C3A0005D1F4093923750939337F801E78AF08EE0
:10C3B00080E001C08DE0DF91CF911F910F91FF9040
:10C3C000EF900895CF93DF932EE1C7E8D4E33F8148
:10C3D0003F3F59F00A80DB81C02D209719F480E09F
:10C3E00090E010C0215099F7FACFBC0184E493E2A9
:10C3F0000E94475F8C839D83019689F3CE010E9442
:10C400001160CE01DF91CF910895EF92FF920F93CB
:10C410001F93CF93DF938B012EE1C7E8D4E33F81D5
:10C420003F3F59F00A80DB81C02D209719F480E04E
:10C4300090E01DC0215099F7FACF7E0121E1E20E74
:10C44000F11C45E050E0BC01C7010E94D9E1B801F0
:10C45000CE010E94A7618111EACFB70184E493E283
:10C460000E94475F8C839D8385E08F83CE01DF919F
:10C47000CF911F910F91FF90EF9008952091F8397F
:10C48000213021F42091A23C213029F4BC018DEE11
:10C4900090E20C94056280E090E008959091F83964
:10C4A000913019F4642F0C94F67E0C94F6C0CF935F
:10C4B000DF93EC018091E52F811103C00E9403D22C
:10C4C00002C00E940EC9682F70E080E090E00E94D8
:10C4D0000DD669877A878B879C8782E08F8380E07F
:10C4E000DF91CF9108950F931F93CF93DF93CDB733
:10C4F000DEB7C058D109CDBFDEBFFC0161857285B2
:10C50000838594850E94E1D58FEF860F863030F0C9
:10C5100080E491E20E943E628EE62AC06093E02FA2
:10C5200081E08093E12FE62FF0E0EE0FFF1FE15A4C
:10C53000FA4E659174914FE450E086EA9CE30E94C4
:10C5400080E19F938F9386E294E19F938F938E0176
:10C550000F5F1F4F1F930F930E943BE3C8010E9480
:10C560003E620F900F900F900F900F900F9080E011
:10C57000C058DF4FCDBFDEBFDF91CF911F910F912C
:10C5800008950F931F93CF93DF93EC018BE592E314
:10C590000E944E4A882329F009851A858B859C853F
:10C5A00011C023E333E34BEC51E469857A858B8535
:10C5B0009C850E9412D88B01AB01BC0149875A8728
:10C5C0006B877C872C813D81F901EE0FFF1FE20F05
:10C5D000F31FEE0FFF1FEE0FFF1FEE0FFF1FEA55B9
:10C5E000FA4EA591B491A801BC014D935D936D9352
:10C5F0007C931397F901EE0FFF1FE20FF31FEE0F6D
:10C60000FF1FEE0FFF1FEE0FFF1FE156FA4E859141
:10C610009491888784E08F8380E0DF91CF911F9190
:10C620000F91089560E375E10C948CC16CE075E1A5
:10C630000C948CC160ED74E10C948CC16CE974E1D4
:10C640000C948CC16FE474E10C948CC11F93CF9354
:10C65000DF93EC0110E08881882301F10E94E760FC
:10C6600045E050E0BE0188E994E30E94D9E168E921
:10C6700074E384E493E20E94475F80938B34909349
:10C680008C3487E894E30E94116042E063E080E02C
:10C690000E944E621F5F26961D31E9F684E0DF910D
:10C6A000CF911F910895CF93DF93CDB7DEB7EC976D
:10C6B000CDBFDEBF8CE3E8E1F0E2DE011196019030
:10C6C0000D928A95E1F7CE0101960E942663EC96C1
:10C6D000CDBFDEBFDF91CF910895CF93DF93CDB76C
:10C6E000DEB7AA97CDBFDEBF8AE2E4E5F0E2DE0165
:10C6F000119601900D928A95E1F7CE0101960E9464
:10C700002663AA96CDBFDEBFDF91CF910895CF9368
:10C71000DF93CDB7DEB76E97CDBFDEBF8EE1EEE71C
:10C72000F0E2DE01119601900D928A95E1F7CE01BB
:10C7300001960E9426636E96CDBFDEBFDF91CF913A
:10C740000895CF93DF93EC0143E759E763E770E087
:10C75000498B5A8B6B8B7C8B0E94966042E063E026
:10C7600080E00E944E62CE010E948763CE010E944B
:10C770006D6320E731E340E0298B3A8B4B8BCE0190
:10C780000E94966042E063E080E00E944E62CE012B
:10C79000DF91CF910C945363CF92DF92EF92FF928F
:10C7A000FC01C184D284E384F48420E030E040E8DA
:10C7B0005FE3C701B6010E9470D71816FCF0C701ED
:10C7C000B6010E94E1D56093E22FC701B6019F77C1
:10C7D0002CEA35EC47E257E30E9470D718163CF478
:10C7E00060E470E080E00E9416C780E008C060E866
:10C7F00070E080E00E9416C780E001C08EE6FF90E6
:10C80000EF90DF90CF900895CF92DF92EF92FF925A
:10C81000FC01C184D284E384F48420E030E040E071
:10C8200050E4C701B6010E9470D71816FCF0C7018A
:10C83000B6010E94E1D56093E42FC701B6019F774E
:10C840002CEA35EC47E257E30E9470D718163CF407
:10C8500064E070E080E00E9416C780E008C068E0F5
:10C8600070E080E00E9416C780E001C08EE6FF9075
:10C87000EF90DF90CF900895CF92DF92EF92FF92EA
:10C88000FC01C184D284E384F48420E030E040E8F9
:10C890005FE3C701B6010E9470D71816FCF0C7010C
:10C8A000B6010E94E1D56093E32FC701B6019F77DF
:10C8B0002CEA35EC47E257E30E9470D718163CF497
:10C8C00060E170E080E00E9416C780E008C060E28E
:10C8D00070E080E00E9416C780E001C08EE6FF9005
:10C8E000EF90DF90CF9008958CE891E0089521E0DB
:10C8F0008334914008F020E0822F08959C012F5549
:10C90000314081E02932310508F080E0089521E0CE
:10C910008036914008F020E0822F0895CF92DF9278
:10C92000EF92FF92CF93DF93EC01C984DA84EB841A
:10C93000FC84A7019601C701B6010E9433D9811179
:10C940003CC0E894F7F82FEF3FEF4FE75FE7C701F0
:10C95000B6010E9433D981110AC02FEF3FEF4FE794
:10C960005FE7C701B6010E946DD5181634F18C81BE
:10C970009D81FC01EE0FFF1FE80FF91FEE0FFF1F57
:10C98000EE0FFF1FEE0FFF1FE256FA4EE491E3FF9A
:10C9900014C08BE592E30E944E4A81110EC025E837
:10C9A00032E441E25DE369857A858B859C850E944E
:10C9B00012D869877A878B879C87DF91CF91FF9008
:10C9C000EF90DF90CF9008958091E12F882349F078
:10C9D0001092E12F6091E02F80E00E941EC780E05E
:10C9E000089583E00895CF93DF93E091163AF09194
:10C9F000173A04C0E093163AF093173AEF01819189
:10CA0000982F9D7F9032B1F38930A1F34FE450E02D
:10CA1000BE018CE19CE30E94D9E16881611105C0EF
:10CA20008091F83981115CC028C0613221F4DF9116
:10CA3000CF910C942A55653221F4DF91CF910C945B
:10CA40002E556E3721F4DF91CF910C9432556B3710
:10CA500041F481E08093F839CE01DF91CF910C94BD
:10CA6000F37970E080E791E20E94AEE1892B59F002
:10CA70001092F839CE010E944EBD6CE17CE3DF914B
:10CA8000CF910C948EBE8091F839811109C0CE01EE
:10CA90000E9406706CE17CE3DF91CF910C948EBE16
:10CAA0000E94E760EC0127E633E640E0298B3A8BF1
:10CAB0004B8B6091163A7091173A0E94A76185E0FE
:10CAC0008F838091163A9091173A0E94067042E047
:10CAD00060E00E944E6280E0DF91CF910C9461AAE9
:10CAE000DF91CF910895FF920F931F93CF93DF9320
:10CAF0001F921F92CDB7DEB7F82EEAEDF9E324E9D5
:10CB000032E0DF01C9011D920197E9F72FEE32E112
:10CB10002083318320936C3C30936D3C00E010E225
:10CB20002CED33E40093E0391093E1392093E2399E
:10CB30003093E3390CEE11E528E73FE30093E43945
:10CB40001093E5392093E6393093E73900E010E09F
:10CB500020EA30E40093E8391093E9392093EA3968
:10CB60003093EB3900E010E020E83FE30093EC392C
:10CB70001093ED392093EE393093EF3983E08093B1
:10CB8000F9398F2D4A8369830E942EC76981862FC8
:10CB90000E9439C74A81842F0E9444C7F092DF2F38
:10CBA000F092DD2F0F900F90DF91CF911F910F9199
:10CBB000FF900895CF93DF931F921F92CDB7DEB7FA
:10CBC00080E6F82E01E010E00E945B788230E1F30D
:10CBD0000E9462788230C1F30E942D4A863009F0AB
:10CBE000D9C00E9418C58090FF399090003AA0905B
:10CBF000013AB090023A86169706A806B90620F7C1
:10CC00000E9418C56C597F4F8F4F9F4F6093FF391B
:10CC10007093003A8093013A9093023A0E94D17740
:10CC2000D3CF0E9429BC882329F08CEC0E946F4E40
:10CC3000823051F20E948155823031F20E94559D1E
:10CC4000823011F20E94E55C8093F63C81112EC087
:10CC50008091DA399091DB398F3E924109F0AAC078
:10CC600080916C3C90916D3C8F3E924109F0A2C046
:10CC700097C00E944F818093F63C811117C00E949B
:10CC8000B6B28093F63C811111C00E94D16F80939F
:10CC9000F63C81110BC00E943DC68093F63C811189
:10CCA00005C00E948AB3823031F48ECF0E946F4E4D
:10CCB0008230B9F789CF0E9493AA823009F484CFD9
:10CCC0000E94FFAB823009F47FCF0E94BBAC823060
:10CCD00009F47ACF09831A8368E17AE3CE010196D9
:10CCE0000E9453C78093163A9093173A8F3F2FEFC5
:10CCF000920739F48DE00E94584E823009F464CFD7
:10CD000004C0892B11F00E94F3640E94B48B82301E
:10CD100009F45ACF0E94086B823009F455CF0E9463
:10CD2000C76D823009F450CF0E94AC6F823009F495
:10CD300049CF0E94FC4B823009F444CF0E94048208
:10CD40008430F0F53FCF8091F939843038F484E0B5
:10CD50008093F9390E942E550E9402A883E090E04A
:10CD600089839A8368E17AE3CE0101960E9453C7D2
:10CD70008093163A9093173A8F3F2FEF920721F442
:10CD80008DE00E94584E1ECF892B09F41BCF0E94C4
:10CD9000F36418CF0E942D4A823009F44BCF41CF63
:10CDA0001092F63C0E942A4E8093F63C882309F4A8
:10CDB00060CF7CCFF092F63C80E60E946F4E78CF39
:10CDC0008091222A9091232A0E9477D0682F70E0C8
:10CDD00080E090E00E940FD620E030E048E451E48B
:10CDE0000E9470D787FFEECE0E94E464823009F083
:10CDF000AACFE8CE8091DF2F8093DD2F0895809316
:10CE0000DD2F08958093DE2F0895CF93C82F809152
:10CE10008F23882379F040E050E0BA018C2F0E94E4
:10CE2000D44FEC2FFF27E7FDF095E05DFD4C81E04E
:10CE300080830AC06C2F85EF95E50E94734BAB0190
:10CE4000BC018C2F0E94D44F4091B6235091B72340
:10CE50006091B8237091B9238C2F0E94D5588EEC25
:10CE600098E6809390239093912382E0CF91089548
:10CE7000CF92DF92EF92FF920F931F93CF93DF93A6
:10CE8000CDB7DEB7E097CDBFDEBF98E17E01A9E167
:10CE9000EA0EF11CF701A92F1192AA95E9F7FE01FC
:10CEA00031966F0111929A95E9F7F60194E08902A3
:10CEB000E00DF11D1124408F518F628F738F80E040
:10CEC00090E0A0E8BFE380839183A283B3830093C3
:10CED00098321093993220939A3230939B320E9469
:10CEE00087820E943255B601C7010E94FC5280938E
:10CEF000F63C811101C082E0E096CDBFDEBFDF913C
:10CF0000CF911F910F91FF90EF90DF90CF900895F8
:10CF10000F931F93E0918923FF27E7FDF095EB5FC7
:10CF2000FF4C9381913099F400919A2310919B23A7
:10CF300020919C2330919D234091A2235091A323C3
:10CF40006091A4237091A5230E9438671DC0E091D1
:10CF50008A23FF27E7FDF095EB5FFF4C938191302B
:10CF600099F400919A2310919B2320919C23309156
:10CF70009D234091A2235091A3236091A4237091FB
:10CF8000A52370580E9438678EEC97E68093902313
:10CF90009093912382E01F910F9108950F931F9317
:10CFA000CF93C82F85E3C802F0011124EF5FFE4C38
:10CFB00040815181628173818C2F0E94D5580091EC
:10CFC0009A2310919B2320919C2330919D23409183
:10CFD00096235091972360919823709199238C2FD9
:10CFE0000E9438678DE598E6809390239093912373
:10CFF00082E0CF911F910F9108950F931F9300919D
:10D000009A2310919B2320919C2330919D23409142
:10D01000A6235091A7236091A8237091A9230E9471
:10D02000386785E097E6809390239093912382E080
:10D030001F910F9108950E9487828091AF230E94D3
:10D040003D4F8091AE230E94834E8091B0230E9479
:10D05000874E8091B1230E94E8528091B223909133
:10D06000B323A091B423B091B523809398329093C9
:10D070009932A0939A32B0939B3264E08BE592E3AD
:10D080000E946B4A0E94DD5510922C3280E0089578
:10D09000CF93C82F4091B6235091B7236091B82306
:10D0A0007091B9230E94D5588C2F0E941B6880E094
:10D0B0000E9461AA80EFCF9108950F931F93E09192
:10D0C0008923FF27E7FDF095EB5FFF4C93819130BB
:10D0D00039F088E498E6809390239093912318C0C8
:10D0E00000919E2310919F232091A0233091A12392
:10D0F0004091A2235091A3236091A4237091A52372
:10D100000E9438678DEF97E6809390239093912348
:10D1100082E01F910F910895FF920F931F93CF9379
:10D12000DF93CDB7DEB7C058D109CDBFDEBFF82E33
:10D130000E94E7608EEFF81205C085E791E20E9439
:10D140003E6219C08F2D0E9472561F928F9324EB5E
:10D150003AE33F932F938E010F5F1F4F1F930F935F
:10D160000E943BE3C8010E943E620F900F900F9017
:10D170000F900F900F9042E062E080EF0E944E62AD
:10D180008F2D0E941B6880EFC058DF4FCDBFDEBFE0
:10D19000DF91CF911F910F91FF9008954F925F9271
:10D1A0006F927F929F92AF92BF92CF92DF92EF9257
:10D1B000FF920F931F93CF93DF938F3F09F045C0EA
:10D1C0002CEA35EC47E257E3609193337091943346
:10D1D00080919533909196330E9470D718160CF475
:10D1E00069C12CEA35EC47E257E360918B337091CB
:10D1F0008C3380918D3390918E330E9470D71816A6
:10D200000CF45DC12CEA35EC47E257E360918F33B3
:10D210007091903380919133909192330E9470D7A6
:10D2200018160CF455C12CEA35EC47E257E360912F
:10D230009733709198338091993390919A330E94EB
:10D2400070D718160CF43FC171C18230A1F52CEAD9
:10D2500035EC47E257E360918B3370918C338091CA
:10D260008D3390918E330E9470D718160CF427C11D
:10D270002CEA35EC47E257E360918F33709190339D
:10D2800080919133909192330E9470D718160CF4CC
:10D290001FC12CEA35EC47E257E360919733709158
:10D2A00098338091993390919A330E9470D71816D1
:10D2B0000CF409C131C18823D9F2813051F32CC15A
:10D2C0007E018DEEE80EF11CF70180819181A28133
:10D2D000B381BC01CD019F772CEA35EC47E257E3DF
:10D2E0000E946DD587FD46C06E01F1EFCF0ED11CB7
:10D2F000F601408051806280738020E030E0A90117
:10D30000C301B2010E946DD587FD34C0FE01EF520A
:10D31000FF4F208131814281538134976081718137
:10D32000828193810E94C4D39B01AC015F77C301CA
:10D33000B2010E94C5D32B013C019F772CEA35EC4A
:10D3400047E257E30E946DD587FD14C0AB2CAA0CB1
:10D350008A2D0E9423BC80938723992493949A0C4E
:10D36000892D0E9423BC80938823209187238227C4
:10D3700080FD02C08B2DDBC0B0928623F801808136
:10D380009181A281B381BF7780939A2390939B234D
:10D39000A0939C23B0939D23F7014081518162812A
:10D3A00073817F7740939E2350939F236093A023A4
:10D3B0007093A12320FF2DC0A092892390928A23ED
:10D3C00077FA709477F8709440929623509297234E
:10D3D0006092982370929923F60180819181A281B5
:10D3E000B3818093A2239093A323A093A423B0930B
:10D3F000A523CB50DF4F88819981AA81BB8180937F
:10D40000A6239093A723A093A823B093A9238A2DA2
:10D410002AC090928923A0928A2340929623509208
:10D4200097236092982370929923F60180819181CD
:10D43000A281B381B0588093A2239093A323A09399
:10D44000A423B093A523CB50DF4F88819981AA8173
:10D45000BB81B0588093A6239093A723A093A823C1
:10D46000B093A923892D0E9423BC8D7F813039F090
:10D470008EEC98E6809390239093912369C08091DD
:10D480008A230E9423BC811103C08FEF80938A23DB
:10D490008B2D0E94CA586093B6237093B723809354
:10D4A000B8239093B92388E897E6809390239093CC
:10D4B00091234EC082E090E032E0B32E0DC080E0B8
:10D4C00090E0B12C09C083E090E023E0B22E04C0CC
:10D4D00081E090E0BB24B394FC01E05DFD4C108240
:10D4E00025E3289FE001299FD00D1124C85DDF4C62
:10D4F0008E0107511F4FF80180819181A281B38174
:10D50000BC01CD019F772CEA35EC47E257E30E943E
:10D510006DD587FFD5CE2ECF81E080932F328BE162
:10D5200098E6809390239093912312C08EEFDF9121
:10D53000CF911F910F91FF90EF90DF90CF90BF9010
:10D54000AF909F907F906F905F904F900C948C68FD
:10D5500082E0DF91CF911F910F91FF90EF90DF90CC
:10D56000CF90BF90AF909F907F906F905F904F90C3
:10D570000895CF93DF93C9E5D2E3888199810E9412
:10D580004E4A8093AE23888199810E94494A8093B4
:10D59000AF23888199810E94584A8093B023888163
:10D5A00099810E945D4A8093B123888199810E946C
:10D5B000644A6093B2237093B3238093B42390930F
:10D5C000B52381E00E94834E81E00E94874E80E077
:10D5D0000E943D4F81E00E94E85281E080938F23BA
:10D5E0008FEF809386238EEC98E680939023909320
:10D5F000912383E080932C3210922F3280E0DF91D0
:10D60000CF9108950E94B96A10928F2380E0089507
:10D6100080912C32833059F40E94624A813049F063
:10D62000E0919023F091912380918623199483E0D7
:10D63000089582E0089583E29BE68093CB23909344
:10D64000CC2382E008952F923F924F925F926F9287
:10D650007F928F929F92AF92BF92CF92DF92EF9282
:10D66000FF920F931F93CF93DF93CDB7DEB7CA54CA
:10D67000D109CDBFDEBF98E19E01275E3F4F29ABA8
:10D680003AABD901E92F1D92EA95E9F72851310902
:10D690001901D9011D929A95E9F724E08202F0015F
:10D6A00011242B96EEAFFFAF2B97E20DF31D80E018
:10D6B00090E0A0E8BFE380839183A283B383C0900E
:10D6C000C323D090C423E090C523F090C62340909C
:10D6D000BF235090C0236090C1237090C2238090DC
:10D6E000BB239090BC23A090BD23B090BE23A50186
:10D6F0009401C301B2010E946DD518165CF080E060
:10D7000090E0A0E8BFE329968CAF9DAFAEAFBFAF6E
:10D7100029970AC080E090E0A0E8BFEB29968CAF83
:10D720009DAFAEAFBFAF2997A3019201C501B40170
:10D730000E94C4D30E94DCD59B0177FF04C022273E
:10D740003327261B370BB901882777FD8095982F43
:10D750000E940FD625966CAF7DAF8EAF9FAF2597F9
:10D76000C0929832D0929932E0929A32F0929B32E3
:10D770000E9487820E94325520E030E040E050E471
:10D7800025966CAD7DAD8EAD9FAD25970E9470D76F
:10D7900018166CF08091C7239091C823A091C923DB
:10D7A000B091CA238BAF9CAFADAFBEAFDBC02AE058
:10D7B00037ED43E25CE325966CAD7DAD8EAD9FAD5C
:10D7C00025970E9470D718162CF709E110E08AE01F
:10D7D000882E87ED982E83E2A82E8CE3B82E412C5C
:10D7E000512C32012B96AEADBFAD2B97A20DB31DC0
:10D7F00058962196AEAFBFAF21974BAA5CAA6DAAEF
:10D800007EAA8FAA98AEA9AEBAAE29962CAD3DAD30
:10D810004EAD5FAD29976FA978AD89AD9AAD0E94E5
:10D8200012D89B01AC016091BF237091C0238091FD
:10D83000C1239091C2230E94C5D32196EEADFFADC6
:10D8400021976083718382839383C0929832D092B0
:10D850009932E0929A32F0929B32B101CE01499610
:10D860000E94FC528093F63C8111AAC020E030E077
:10D8700040E85FE36BA97CA98DA99EA90E94C5D34E
:10D880006BAB7CAB8DAB9EAB20E030E048EC51E461
:10D890000E9474D59B01AC0160E070E080E291E4ED
:10D8A0000E9475D82B013C018091C7239091C82319
:10D8B000A091C923B091CA238BAF9CAFADAFBEAFCF
:10D8C000C090C323D090C423E090C523F090C6231A
:10D8D000A7019601BC01CD010E94C4D34B015C019C
:10D8E00020E030E040E251E4C301B2010E9474D56F
:10D8F0009B01AC01C501B4010E9412D89B01AC018F
:10D90000C701B6010E94C5D36B017C012BA93CA9BC
:10D910004DA95EA9CA01B9010E94C5D320E030E03B
:10D9200048EC51E40E9474D59B01AC016FA978AD1D
:10D9300089AD9AAD0E94C5D36FAB78AF89AF9AAF6E
:10D940009B01AC0125966CAD7DAD8EAD9FAD25974D
:10D950000E9470D7181634F40150110901151105F1
:10D9600009F053CF8BAD9CADADADBEAD8093983279
:10D9700090939932A0939A32B0939B322B96EEAD4E
:10D98000FFAD2B97E20DF31D8091BB239091BC233B
:10D99000A091BD23B091BE23808F918FA28FB38FB2
:10D9A000B101CE0149960E94FC528093F63C811150
:10D9B00007C087EF9CE68093CB239093CC2382E033
:10D9C000C65BDF4FCDBFDEBFDF91CF911F910F91BF
:10D9D000FF90EF90DF90CF90BF90AF909F908F908F
:10D9E0007F906F905F904F903F902F900895CF93CE
:10D9F000DF931F92CDB7DEB789830E948782409163
:10DA0000D5235091D6236091D7237091D823898153
:10DA10000E94D5588091D2230E943D4F8091D123FE
:10DA20000E94834E8091D3230E94874E8091D423FD
:10DA30000E94E8528091CD239091CE23A091CF23D4
:10DA4000B091D0238093983290939932A0939A32D8
:10DA5000B0939B3264E08BE592E30E946B4A0E9494
:10DA6000DD5510922C3281EA91E20E94E5E280E0DD
:10DA70000F90DF91CF9108950F931F93CF93C82FED
:10DA800009E512E3F801808191810E944E4A80935A
:10DA9000D123F801808191810E94494A8093D22349
:10DAA000F801808191810E94584A8093D323F80124
:10DAB000808191810E945D4A8093D423F801808106
:10DAC00091810E94644A6093CD237093CE2380930A
:10DAD000CF239093D0238C2F0E94CA586093D523D4
:10DAE0007093D6238093D7239093D82381E00E940C
:10DAF000834E80E00E94874E80E00E943D4F81E08F
:10DB00000E94E85240E050E060E271E44093C32399
:10DB10005093C4236093C5237093C62385E3C89FA5
:10DB2000F0011124EF50FF4C4081518162817381DB
:10DB30004093C7235093C8236093C9237093CA238B
:10DB40006C2F85EF95E50E94604B6093BF23709327
:10DB5000C0238093C1239093C2230E94A259609353
:10DB6000BB237093BC238093BD239093BE23C093AB
:10DB7000BA238BE19BE68093CB239093CC2384E064
:10DB800080932C3280E0CF911F910F910895809166
:10DB90002C32843059F40E94624A813049F0E0917D
:10DBA000CB23F091CC238091BA23199483E008957C
:10DBB00082E00895E091DB23F0E0EB5FFF4C83818E
:10DBC000882341F085EF9DE68093D9239093DA2353
:10DBD00082E0089568E274E280E194E20E94FC52DF
:10DBE0008093F63C882371F308951F93CF93DF93BE
:10DBF000E091DB23F0E0EB5FFF4C81E0938191301B
:10DC000009F080E080933632C7E3D2E310E0812F41
:10DC10000E947596AB01BC01812F0E94D44F612FE9
:10DC20008091593290915A320E94604B6993799356
:10DC3000899399931F5F163051F78BEA91E20E9406
:10DC4000F37981E69EE68093D9239093DA2382E0EC
:10DC5000DF91CF911F9108951F93CF93DF930E947F
:10DC600087828091DC2380930530E091DB23F0E014
:10DC70008091DD23EB5FFF4C83870E9440BCC0EEA8
:10DC8000D3E210E04991599169917991812F0E94D5
:10DC9000D5581F5F1630B1F78091DF230E943D4FAA
:10DCA0008091DE230E94874E64E08BE592E30E9420
:10DCB0006B4A0E94DD5510922C32DF91CF911F915B
:10DCC00008950E942C6E80E008950F931F93CF93C8
:10DCD000DF93CDB7DEB7C058D109CDBFDEBF182F57
:10DCE0000E94E7601E3F29F488EB91E20E943E62A9
:10DCF00019C0812F0E9472561F928F9382EE9AE371
:10DD00009F938F938E010F5F1F4F1F930F930E945E
:10DD10003BE3C8010E943E620F900F900F900F905E
:10DD20000F900F9042E062E08AEF0E944E620E94E4
:10DD30002C6E8AEFC058DF4FCDBFDEBFDF91CF9191
:10DD40001F910F910895FF920F931F93CF93DF932D
:10DD50001092363282E080932C3200EE13E2C1E062
:10DD6000D1E3F12C8F2D0E94CA58F8016193719371
:10DD7000819391938F01488159816A817B818F2D95
:10DD80000E94D5586F2D8091593290915A320E943D
:10DD9000604BF801648B758B868B978BF394E596BB
:10DDA000F6E0FF12DFCF60E174E288EF93E20E94B9
:10DDB0001BC22AE43CE042E85EE30E946DD587FF87
:10DDC00003C08EEF0E94656EC4E0D4E213E0699157
:10DDD0007991899199912C893D894E895F890E9419
:10DDE000C4D39F772CEA35EC47E257E30E9470D703
:10DDF00018161CF4812F0E94656E1F5F163039F7CC
:10DE000084E08093DB23809114308093DD2381E0D4
:10DE100080931430809105308093DC23109205307C
:10DE20000E9440BC8091593290915A320E94494AD6
:10DE30008093DF238091593290915A320E94584A40
:10DE40008093DE2380E00E94874E80E00E943D4F59
:10DE500080E00E949CAE8AED9DE68093D92390934A
:10DE6000DA2382E0DF91CF911F910F91FF90089507
:10DE70000F931F93CF93DF938C01EB018091A4321A
:10DE8000882399F08091983290919932A0919A329A
:10DE9000B0919B32BC01CD019F772CEA35EC47E273
:10DEA00057E30E946DD587FD4FC088819981AA8173
:10DEB000BB81BC01CD019F772CEA35EC47E257E3EB
:10DEC0000E9470D71816F4F48C819D81AE81BF81B9
:10DED000BC01CD019F772CEA35EC47E257E30E9465
:10DEE00070D718167CF488859985AA85BB85BC01F6
:10DEF000CD019F772CEA35EC47E257E30E9470D7BB
:10DF0000181624F188E1F801A0E1B4E201900D9225
:10DF10008A95E1F788E1FE01A8E2B4E201900D9252
:10DF20008A95E1F788E1E7E3F2E3DF011D928A9544
:10DF3000E9F782E08093363283EA9EE68093D92324
:10DF40009093DA2380E003C08EE801C086E8DF9179
:10DF5000CF911F910F91089580912C32823021F042
:10DF600080913632823049F40E94624A813039F021
:10DF7000E091D923F091DA23199483E0089582E0A7
:10DF80000895EEE6FCE380E2DF011D928A95E9F751
:10DF90008FEE92E180938C3C90938D3C80839183B3
:10DFA000089580918C3C90918D3C8F3E924111F070
:10DFB0008CE5089580916E3C90916F3C8F3E92412C
:10DFC000B9F780E00895CF93DF93C82FCB01BA0152
:10DFD0000E94C1D827E0C29FE0011124C259D34C4E
:10DFE0000E94DCD56D837E838F839887DF91CF91EC
:10DFF000089597E0899FF0011124E259F34C65815F
:10E000007681878190850E940FD608952F923F9246
:10E010004F925F926F927F928F929F92AF92BF9238
:10E02000CF92DF92EF92FF920F931F93CF93DF93E4
:10E03000CDB7DEB72797CDBFDEBF8C011B828091A5
:10E040002B32823009F40EC7D801BC90B11037C70B
:10E0500080E06E01B3E0CB0ED11C3DC0F6018081A3
:10E06000811108C0B72CD7011C926E01B3E0CB0E12
:10E07000D11C22C7883239F4B72CF7011082FFEF88
:10E08000CF1ADF0A19C78B33B9F3A82EB12CC501FB
:10E090000E9435E1892B39F4B50182EE91E20E94AC
:10E0A000AEE1892B51F047018FEF881A980AC5011C
:10E0B0000E9459E1D7018C937401BFEFCB1ADB0AA0
:10E0C000F70180818111CACFB72CD8018C916E01E4
:10E0D000B3E0CB0ED11CF8011CC08E32E1F090E011
:10E0E000C0970A9790F08181803391F4828190E00B
:10E0F000C0970A9760F4DF01119611968C911197E1
:10E100008D938111FACF808104C0818101C080E3A9
:10E1100031968111E2CFF601A080A11007C036C070
:10E12000D6011196AC90BFEFCB1ADB0A76018A2C90
:10E13000912CC4010E9449E1892B91F7C4010E94EE
:10E1400051E18D369105A1F4F601818190E00E94A4
:10E1500051E18337910561F4D60112968C9190E0DC
:10E160000E9451E18736910519F4F601339602C0F9
:10E17000FE013396AA2061F08A2DD701893209F475
:10E180001C9211968C918111F9CF02C0FE01339639
:10E19000BFE2BB1609F468C68081882319F0CF015D
:10E1A0000E94255580E1EEE8FCE3DF011D928A958F
:10E1B000E9F78BE5E4E8F3E3DF01982F1D929A95E8
:10E1C000E9F7E9E2F3E3DF011D928A95E9F78BE5D0
:10E1D00092E30E94464A80932A33812C912C80E856
:10E1E000A82E8FE3B82E5524539492E0492E24E0B4
:10E1F000322E23C4C701B6010E94E1D5862F90E0DC
:10E200008F35910508F034C6FC01EC50FF4F0C949B
:10E21000B8DD10922A335092853380918F3C8F5F06
:10E2200080938F3C0AC450922A3350928533809158
:10E230008F3C8F5F80938F3C00C440922A33509272
:10E24000853380918F3C8F5F80938F3CF6C383E052
:10E2500080932A335092853380918F3C8F5F8093D7
:10E260008F3CEBC38DE08093293350928433E5C318
:10E2700088E0B2C0109259335092B4338091903CF0
:10E280008F5F8093903CD9C3509259335092B433EE
:10E290008091903C8F5F8093903CCFC340925933E4
:10E2A0005092B4338091903C8F5F8093903CC5C373
:10E2B00010925A335092B5338091933C8F5F809384
:10E2C000933CBBC350925A335092B5338091933CE8
:10E2D0008F5F8093933CB1C3C701B6010E942CD9D4
:10E2E0006C837D838E839F8320E030E040E251E4A5
:10E2F000C701B6010E9412D86B017C0120E030E01A
:10E3000040E251E46C817D818E819F810E9412D810
:10E310009B01AC01C701B6010E94C4D30E94E1D5A4
:10E32000623001F128F4662341F0613089F0A0C524
:10E330006330E9F0643001F19BC5B5E0B093293357
:10E340005092843380918E3C8F5F80938E3C75C356
:10E35000309229336093843380918E3C8F5F809319
:10E360008E3C6BC3509229335092843366C34092E3
:10E3700029335092843361C383E0809329335092D0
:10E3800084335BC3C701B6010E942CD96C837D83A3
:10E390008E839F8320E030E040E251E4C701B60164
:10E3A0000E9412D86B017C0120E030E040E251E491
:10E3B0006C817D818E819F810E9412D89B01AC016E
:10E3C000C701B6010E94C4D30E94E1D5662319F0AB
:10E3D000613061F04DC587E08093293350928433DA
:10E3E00080918E3C8F5F80938E3C27C3E6E0E09364
:10E3F00029336093843380918E3C8F5F80938E3C71
:10E400001CC3C701B6010E942CD96C837D838E8307
:10E410009F8320E030E040E251E4C701B6010E9452
:10E4200012D86B017C0120E030E040E251E46C81C5
:10E430007D818E819F810E9412D89B01AC01C70112
:10E44000B6010E94C4D30E94E1D5623009F010C524
:10E450008EE08093293350928433EFC250925C3324
:10E460005092B733EAC250925B335092B6338091E8
:10E47000973C8F5F8093973CE0C240925B33509211
:10E48000B6338091973C8F5F8093973CD6C283E0F0
:10E4900016C030925B335092B6338091973C8F5FB9
:10E4A0008093973CCAC2F5E0F0935B335092B63349
:10E4B0008091973C8F5F8093973CBFC286E08093AA
:10E4C0005B335092B6338091973C8F5F8093973C3B
:10E4D000B4C2C701B6010E942CD96C837D838E83A0
:10E4E0009F8320E030E040E251E4C701B6010E9482
:10E4F00012D86B017C0120E030E040E251E46C81F5
:10E500007D818E819F810E9412D89B01AC01C70141
:10E51000B6010E94C4D30E94E1D5662319F0613090
:10E5200059F0A6C410925E335092B9338091983C52
:10E530008F5F8093983C81C260935E336093B93360
:10E540008091983C8F5F8093983C77C240925E3375
:10E550005092B9338091983C8F5F8093983C6DC204
:10E5600030922A335092853380918F3C8F5F809315
:10E570008F3C63C2C701B6010E942CD96C837D8396
:10E580008E839F8320E030E040E251E4C701B60172
:10E590000E9412D86B017C0120E030E040E251E49F
:10E5A0006C817D818E819F810E9412D89B01AC017C
:10E5B000C701B6010E94C4D30E94E1D5662319F0B9
:10E5C000613059F055C410925F335092BA33809144
:10E5D000913C8F5F8093913C30C210926033609386
:10E5E000BB338091913C8F5F8093913C26C2C701E1
:10E5F000B6010E942CD96C837D838E839F8320E09B
:10E6000030E040E251E4C701B6010E9412D86B012C
:10E610007C0120E030E040E251E46C817D818E811C
:10E620009F810E9412D89B01AC01C701B6010E94D4
:10E63000C4D30E94E1D5662319F0613059F018C4A3
:10E6400050925F335092BA338091913C8F5F8093A8
:10E65000913CF3C1609360336093BB338091913CF4
:10E660008F5F8093913CE9C1C701B6010E942CD90C
:10E670006C837D838E839F8320E030E040E251E411
:10E68000C701B6010E9412D86B017C0120E030E086
:10E6900040E251E46C817D818E819F810E9412D87D
:10E6A0009B01AC01C701B6010E94C4D30E94E1D511
:10E6B000613089F028F06230A1F06330C1F0D8C336
:10E6C00099E0909329335092843380918E3C8F5FF0
:10E6D00080938E3CB2C1AAE0A09329336093843327
:10E6E000ACC1BBE0B093293350928433A6C1ECE0B7
:10E6F000E093293350928433A0C110925433509246
:10E70000AF338091923C8F5F8093923C96C1509240
:10E7100054335092AF338091923C8F5F8093923C00
:10E720008CC1C701B6010E94E1D5862F90E08D33E0
:10E73000910508F09BC3FC01ED5AFE4F0C94B8DD27
:10E7400010922B33509286338091993C8F5F809347
:10E75000993C73C150922B33509286338091993CEF
:10E760008F5F8093993C69C1509266335092C13358
:10E7700080919B3C8F5F80939B3C5FC1409266334E
:10E780005092C13380919B3C8F5F80939B3C55C1DD
:10E79000109266335092C13380919B3C8F5F80937F
:10E7A0009B3C4BC1509263335092BE3346C1509252
:10E7B00064335092BF3380919C3C8F5F80939C3C2C
:10E7C0003CC1509265335092C03380919C3C8F5F26
:10E7D00080939C3C32C1109265335092C03380913B
:10E7E0009C3C8F5F80939C3C28C150925733509241
:10E7F000B23380919D3C8F5F80939D3C1EC11092EF
:10E8000057335092B23380919D3C8F5F80939D3CF3
:10E8100014C1509255335092B03380919D3C8F5F1C
:10E8200080939D3C0AC150926F335092CA338091BD
:10E830009D3C8F5F80939D3C00C1C701B6010E9443
:10E840002CD90E94E1D5609362335092BD33F5C05C
:10E85000C0924833D0924933E0924A33F0924B331E
:10E860008092A3339092A433A092A533B092A633A2
:10E87000E4C0C0927033D0927133E0927233F09260
:10E8800073338092CB339092CC33A092CD33B0923D
:10E89000CE33D3C0C0926733D0926833E0926933ED
:10E8A000F0926A338092C2339092C333A092C43301
:10E8B000B092C533C2C0C0923033D0923133E092AF
:10E8C0003233F092333380928B3390928C33A09218
:10E8D0008D33B0928E33B1C0C0923433D092353381
:10E8E000E0923633F092373380928F3390929033A8
:10E8F000A0929133B0929233A0C0C0923833D0929C
:10E900003933E0923A33F0923B33809293339092D2
:10E910009433A0929533B09296338FC0C0923C331B
:10E92000D0923D33E0923E33F0923F338092973362
:10E9300090929833A0929933B0929A337EC0C0924D
:10E940004033D0924133E0924233F092433380928D
:10E950009B3390929C33A0929D33B0929E336DC0B6
:10E96000C0924433D0924533E0924633F09247331D
:10E9700080929F339092A033A092A133B092A233A1
:10E980005CC0C0927833D0927933E0927A33F092BF
:10E990007B338092D3339092D433A092D533B0920C
:10E9A000D6334BC0C0927C33D0927D33E0927E331D
:10E9B000F0927F338092D7339092D833A092D9339C
:10E9C000B092DA333AC0C0928033D0928133E09271
:10E9D0008233F09283338092DB339092DC33A092C7
:10E9E000DD33B092DE3329C0C0927433D0927533D8
:10E9F000E0927633F09277338092CF339092D03397
:10EA0000A092D133B092D23318C0C701B6010E9490
:10EA1000E1D560932C3370932D3380932E339093F4
:10EA20002F3381E090E0A0E0B0E0809387339093B3
:10EA30008833A0938933B0938A33D8012C90222055
:10EA400009F424C2822D90E00E9440E1892B09F450
:10EA50002FC23801BFEF6B1A7B0AF8018181803326
:10EA600049F48281883531F40E5F1F4FC12CD12CBF
:10EA7000760100C2BE016F5F7F4FC3010E94D8DDE7
:10EA80006B017C0109811A816016710609F0F2C1DF
:10EA900011C2809154330E94E852182F01C010E037
:10EAA0006091A3337091A4338091A5339091A633E4
:10EAB0000E94E1D5662359F0609148337091493343
:10EAC00080914A3390914B330E94B752182F609136
:10EAD000A7337091A8338091A9339091AA330E94F3
:10EAE000E1D5662371F060914C3370914D33809184
:10EAF0004E3390914F330E94E1D5862F0E9493545C
:10EB0000182F6091AB337091AC338091AD339091FD
:10EB1000AE330E94E1D5662371F06091503370915D
:10EB2000513380915233909153330E94E1D5862F17
:10EB30000E94D254182F6091C2337091C3338091D8
:10EB4000C4339091C5330E94E1D5662359F060919A
:10EB50006733709168338091693390916A330E9472
:10EB6000D0AE182F6091C6337091C7338091C833EF
:10EB70009091C9330E94E1D5662371F060916B33A7
:10EB800070916C3380916D3390916E330E94E1D51A
:10EB9000862F0E941155182F8091BD33882329F0AC
:10EBA000809162330E945053182F8091BE33882386
:10EBB00029F0809163330E948453182F8091C133D0
:10EBC000882329F0809166330E949CAE182F809193
:10EBD000BF33882329F0809164330E94B953182FE2
:10EBE0008091C033882329F0809165330E94ED53D2
:10EBF000182F8091B033882329F0809155330E94DB
:10EC00006854182F8091B133882329F080915633AE
:10EC10000E94A754182F8091CA33882329F080912D
:10EC20006F330E94E654182F8091B233882329F065
:10EC3000809157330E946054182F809129338D3072
:10EC400029F08091B4338823A9F00FC0609170330C
:10EC50007091713380917233909173330E94F052AE
:10EC60008093F63C882369F32FC1809159330E9429
:10EC70007F4E182F8091B533882329F080915A3325
:10EC80000E94834E182F8091B633882329F08091FB
:10EC90005B330E943D4F182F8091B933882329F0B0
:10ECA00080915E330E94EC52182F8091BA338823F2
:10ECB00029F080915F330E94874E182F40912933AD
:10ECC00050E04F30510508F0B6C0FA01E057FE4F52
:10ECD0000C94B8DD0E943952182FADC06BE873E375
:10ECE00080E393E30E944452182FA5C00E947852FB
:10ECF000182FA1C06BE873E380E393E30E94835273
:10ED0000182F99C00E94B96A182F95C06BE873E359
:10ED100080E393E30E940350182F8DC00E94026B82
:10ED2000182F89C06BE873E380E393E30E94386F88
:10ED3000182F81C06091703370917133809172335C
:10ED4000909173330E94E1D5862F2BE833E340E3A3
:10ED500053E3609158330E948B4E182F6CC06BE8C0
:10ED600073E380E393E30E948050182F64C00E94F5
:10ED70003351182F60C00E949A51182F5CC00E9416
:10ED8000D151182F58C060915C338BE592E30E94FB
:10ED9000E14A80912A33843038F48230D8F48823D1
:10EDA00049F0813079F047C0843009F044C0809345
:10EDB0005F3241C06BE873E380E393E30E94095242
:10EDC000182F39C06BE873E380E393E30E94FC5291
:10EDD000182F31C0A0908033B0908133C09082331F
:10EDE000D0908333E0907C33F0907D3300917E337C
:10EDF00010917F33209178333091793340917A3379
:10EE000050917B338F93809177338F9380917633BA
:10EE10008F93809175338F93809174338F936BE8C8
:10EE200073E380E393E30E941784182F0F900F90F1
:10EE30000F900F900F9060E08BE592E30E94E14A03
:10EE400080918633813061F480912B33811104C02D
:10EE50000E941056812F38C00E944156812F34C025
:10EE6000812F32C08BEC30C083E02EC084E82CC0F0
:10EE700083E82AC0822D90E0FC01E154F109EA31D7
:10EE8000F105B0F7E156FE4F0C94B8DD1092F63C58
:10EE900060912C3370912D3380912E3390912F33CC
:10EEA0000E947B4A8091AF33882309F4F8CDF1CDDD
:10EEB00085E60AC086E608C0D8018C910CC96801B5
:10EEC0008B2D78017B2CD6C82796CDBFDEBFDF9176
:10EED000CF911F910F91FF90EF90DF90CF90BF9057
:10EEE000AF909F908F907F906F905F904F903F90EA
:10EEF0002F900895CF93DF93EC016CE17CE30E94A7
:10EF0000A7618093F63C811102C095E09F83DF9159
:10EF1000CF910895FC018789908D0C94067083FF32
:10EF200006C0E091FD2FF091FE2F90E2958382FFC5
:10EF300006C0E091FF2FF091003090E2958381FFB1
:10EF400006C0E0910130F091023090E2958380FF9D
:10EF500006C0E0910330F091043080E2858308958B
:10EF600083FF06C0E091FD2FF091FE2F90E2968383
:10EF700082FF06C0E091FF2FF091003090E296836F
:10EF800081FF06C0E0910130F091023090E296835B
:10EF900080FF06C0E0910330F091043080E2868368
:10EFA00008958091FA39811107C084E00E948F771B
:10EFB00081E08093FA39089584E00E94B07710923E
:10EFC000FA390895CF92DF92EF92FF920F931F9339
:10EFD000CF93DF93C12C26E0D22EC092ED2FD0929A
:10EFE000EE2F30EAE32E36E0F32EE092EF2FF09290
:10EFF000F02F00E816E00093F12F1093F22FC0E6F7
:10F00000D6E0C093F32FD093F42FC092F52FD09277
:10F01000F62FC093F72FD093F82F0093F92F10936A
:10F02000FA2FE092FB2FF092FC2F2DEC3CEC4CEDF4
:10F0300050E40E9470D7C092FD2FD092FE2FE09234
:10F04000FF2FF092003018164CF4C0930130D0938B
:10F050000230009303301093043008C00093013055
:10F0600010930230C0930330D0930430DF91CF91DE
:10F070001F910F91FF90EF90DF90CF9008950E9425
:10F0800017D360E070E080E091E40E94E2770C9496
:10F0900036D381E08093033A089520E093E088ED31
:10F0A00008B618BE84BF909380002091820021FD95
:10F0B000FCCF08BEFFCF8091033A81110E944D78AA
:10F0C00083E008958091043A882341F0F89461E048
:10F0D00089E790E00E9419D382E0089583E00895C3
:10F0E000CF93DF93CDB7DEB7AD97CDBFDEBF21E2C3
:10F0F000E5EEF1E2DE01119601900D922A95E1F71D
:10F1000022E02093CA01DE019296E8E0F0E024912B
:10F110002D933196EE30F105D1F72DE228A7E0E1ED
:10F12000F0E0E491EF7121E030E02C0F3D1F2E0F55
:10F13000311DF901208129A7E2E1F0E0E491EF71AE
:10F140009E012E0F311DF90121812AA7E4E1F0E093
:10F15000E491EF719E012E0F311DF90121812BA742
:10F160001CA61092CA0125E0FC012783BE016E5D3A
:10F170007F4F0E94A7618093F63CAD96CDBFDEBF66
:10F18000DF91CF91089581E08093043A80E0089563
:10F19000CF93DF93EC0120E030E040E051E469855B
:10F1A0007A858B859C850E9470D718166CF0CE01ED
:10F1B0000E94D05E69857A858B859C850E94E27766
:10F1C0000E9440BC80E001C08DE6DF91CF910895A0
:10F1D00064E87BE30C94CBC166E67BE30C94CBC183
:10F1E00067E47BE30C94CBC169E27BE30C94CBC175
:10F1F00065E17BE30C9476C1CF93DF938AEC96E4D0
:10F200009F938F93CEEAD9E589818F9388818F93DD
:10F210000E9447E284E994E49F938F9389818F93BE
:10F2200088818F930E9447E28CE094E49F938F93B0
:10F2300089818F9388818F930E9447E282E493E4CF
:10F240009F938F9389818F9388818F930E9447E248
:10F250000E9402A88DB79EB740968DBF9EBF80E0EA
:10F26000DF91CF910895CF93DF938DE193E49F9346
:10F270008F93CEEAD9E589818F9388818F930E94FD
:10F2800047E28FEA91E49F938F9389818F938881DE
:10F290008F930E9447E284E290E49F938F93898149
:10F2A0008F9388818F930E9447E28CE094E49F9330
:10F2B0008F9389818F9388818F930E9447E282E4A4
:10F2C00093E49F938F9389818F9388818F930E947A
:10F2D00047E28DB79EB744968DBF9EBF80E0DF9119
:10F2E000CF910895CF93DF9383E090E49F938F9322
:10F2F000CEEAD9E589818F9388818F930E9447E276
:10F3000085E89CE39F938F9389818F9388818F9366
:10F310000E9447E282E493E49F938F9389818F93C5
:10F3200088818F930E9447E28DB79EB70C968DBF60
:10F330009EBF80E0DF91CF910895CF93DF938DE55D
:10F340009CE39F938F93CEEAD9E589818F9388813F
:10F350008F930E9447E28CEE9BE39F938F9389816A
:10F360008F9388818F930E9447E282E493E49F9376
:10F370008F9389818F9388818F930E9447E28DB705
:10F380009EB70C968DBF9EBF80E0DF91CF91089510
:10F39000CF93DF9389EC9BE39F938F93CEEAD9E5DC
:10F3A00089818F9388818F930E9447E280EA9BE353
:10F3B0009F938F9389818F9388818F930E9447E2D7
:10F3C00082E493E49F938F9389818F9388818F93B5
:10F3D0000E9447E28DB79EB70C968DBF9EBF80E01E
:10F3E000DF91CF9108952F923F924F925F926F924B
:10F3F0007F928F929F92AF92BF92CF92DF92EF92C5
:10F40000FF920F931F93CF93DF93CDB7DEB76A9729
:10F41000CDBFDEBF5C010E94E7602C011F86188A09
:10F42000198A1A8AF50101900020E9F73197EA1943
:10F43000FB09E130F24008F002C2D5018C9188232B
:10F4400059F17501BFEFEB1AFB0A850120E021118C
:10F4500015C0883229F08132C8F08F37B9F001C069
:10F4600021E06801EFEFCE1ADE0A90E02A8F0E94B9
:10F4700051E1D8018C9386012A8D08C021E08932A0
:10F4800009F420E0F80180830F5F1F4FD7018D91B1
:10F490007D018111DCCF01C08501F801108210923D
:10F4A000F63CFDE19F2EAAE36A2EA2E27A2E812C81
:10F4B000B6E02B2E03C09A9409F49CC18BE79CE222
:10F4C000A2E2B0E08B879C87AD87BE876B8A7C8A7F
:10F4D0008D8A8DE79CE2A2E2B0E08F839887A987AE
:10F4E000BA87E6E0F2E2DE011196822D01900D92DC
:10F4F0008A95E1F7C2010E94EE5F8501075F1F4F09
:10F5000075019FEFA91AB90AD7016C9170E0CE017D
:10F510000B960E94AEE1892B21F487010E5D1F4FEF
:10F5200004C0A016B10661F793C16501BFEFAB1A25
:10F53000BB0AF601608170E0CE0143960E94AEE105
:10F54000892B91F0D6011D928D0192012F5E3F4FC4
:10F55000288F398F46E050E0B701C9010E94D9E1F8
:10F560003AE0C30ED11C04C0A016B106F1F670C17A
:10F570005801D8013D908D01E32CF12CC7010E9468
:10F5800035E1892B59F4B701CE0101960E94AEE115
:10F59000892B21F40C151D0559F75AC18501BEE6CA
:10F5A0003B1641F0E2E23E120CC0D50111968C915F
:10F5B0008232A9F5F201178211861286138614860B
:10F5C000A3C0B0E3EB1AF108EAE0EE16F10418F07C
:10F5D000FDE23F1217C0BE016A5E7F4FC5010E9467
:10F5E000D8DDD20119966D937D938D939C931C97D2
:10F5F0008E899F898A159B0509F42DC1E4E0179631
:10F60000EC9382C0FBE73F124FC0E7E0D2011796B0
:10F61000EC93FFEFAF1ABF0AE2E0FE2E95C02FEF8A
:10F62000A21AB20AE5E0D2011796EC9362E270E00A
:10F63000C5010E94AEE18E8B9F8B009709F408C133
:10F64000DC011C92F50101900020E9F73197EA19DD
:10F65000FB093397C8F0F80181818033A9F48281D6
:10F66000883791F440E050E060E070E0C5010E940E
:10F6700049DFD20119966D937D938D939C931C97CE
:10F6800083E017968C9308C0B501C2010E94A76160
:10F690008093F63C811153C0AE88BF88BFEFAB1A90
:10F6A000BB0AAE8ABF8A30C0E4E73E120EC0E1E07A
:10F6B000D2011796EC9380E090E0A0E8BFE3F2015E
:10F6C00081879287A387B4871FC0F6E63F120CC0DC
:10F6D000E1E0D2011796EC93179719961D921D92AF
:10F6E0001D921C921C9710C0BBE53B12B1C0F201E9
:10F6F0002782B501C2010E94A7618093F63C811167
:10F700001EC077E6F72E7DC0BE01695F7F4FC50141
:10F710000E94F3E15C01009709F49AC0DC018C912E
:10F720008D3729F411968C91F50131965F018C3259
:10F7300009F48BC0FFEFAF1ABF0AF12C05C0F82EF9
:10F7400022E0281708F45DC08F858201035F1F4FF8
:10F75000882341F043E050E0BE01615F7F4FC80164
:10F760000E94D9E1688D798DC8010E94475FD2015E
:10F7700014968D939C9315978F3FBFEF9B07B9F11C
:10F780000E947E64882371F0888D998D0E94305F7D
:10F79000882341F043E050E0688D798DCE010F96CB
:10F7A0000E94D9E1F201428053804114510411F1C9
:10F7B000F11081CE80918E34811108C087E894E3E6
:10F7C0000E94E35B8093F63CF82E1BC080912B32A5
:10F7D000823099F087E894E30E94B95B8093F63C0D
:10F7E00081110EC087E894E30E94365C0AC064E68B
:10F7F000F62E07C050E7F52E04C04BECF42E01C0E6
:10F80000F82E42E060E08F2D0E944E6281E00E945F
:10F8100061AA6A96CDBFDEBFDF91CF911F910F9194
:10F82000FF90EF90DF90CF90BF90AF909F908F9020
:10F830007F906F905F904F903F902F9008958BE650
:10F840008093F63C3BE6F32EDCCF22E0F22E7CCF19
:10F850009FE6F92ED6CF86E6F82ED3CF2F923F9291
:10F860004F925F926F927F928F929F92AF92BF92D0
:10F87000CF92DF92EF92FF920F931F93CF93DF937C
:10F8800000D000D0CDB7DEB78C0169837A834B837B
:10F890005C835A0128E0A21AB108A60EB71EDC014B
:10F8A00016967C907B01BFEFEB1AFB0A8BE7FB01FE
:10F8B000808380E0912C95E0692E20E1422E22E2A7
:10F8C000522E3CE0232E32E2332E4DE7842EED8281
:10F8D000FE82D80117969C919F3F09F429C1882385
:10F8E00039F02CE2ED81FE8120833196ED83FE8399
:10F8F0008091A03C811119C0C80141969F938F93BC
:10F900003F922F923E813F938D818F930E9412E30D
:10F91000AD81BE81A80FB91FAD83BE830F900F903C
:10F920000F900F900F900F9018C0C80141969F93B1
:10F930008F935F924F92BE81BF93ED81EF930E94B0
:10F9400012E32D813E81280F391F2D833E830F90B6
:10F950000F900F900F900F900F90D80117968C91E9
:10F960001797843059F51996CD90DD90ED90FC9065
:10F970001C97A7019601C701B6010E9433D98111D6
:10F9800017C0E894F7F82FEF3FEF4FE75FE7C701A5
:10F99000B6010E9433D9811121C12FEF3FEF4FE70C
:10F9A0005FE7C701B6010E946DD518160CF016C1AD
:10F9B000F801118612861386148610C1811113C0B6
:10F9C000E6E1F2E2AD81BE81862D01900D928A952D
:10F9D000E1F72D813E812C5F3F4F2D833E83D8017F
:10F9E00017968C9199C0823061F4F80184858F93C9
:10F9F00083858F9382858F9381858F93ABE1B2E26C
:10FA000014C0833029F5D8011C968C911C978F93D4
:10FA10001B968C911B978F931A968C911A978F93A4
:10FA200019968C918F93A1E2B2E2BF93AF93FE81BE
:10FA3000FF932D812F930E9412E3AD81BE81A80F09
:10FA4000B11DAD83BE83F8018781CDBFDEBF64C029
:10FA5000853059F4D80158968C9158978F935796C2
:10FA60008C918F93A9E2B2E20CC0863009F5D801DF
:10FA700058968C9158978F9357968C918F93AEE2AE
:10FA8000B2E2BF93AF93FE81FF932D812F930E942B
:10FA900012E3AD81BE81A80FB11DAD83BE83F80115
:10FAA00087810F900F900F900F900F900F9034C0A0
:10FAB000813091F52CEA35EC47E257E3D8011996ED
:10FAC0006D917D918D919C911C970E946DD587FFC2
:10FAD00012C0E3E3F2E2AD81BE8186E001900D92B7
:10FAE0008A95E1F7ED81FE813596ED83FE83D8019D
:10FAF00017968C9111C0E9E3F2E2AD81BE81862DAB
:10FB000001900D928A95E1F7ED81FE813496ED83A7
:10FB1000FE83D80117968C91873049F42BE7ED814D
:10FB2000FE8120833196ED83FE8380E001C081E079
:10FB3000AD81BE81AA15BB0518F08FEF9FEF65C0A0
:10FB4000F801028113810115110549F0D8011696BB
:10FB50009C912FEF290D99153CF0992EBACEED808E
:10FB6000FE807914B4F020C0ED81FE81D801CF0170
:10FB70000196808216969C9016973FEF320F921650
:10FB80001CF4232FFC01F3CF8D839E838D0181E034
:10FB9000A0CEF7012DE7CF01019620839A94791426
:10FBA00014F4FC01F8CF7C018DE79AE0A0E0F701A6
:10FBB00080839183A283F2E0EF0EF11C89819A8108
:10FBC0002B813C81820F931F8E159F0508F4B5CFC2
:10FBD000C701A981BA818A1B9B0B17C0C8010E946B
:10FBE0008E64F801418552856385748520858D81F9
:10FBF0009E810E940FC42D813E81280F311D2D83CF
:10FC00003E83D80117968C9187CF2696CDBFDEBF55
:10FC1000DF91CF911F910F91FF90EF90DF90CF90E8
:10FC2000BF90AF909F908F907F906F905F904F901C
:10FC30003F902F90089540E052E06CE17AE30E94FB
:10FC40002E7C6091AE597091AF598CE19AE30C947F
:10FC500096E2EF92FF920F931F93CF93DF93CDB76E
:10FC6000DEB76297CDBFDEBFF82E90919E3C992300
:10FC700009F4B2C08FE6F81212C00E94E7606CE18E
:10FC80007CE38091163A9091173A0E94EFC3BC0131
:10FC90008CE091E20E94056207E814E34AC080917B
:10FCA0002B3207E814E3882309F443C0EE24EA94D6
:10FCB000C8010E94AE5F8823E1F1823029F480916F
:10FCC000A53C811120C01DC0843029F48091A23C44
:10FCD000811119C016C08530B1F48091A43C8823ED
:10FCE00081F0F80181859285A385B485BC01CD01A1
:10FCF0009F772CEA35EC47E257E30E946DD587FFEA
:10FD000002C0F801E782F801028113810115110593
:10FD100079F60FC0F801028113810115110549F42C
:10FD200040E052E06CE17AE38EE694E30E942E7CA0
:10FD300053C0F80197819F3F69F78091E52F8111AA
:10FD40001AC08091193A8F938091183A8F931F921D
:10FD5000FF928EE392E29F938F93CE0101967C01F6
:10FD6000FF928F930E9412E31092183A1092193A60
:10FD7000CDBFDEBF13C00E940EC91F928F931F928A
:10FD8000FF9286E492E29F938F93CE0101967C01CD
:10FD9000FF928F930E9412E3CDBFDEBFB701C8016F
:10FDA0000E94A761F801168286E0878386E690E0CC
:10FDB000818B928B1282138240E052E06CE17AE3F5
:10FDC0008EE694E30E942E7C6091AE597091AF59FB
:10FDD0008CE19AE30E9496E26296CDBFDEBFDF918E
:10FDE000CF911F910F91FF90EF900895613019F01E
:10FDF000623029F0089587E894E30C941B7E0C94FC
:10FE0000297ECF92DF92EF92FF92FC01C184D284CF
:10FE1000E384F48420E030E040EA50E4C701B60116
:10FE20000E9470D718160CF453C0C701B6010E9487
:10FE3000E1D560939E3C1092A13C1092A23C10929E
:10FE4000A33C1092A43C1092A53C20E030E040E896
:10FE50005FE3C701B6010E9470D787FD03C081E050
:10FE60008093A13C20E030E040E050E4C701B601BF
:10FE70000E9470D787FD03C081E08093A23C20E000
:10FE800030E040E450E4C701B6010E9470D787FD1E
:10FE900003C081E08093A33C20E030E040E850E4E0
:10FEA000C701B6010E9470D787FD03C081E080932F
:10FEB000A43C20E030E040EA50E4C701B6010E94D3
:10FEC00070D787FD07C081E08093A53C80E003C028
:10FED0008EE601C080E0FF90EF90DF90CF90089514
:10FEE0006CE677E40C948CC165E177E40C948CC1EA
:10FEF00061EE76E40C948CC1BF92CF92DF92EF92C8
:10FF0000FF920F931F93CF93DF93CDB7DEB7689720
:10FF1000CDBFDEBF6B0128E1FC01DE01119601902F
:10FF20000D922A95E1F78CEEE82E80E3F82E8E01F3
:10FF30000F5F1F4FB12CF7018081823029F4F80147
:10FF40001082118212821382809130588B1114C05A
:10FF5000209143583091445840914558509146580B
:10FF6000F80160817181828193810E9412D8F6012B
:10FF7000608371838283938380914F588B1114C067
:10FF8000209162583091635840916458509165585F
:10FF9000F80160817181828193810E9412D8F601FB
:10FFA000648375838683978380916E588B1114C008
:10FFB00020918158309182584091835850918458B3
:10FFC000F80160817181828193810E9412D8F601CB
:10FFD000608771878287938780918D588B1114C0B9
:10FFE0002091A0583091A1584091A2585091A35807
:10FFF000F80160817181828193810E9412D8F6019B
:020000021000EC
:100000006487758786879787B394F5E3EF0EF11CB5
:100010000C5F1F4F86E0B8128ECF6896CDBFDEBF53
:10002000DF91CF911F910F91FF90EF90DF90CF90D4
:10003000BF900895F8940E943F780E9471800E94BA
:1000400036D30E94BDC50E94FBB20E94C16F0E94C0
:1000500040BC0E9459A540E060E080E00E947365CA
:100060000E9424610E945F800E9463820E94734FFD
:100070000E942ED38091A20084608093A200809180
:10008000A20082608093A2008091A2008160809390
:10009000A20078940E9402A80E944DBD0E94DA65D9
:1000A000FDCFE82FF0E0EE0FFF1FE856F84B65910B
:1000B00074914FE450E086EA9CE30C9480E18091D7
:1000C000F739823041F440E060E081E00E947365DE
:1000D00080E00E9402670C9407CA682F81E00C94AC
:1000E000D8C61092F73C1092F83C1092F93C10924E
:1000F000FA3C0895CF93DF93EC018C819D81880FAA
:10010000991F880F991F2091F93C3091FA3C820F7A
:10011000931F8093FB3C9093FC3C44E050E061E0F3
:100120007DE30E942ED24091013D5091023D6091AD
:10013000033D7091043D49875A876B877C8780E037
:10014000DF91CF9108958F929F92AF92BF92CF92FD
:10015000DF92EF92FF92CF93DF93EC0180912C32EC
:10016000882369F089E0DF91CF91FF90EF90DF90D5
:10017000CF90BF90AF909F908F900C948CA7898563
:100180009A85AB85BC858093FD3C9093FE3CA09303
:10019000FF3CB093003DCE010E947A808093F63CF4
:1001A00081116EC0C984DA84EB84FC84A7019601B6
:1001B000C701B6010E9433D981112FC046015701F2
:1001C000E894B7F82FEF3FEF4FE75FE7C501B401C1
:1001D0000E9433D981110AC02FEF3FEF4FE75FE74D
:1001E000C501B4010E946DD51816BCF08090FD3C8D
:1001F0009090FE3CA090FF3CB090003DA501940182
:10020000C701B6010E94C4D39F772CEA35EC47E2C0
:1002100057E30E9470D7181674F58091FD3C9091B9
:10022000FE3CA091FF3CB091003D8093013D909336
:10023000023DA093033DB093043D8C819D81880FC6
:10024000991F880F991F2091F93C3091FA3C820F39
:10025000931F8093FB3C9093FC3C44E050E061E0B2
:100260007DE30E94BFD28090FD3C9090FE3CA09028
:10027000FF3CB090003D89869A86AB86BC8680E0C4
:10028000DF91CF91FF90EF90DF90CF90BF90AF9034
:100290009F908F9008950E9456B880E008958091B5
:1002A000053D9091063D8F3E924111F08EE50895F7
:1002B00080912B3D90912C3D8F3E9241B9F78091DA
:1002C0002D3D90912E3D8F3E924181F78091B65405
:1002D0009091B7548F3E924149F78091B8549091D4
:1002E000B9548F3E924111F780914B5690914C56E4
:1002F0008F3E9241D9F680E0089594E0899FF00105
:100300001124EB5FF24C4283538364837583089519
:1003100094E0899FF0011124E854FB4A45AB56ABA9
:1003200067AB70AF08955F926F927F928F929F92AA
:10033000AF92BF92CF92DF92EF92FF920F931F93F3
:10034000CF93DF93CDB7DEB76097CDBFDEBFBE01E1
:100350006F5F7F4F8DEE94E50E947C7FCE0101960A
:100360004C0185E6A82E85E5B82E95E7C92E95E5C2
:10037000D92E25E8E22E25E5F22E05EA15E537EC23
:10038000632E38E5732E512CF40141915191619106
:1003900071914F01F50141935193619371935F0105
:1003A000F60141935193619371936F01F70141936A
:1003B0005193619371937F01852D0E94E36FF80142
:1003C00011921192119211928F01F30110821182F8
:1003D000128213825394F8E16F0E711C84E058125C
:1003E000D3CF6096CDBFDEBFDF91CF911F910F912C
:1003F000FF90EF90DF90CF90BF90AF909F908F9045
:100400007F906F905F90089580912F3D08951F9386
:10041000CF93DF938BE897E1EDE2FDE3DF019C01F1
:100420001D9221503040E1F78FEE92E180932D3DF7
:1004300090932E3D8093B6549093B754C6E3DDE37A
:10044000C093303DD093313DC093323DD093333D86
:10045000C093343DD093353D81E090E06AEF73E581
:1004600020E030E01CEB129FA001139F500D1124DF
:10047000FA01E35DF24CD90111961A9F90011B9F7E
:10048000300D11242A5C324C2387348761877287B0
:10049000BA016A5C724C9C0101968032910519F791
:1004A0008CEB829FF001839FF00D1124E35DF24CF1
:1004B000C387D4876187728780E280932F3DDF9165
:1004C000CF911F910895CF93DF93E8EBF4E585E991
:1004D00091E0DF01EC011D922197E9F7A5E0BDE372
:1004E00088E2ED0119928A95E9F78FEE92E18D93FA
:1004F0009C9380932B3D90932C3D8083918380939C
:100500004B5690934C56DF91CF910C9407820E94EA
:10051000808C0E94078280E00C94304AE091303D4C
:10052000F091313D848581111BC02281338180810E
:1005300091814CEBDF011D924A95E9F722833383C9
:100540008083918381E0848780912F3D81508093C7
:100550002F3D828193818093303D9093313D05C042
:100560008CE10E948CA7E0E0F0E0CF010895A2E3C7
:10057000BDE3ED91FC911197858781E0878782E04B
:100580008487828193818D939C9381E00E94B2AB9A
:100590000C949CB5EF92FF920F931F93CF93DF9330
:1005A00000D01F92CDB7DEB78C014B835C8369838B
:1005B0007A830E948E82FC014B815C8169817A8101
:1005C000009761F48EE02496CDBFDEBFDF91CF911E
:1005D0001F910F91FF90EF900C946F4E83E08587F1
:1005E0008BE491E884839583068317838B017A01DA
:1005F00026E0D8014D915D916D917D918D01CF01E6
:1006000085599F4FDC014D935D936D937C931397B8
:10061000D7014D915D916D917D917D01418B528B03
:10062000638B748B215034962111E3CF83E02496A1
:10063000CDBFDEBFDF91CF911F910F91FF90EF9063
:100640000C94B782CF92DF92EF92FF926B017C0104
:100650000E948E82009739F48EE0FF90EF90DF9039
:10066000CF900C946F4E25EA33E8FC012483358348
:10067000E556FF4FC082D182E282F38221E0FC0185
:10068000278782E00E94B78280E0FF90EF90DF90A2
:10069000CF9008958091343D9091353DFC012485A3
:1006A0003EEF320F323018F424E0248708952430CE
:1006B00011F080E090E00895E091343DF091353DF7
:1006C00022813381808191814CEBDF011D924A951B
:1006D000E9F72283338380839183E091343DF09165
:1006E000353D0280F381E02DE093343DF093353DBC
:1006F0008485823011F483E0848780912F3D8F5F61
:1007000080932F3D8FEF0E94B2AB81E04091303D4E
:100710005091313D2091343D3091353D4217530782
:1007200009F080E00895BC016F5E7F4FDC011696F2
:10073000ED91FC91179785599F4F19950E945C8305
:1007400081110E94DD5580E0089585569F4F20E07D
:1007500034E244E759E4FC01608171818281938134
:100760000E9412D80E94E1D50E940DD60E9460B866
:100770000E945C8381110E94DD5580E00895809184
:10078000343D9091353DFC0124853EEF320F3230EF
:1007900018F424E024870895243011F080E090E0DC
:1007A0000895CF93DF93C091343DD091353D8C8532
:1007B0009EEF980F923018F484E08C8705C0843047
:1007C00019F080E090E010C02097D9F3DE01129676
:1007D000ED91FC9113978785882329F0EC17FD078D
:1007E00011F0DF01F4CFCD01DF91CF910895CF93C8
:1007F000DF93EC012A813B81888199814CEBFB01DD
:10080000DE0101900D924A95E1F72A833B838883AC
:100810009983DF91CF9108958FEE92E180934D56A9
:1008200090934E5680930A5790930B5708952F92AA
:100830003F924F925F926F927F928F929F92AF9270
:10084000BF92CF92DF92EF92FF920F931F93CF93BD
:10085000DF93CDB7DEB76A97CDBFDEBF4C011B017A
:1008600029013A01E986FA860B871C871A2D0B2D80
:10087000E8A8B9A8AAA82BA929838091A432882323
:1008800099F08091983290919932A0919A32B091DA
:100890009B32BC01CD019F772CEA35EC47E257E350
:1008A0000E946DD587FD11C78091CF339091D033D1
:1008B000A091D133B091D233BC01CD019F7731E00B
:1008C0003D832CEA35EC47E257E30E9470D71816B7
:1008D00014F01D8210C02DEC3CEC4CEC5DE36091FB
:1008E00074337091753380917633909177330E9491
:1008F0006DD587FDECC6F10180819181A281B38124
:10090000BC01CD019F77F1E0FD872CEA35EC47E291
:1009100057E30E9470D718160CF01D86F1018481F0
:100920009581A681B781BC01CD019F77F1E0F98B5C
:100930002CEA35EC47E257E30E9470D718160CF00A
:10094000198AF10180859185A285B3852091D333E1
:100950003091D4334091D5335091D6332E8B3F8B89
:10096000488F598F2091D7333091D8334091D93364
:100970005091DA332A8B3B8B4C8B5D8B4091DB3370
:100980005091DC336091DD337091DE33F090A5320D
:10099000F11021C01092955681E08093965682E026
:1009A000809397563D81332341F04D85411195C683
:1009B0005989511192C68CE9C1C6CB01BA019F7702
:1009C0002CEA35EC47E257E30E9470D718160CF07A
:1009D00089C68BE9B3C6BC01CD019F77A1E0AA8F80
:1009E0002CEA35EC47E257E30E9470D718160CF05A
:1009F0001A8EB1E0FB1216C01092955682E08093D9
:100A00009656F0929756ED81EE2339F0FD85F1115F
:100A100064C62A8D222379F260C66A897B898C8913
:100A20009D89CDCF32E0F31217C081E080939556B7
:100A3000F0929656109297564D81442341F0598971
:100A400051114BC68A8D882309F4B5CF46C66E89ED
:100A50007F89888D998DB3CFB101C4010E947F4CED
:100A60009D81992309F451C0209160323091613207
:100A700040916232509163326091B5327091B632DA
:100A80008091B7329091B8320E94C4D39F772CEAFC
:100A900035EC47E257E30E946DD587FF36C02091C1
:100AA0006432309165324091663250916732609184
:100AB000B9327091BA328091BB329091BC320E94AF
:100AC000C4D39F772CEA35EC47E257E30E946DD5FB
:100AD00087FF1BC0209168323091693240916A32A1
:100AE00050916B326091BD327091BE328091BF32B5
:100AF0009091C0320E94C4D39F772CEA35EC47E234
:100B000057E30E946DD587FDE4C58CA980935F32C1
:100B10008BE592E30E94874A86E5EBE5F2E3A4EBDE
:100B2000B6E501900D928A95E1F788E1E5EBF2E3F5
:100B3000A0E5B6E501900D928A95E1F78091A63285
:100B40008111D5C523E333E34BEC51E46E2D7B2DAE
:100B50008A2D99810E9412D84B015C0160938056C6
:100B600070938156809382569093835623E333E3A8
:100B70004BEC51E4C301B2010E9412D86093685655
:100B80007093695680936A5690936B5623E333E3D0
:100B90004BEC51E469857A858B859C850E9412D83F
:100BA00060936C5670936D5680936E5690936F560B
:100BB00023E333E34BEC51E4612F702FC6010E9415
:100BC00012D8162F072F412F502FBC01409370567B
:100BD0005093715660937256709373568091703330
:100BE00090917133A0917233B0917333BC01CD01F8
:100BF0009F770E944AD60E94E1D5609391567093E8
:100C000092568093935690939456A0919556A98BA3
:100C1000B0919656BA8BEB2FF0E0ED83FE837F0107
:100C2000EE0CFF1CEE0CFF1CF101EE0DFF1D808190
:100C30009181A281B381BC01CD019F772CEA35EC73
:100C400047E257E30E946DD5D82EDD1CDD24DD1C64
:100C50003989232F30E029833A838901000F111F3E
:100C6000000F111FF101E00FF11F80819181A2811E
:100C7000B381BC01CD019F772CEA35EC47E257E305
:100C80000E946DD5881F8827881F8D2180939056DC
:100C90002CEA35EC47E257E3C501B4019F770E9487
:100CA00070D718160CF0F9C0F801E05AFD4CD801C5
:100CB000AB54BD4C2D913D914D915C916081718102
:100CC000828193810E94C4D36B017C01ED81FE81FE
:100CD000EE0FFF1FEE0FFF1FE05AFD4CAD81BE81EE
:100CE000AA0FBB1FAA0FBB1FAB54BD4C2D913D914A
:100CF0004D915C9160817181828193810E94C4D306
:100D000069877A878B879C87A5019401C501B40107
:100D10000E9412D820E030E040E850E40E9412D84F
:100D20006D877E878F87988BA7019601C701B601D3
:100D30000E9412D82B013C0129853A854B855C85A0
:100D4000CA01B9010E9412D89B01AC01C301B201D2
:100D50000E94C5D39B01AC016D857E858F859889E6
:100D60000E94C4D32B013C0120E030E0A9010E9485
:100D700070D71816C4F4C301B2010E94EBD82B013E
:100D80003C0129853A854B855C85C701B6010E94E7
:100D90007DD79B01AC01C301B20190580E9474D56C
:100DA0002B013C0103C0412C512C320180915F3258
:100DB000833021F477FA709477F8709420E030E073
:100DC000A901C501B4010E946DD587FF04C077FA5F
:100DD000709477F8709409811A81000F111F000F29
:100DE000111FA801435B594A5A01A3019201698569
:100DF0007A858B859C850E9412D89B01AC01C70126
:100E0000B6010E94C4D320E030E040E05FE30E94DE
:100E100012D8D5015B966D937D938D939C935E97CD
:100E2000AD80BE80AA0CBB1CAA0CBB1CF501E35B09
:100E3000F94A4F01A3019201C701B6010E9412D8DD
:100E40009B01AC0169857A858B859C850E94C5D301
:100E500020E030E040E05FE30E9412D8D4015B96CE
:100E60006D937D938D939C935E97E0919756F0E000
:100E7000EE0FFF1FEE0FFF1FE35BF94A138E148E78
:100E8000158E168EB0918056B987E0918156ED8708
:100E9000209082563090835625C05701F701E35BBE
:100EA000F94A838D948DA58DB68D9C01AD01505866
:100EB000F801E35BF94A838D948DA58DB68DBC0155
:100EC000CD0190580E947DD79B01AB01BC0140939E
:100ED000805650938156609382567093835629872B
:100EE0003D871C01D801A35BB94A5B96CD90DD908C
:100EF000ED90FC905E97E981FA81EE0FFF1FEE0FF7
:100F0000FF1FE754F94A13962D913D914D915C9145
:100F1000169760817181828193810E94C4D3A70159
:100F200096010E94C4D369837A838B839C83D50105
:100F3000A35BB94A5B964D905D906D907C905E97F7
:100F4000ED81FE81EE0FFF1FEE0FFF1FE754F94A00
:100F500013962D913D914D915C9116976081718111
:100F6000828193810E94C4D3A30192010E94C4D3C1
:100F70006D837E838F8398879B01AC0169817A8121
:100F80008B819C810E947DD729853D85A1010E948E
:100F9000C4D34B015C01E894B7F820E030E040E8AE
:100FA0005FE3C501B4010E9470D718160CF4C3C3E7
:100FB0002AE037ED43EA5BE3C501B4010E9470D734
:100FC000181694F42FE632E143E85AE369857D85EB
:100FD000C1010E9412D89B01AC01C501B4010E945D
:100FE00070D718160CF4A7C3A30192015058C7017B
:100FF000B60190580E9438D44B015C01609378563A
:101000007093795680937A5690937B568091A5324F
:10101000813039F4412C512C30E8632E3FEB732E94
:1010200006C0412C512C20E8622E2FE3722E8091B5
:1010300090568823D1F1609191567091925680918B
:101040009356909194560E940DD66B017C012CEA28
:1010500035EC47E257E30E946DD587FD10C0109133
:101060005F322BED3FE049EC50E4C701B6010E942E
:1010700012D89B01AC01C12CD12C7601B9C081E002
:1010800090E0A0E0B0E08093915690939256A093A8
:101090009356B093945610915F322BED3FE049EC9C
:1010A00050E4C12CD12C7601A3C02D813E814F810B
:1010B000588569817A818B819C810E9438D46983AB
:1010C0007A838B839C8360937C5670937D56809348
:1010D0007E5690937F56A50194010E94C4D36B0164
:1010E0007C019F772CEA35EC47E257E30E946DD5EF
:1010F00087FF18C010915F3260919156709192569F
:1011000080919356909194560E940DD62BED3FE01E
:1011100049EC50E40E9412D89B01AC01C12CD12CA7
:10112000760166C029813A814B815C81C501B40199
:101130000E9470D71816F4F42BED3FE049EC50E410
:10114000C301B2010E9412D89B01AC0169817A816E
:101150008B819C810E94C5D360937C5670937D5691
:1011600080937E5690937F56A50194010E94C4D32C
:101170006B017C0110915F32133099F060919156B0
:101180007091925680919356909194560E940DD6EC
:101190002BED3FE049EC50E40E9412D89B01AC01DA
:1011A00027C02BED3FE049EC50E4C301B2010E949F
:1011B00012D89B01AC01C701B6010E94C4D37B01C8
:1011C0008C016091915670919256809193569091B6
:1011D00094560E940DD62BED3FE049EC50E40E945E
:1011E00012D89B01AC01C701D8016C017D010BC075
:1011F000123049F4C301B2010E9412D8A70196012E
:101200000E94C5D30AC0C301B2010E9412D89B013B
:10121000AC01C701B6010E94C4D37B01AB01BC0184
:1012200040938456509385566093865670938756A4
:101230008C0150909756A52DB0E0FD01EE0FFF1FD9
:10124000EE0FFF1FE754F94AAA0FBB1FAA0FBB1FDF
:10125000A35BB94A13962D913D914D915C911697E0
:1012600060817181828193810E94C4D34B015C01B2
:10127000609388567093895680938A5690938B56C4
:101280009701A80169857D85C1010E9412D86B0173
:101290007C0160938C5670938D5680938E569093FC
:1012A0008F56A50194010E947DD769837A838B8331
:1012B0009C83609374567093755680937656909382
:1012C00077568091A432811117C0F0919832FD8336
:1012D0004090993220919A322E8B30919B323A8FE6
:1012E000109298321092993210929A3210929B3248
:1012F00081E08093A43212C02091983230919932CB
:1013000040919A3250919B3269817A818B819C8184
:101310000E9474D56D83472E8E8B9A8F598945E331
:10132000549FF0011124E351FF4C2081318142810F
:101330005381C701B6010E9474D5662E072F182F5E
:10134000792E2D81342D4E895A8D0E946DD587FFBF
:1013500004C06D80042D1E897A8C9A8985E3989F3C
:10136000F0011124E351FF4C2081318142815381EE
:10137000C701B6010E9474D56B017C019B01AC01D1
:10138000662D702F812F972D0E9470D7181624F08C
:101390006C2C0D2D1E2D7F2C862D902FA12FB72D5F
:1013A0008093985690939956A0939A56B0939B56D3
:1013B00020E030E0A901C501B4019F770E9470D7F9
:1013C000181684F5A5E35A9EF0011124E351FF4C51
:1013D0002081318142815381C501B4010E9474D5BD
:1013E0004B015C01E894B7F8A5019401662D702FBC
:1013F000812F972D0E9470D7181614F4A72C04C0C3
:10140000682C092D1A2DAB2C862D902FA12FBA2DCB
:101410008093985690939956A0939A56B0939B5662
:10142000B62C02C0B62CA72CC0902E30D0902F30F6
:10143000E0903030F090313020E030E040E850E48F
:10144000C701B6010E9412D82B013C0129853D85B8
:10145000A10169857D85C1010E94C5D3A7019601BF
:101460000E94C4D39B01AC01C301B2010E9412D8F7
:101470000E94EBD82B013C0120EC31EE44E65CE409
:101480006B2D702F812F9A2D0E9412D820E030E40E
:101490004CE156E40E9474D56B017C0120913730F9
:1014A000309138304091393050913A3069817A81A9
:1014B0008B819C810E9474D54B015C01A301920138
:1014C00069817A818B819C810E9474D58701760124
:1014D000A50194010E94F7C20E944AD67B018C01AB
:1014E00020E030E040E85FE30E9470D718163CF43B
:1014F000B701C8010E94DCD54B015C0108C0812CFA
:10150000912C54018394E12CF12C00E81FE3C701D6
:10151000D80180939C5690939D56A0939E56B0936D
:101520009F569701A80160919856709199568091A5
:101530009A5690919B560E9474D56093E956709389
:10154000EA568093EB569093EC568092A056909278
:10155000A156A092A256B092A3569701A8016091FD
:1015600084567091855680918656909187560E9438
:1015700074D56093A4567093A5568093A656909305
:10158000A7569701A801609188567091895680915D
:101590008A5690918B560E9474D56093A85670938A
:1015A000A9568093AA569093AB5680907856909007
:1015B0007956A0907A56B0907B56C501B4010E942E
:1015C000E1D8C0908056D0908156E0908256F0903D
:1015D00083560091955610E0000F111F000F111F48
:1015E000035B194AA70196010E9412D89B01AC0126
:1015F000F80163817481858196810E94C4D36093D0
:10160000AC567093AD568093AE569093AF56C501CD
:10161000B4010E9471D59B01AC010091965610E077
:10162000000F111F000F111F035B194AC701B601FC
:101630000E9412D89B01AC01D80113966D917D9147
:101640008D919C9116970E94C4D36093B05670936D
:10165000B1568093B2569093B356A0919756B0E08E
:10166000FD01EE0FFF1FEE0FFF1FE754F94AAA0F0F
:10167000BB1FAA0FBB1FA35BB94A13968D919D9107
:101680000D90BC91A02D80839183A283B38310928F
:10169000F63C8091745690917556A0917656B09113
:1016A0007756BC01CD019F772CEA35EC47E257E332
:1016B0000E946DD587FD0FC00E94D05582E08093B7
:1016C0004F560E94E24B80E039C08EE837C08EE969
:1016D00035C08FE933C089EC31C0B101C4010E942B
:1016E0007F4CC2C9B101C4010E947F4C0ECA8E2D2D
:1016F0009B2DAA2DB9818093805690938156A093FB
:101700008256B093835640926856509269566092C2
:101710006A5670926B5629853A854B855C85209375
:101720006C5630936D5640936E5650936F564C01E5
:101730005D01C60148CA8BE98093F63C6A96CDBF2D
:10174000DEBFDF91CF911F910F91FF90EF90DF905F
:10175000CF90BF90AF909F908F907F906F905F9051
:101760004F903F902F9008958F929F92AF92BF928B
:10177000CF92DF92EF92FF92CF93DF9380914F56FB
:10178000882309F4B1C00E940482843010F482E0FE
:10179000ACC02091A4563091A5564091A6565091C8
:1017A000A756609178567091795680917A569091AB
:1017B0007B560E94C5D36B017C0160937856709371
:1017C000795680937A5690937B560E94E1D8809008
:1017D000805690908156A0908256B0908356C091CA
:1017E0009556D0E0CC0FDD1FCC0FDD1FC754D94A72
:1017F000A50194010E9412D89B01AC016091AC56E6
:101800007091AD568091AE569091AF560E94C5D35F
:10181000688379838A839B83C701B6010E9471D54F
:101820009B01AC01C0919656D0E0CC0FDD1FCC0FD0
:10183000DD1FC754D94AC501B4010E9412D89B01CB
:10184000AC016091B0567091B1568091B2569091B2
:10185000B3560E94C5D3688379838A839B83C091E2
:101860009756D0E0CC0FDD1FCC0FDD1FC754D94AEF
:101870002091A8563091A9564091AA565091AB5646
:10188000688179818A819B810E94C5D3688379832D
:101890008A839B8384EB96E50E94969688E1E9EB28
:1018A000F6E5A0E5B6E501900D928A95E1F7809105
:1018B000A0569091A156A091A256B091A35601971F
:1018C000A109B1098093A0569093A156A093A25666
:1018D000B093A356181619061A061B060CF457CF18
:1018E00010924F5680E001C083E0DF91CF91FF90CE
:1018F000EF90DF90CF90BF90AF909F908F90089522
:1019000010924F5608954F925F926F927F928F92EE
:101910009F92AF92BF92CF92DF92EF92FF92CF93BE
:10192000DF93CDB7DEB76497CDBFDEBF69837A831F
:101930008B839C8369017A0120E030E040E751E429
:101940000E9412D84B015C0120E030E040E751E4F6
:10195000C701B6010E9412D89B01AC01C501B401B8
:101960000E94C4D36D877E878F87988B20E030E0FC
:1019700040E251EC69817A818B819C810E9412D86E
:101980004B015C0120E030E040E251E4C701B601C8
:101990000E9412D89B01AC01C501B4010E94C5D3BD
:1019A000698B7A8B8B8B9C8B2091CD553091CE554A
:1019B0004091CF555091D05560E070E080E89FE3B2
:1019C0000E9474D54B015C0120E030E040EC50EC0B
:1019D00069817A818B819C810E9412D82B013C0104
:1019E00020E030E040EC50E4C701B6010E9412D87C
:1019F0009B01AC01C301B2010E94C5D3A5019401B2
:101A00000E9412D8A50194010E9412D8A501940148
:101A10000E9412D8A50194010E9412D8A501940138
:101A20000E9412D86B017C01A50194016D857E8511
:101A30008F8598890E9412D8A50194010E9412D81E
:101A4000A50194010E9412D8A50194010E9412D808
:101A50006D837E838F839887A501940169897A8934
:101A60008B899C890E9412D8A50194010E9412D8EA
:101A7000A50194010E9412D869877A878B879C8779
:101A800020E030E042EF50E4C701B6010E9412D8D6
:101A90002B013C0120E030E040EA50E46D817E8182
:101AA0008F8198850E9412D89B01AC01C301B201BD
:101AB0000E94C5D32B013C0120E030E040E550E41A
:101AC00069857A858B859C850E9412D89B01AC0123
:101AD000C301B2010E94C5D36093F1557093F255D2
:101AE0008093F3559093F45520E030E045EA52E4BA
:101AF000C701B6010E9412D82B013C0120E030E062
:101B000048EE51E46D817E818F8198850E9412D8C4
:101B10009B01AC01C301B2010E94C5D32B013C0162
:101B200020E030E040E151E469857A858B859C8531
:101B30000E9412D89B01AC01C301B2010E94C5D31F
:101B40006093ED557093EE558093EF559093F0555B
:101B500020E030E04FE753E4C701B6010E9412D8FD
:101B60002B013C0120E030E040E452E46D817E81B5
:101B70008F8198850E9412D89B01AC01C301B201EC
:101B80000E94C5D32B013C0120E030E040EC50E442
:101B900069857A858B859C850E9412D89B01AC0152
:101BA000C301B2010E94C5D36093E9557093EA5511
:101BB0008093EB559093EC5520E030E046E953E4F8
:101BC000C701B6010E9412D82B013C0120E030E091
:101BD00040EC51E46D817E818F8198850E9412D8FE
:101BE0009B01AC01C301B2010E94C5D36093E555CE
:101BF0007093E6558093E7559093E85520E030E0E8
:101C000040EF52E4C701B6010E9412D86093E1553B
